:1000000000400020F15F000031600000336000001C
:1000100000000000000000000000000000000000E0
:10002000000000000000000000000000356000003B
:100030000000000000000000376000003960000090
:100040003B600000554700006D6400003B6000000D
:100050003B600000000000003B6000003B600000CF
:100060003B6000003D6700003B6000003B6000001B
:100070003B6000003B6000003B6000003B60000014
:100080003B600000D56800003B6000003B60000062
:100090003B6000003B6000003B6000003B600000F4
:1000A0003B6000003B60000000000000000000001A
:1000B0000000000000000000000000000000000040
:1000C00010B5064C2378002B07D1054B002B02D02E
:1000D000044800E000BF0123237010BD500200203F
:1000E0000000000098D00000044B10B5002B03D096
:1000F0000349044800E000BF10BDC04600000000F6
:100100005402002098D00000164B002B00D1144B55
:100110009D46402292029A1A924600218B460F4633
:100120001348144A121A0AF073F90F4B002B00D02F
:1001300098470E4B002B00D0984700200021040068
:100140000D000D48002802D00C4800E000BF0AF066
:100150001FF92000290006F0A7F90AF0F3F8C046BD
:100160000000080000400020000000000000000027
:1001700050020020A82F0020000000000000000016
:100180000123034010D104280CD90268120909D0B8
:10019000531E9B001A1DC1180979002902D0013392
:1001A0009342F8D1180070470023FBE70378002B37
:1001B00003D05AB2002A01DB013070473F2293433B
:1001C000C03B59424B41C01803789343802BF4D174
:1001D0000130F9E710B500240378002B01D120008D
:1001E00010BDFFF7E3FF0134F6E770B5002204000D
:1001F0000D00411C092002F00DFF002806D001234C
:100200006200134343600023A34200DB70BD9A00E9
:10021000A958821891600133F6E770B5012803DC14
:100220001C2000F093FE70BD01230D6811201D42BB
:10023000F7D04868184206D1042804D90F23026871
:100240001340042B01D00E20EBE702F04DFD6D10A2
:100250000400002D03DDFFF7BDFFA84206DA1220DF
:10026000DFE72000FFF7A2FF0400013D012DF8D1D8
:1002700020787F2809DDDF280BDCF8233F22DB0014
:10028000800118406378134018430123400018434D
:10029000C9E7EF280BDCFC22637812019B011340B5
:1002A0003F220007000C0343A0781040ECE7F7283A
:1002B00012DCFC22637892021B031340E0228004CC
:1002C000520310403F221843E3781340FC220343BB
:1002D000A07812018001E8E701204042D5E7F0B59F
:1002E000070085B00D001C20012F06DD4C6801239E
:1002F00022001A40019203D10D2000F027FE54E0A5
:10030000022F02D08A681A42F6D001232E681E42BC
:1003100000D07EE0042E00D87BE01C41002C00DCE5
:100320001C000F2332681340092B29D173685B101E
:100330000193022F05D0AB68019A5B109A4200DD51
:100340000193019B01221F1B0137FB43DB171F4059
:10035000791C092002F05EFE061E09D001237F00F1
:100360001F4303002A68083347600199A14202DA5B
:10037000300005B0F0BD0134A100515802C3F4E7CC
:10038000042B46D1300002F0AFFCFFF723FF0290B0
:10039000022F04D0AB685B10984200DD0293029BF1
:1003A0009C4204DD002002F0A1FE0600E0E73000E0
:1003B00002F09AFC0700019B9C4222DC300001976E
:1003C00002F092FC03903800FFF7F0FE029B01342C
:1003D0000700A342F7DA019BC71A380002F086FE35
:1003E000061EC5D002F080FC0400286802F07CFCE8
:1003F000039A019B991A41183A00200009F0ECFF7A
:10040000B6E73800FFF7D2FE019B070001330193E6
:10041000D1E7212071E7F8B54D680F00EB0706D44E
:10042000042D04D90F232E683340092B03D00B2051
:1004300000F08CFDF8BD6B6836095C10731EA3429A
:100440000FD80321200007F09FFE6421642803DCFD
:100450000100032800DA03212800891902F00AFEAE
:1004600005002B6800201B09013B9C42E2D23A6840
:10047000A31C9B005A510123013464001C436C608F
:10048000D8E7F0B585B0012803DC1C2000F05EFD44
:1004900029E001254F682A00022806D08B682B42EC
:1004A00003D05D10002D00DC15000124274200D090
:1004B00074E0042F00D871E00F223B680E681340EF
:1004C000042B25D1264205D1042E03D933681340CD
:1004D000042B01D00E20D9E73800FFF751FEA842C7
:1004E00003DA0120404205B0F0BD380002F0FCFB09
:1004F0000700300002F0F8FB013D010078190AF016
:1005000026FB0028EDD0C01B013040002043EAE765
:10051000092B43D17B685B1000939D42E1DC3000E6
:1005200020402ED1042E2BD90F22336820001340F7
:10053000042B26D1300002F0D7FB0F2325000290B8
:100540000393631C01939B00F858864202D1640018
:100550002800DBE728420ED104280CD90368039A4F
:100560001340042B07D102F0BFFB010002980AF0F0
:10057000C1FA0028EBD0019C009B9C42E1DDB0E772
:100580002000431C9A00BA58B24202D14000012414
:10059000BCE71800009B9842F3DDA2E7212075E735
:1005A00010B502F085FB43000120184310BD000088
:1005B00010B57F2902DC0170013010BD1A4B994241
:1005C0000CDC40238A115B42134303703F230B4032
:1005D00080214942194341700230EEE7134B9942A2
:1005E00010DC20230A135B4213433F248022037054
:1005F0008B1152422340214013430A4343708270BF
:100600000330DAE70A4B9942D7DCF0230370603BF2
:100610004370113B8A11FF3B1A4382703F22114005
:100620001943C1700430C8E7FF070000FFFF000056
:10063000FF0F0100F0B50D0085B0002803DC1C2081
:1006400000F084FC0DE009680122080010400AD087
:1006500002AC11412000FFF7ABFF011B200002F0AC
:1006600051FD04001AE004293FD90F230C682340F0
:10067000092B3AD14B685B10019303239C46019BE5
:100680009A420EDD02F032FD041E07D02E680125CD
:1006900002F02AFB2F00019B9D421DDD200005B0CA
:1006A000F0BD01329300CC580123234001D10D202D
:1006B000C6E764107F2C0DDD0D4E0223B44209DD28
:1006C0000C4E6346B44205DD00270B4EE30FA642F5
:1006D0007B419B00C018D2E70135AB00F15839428D
:1006E000E5D04910FFF764FFD5E72120A8E7C04611
:1006F000FF070000FFFF0000FF0F010010B504001E
:100700000120084010D104290DD90F230A68134095
:10071000042B08D1080002F0E7FA010020000AF0DB
:10072000E9F94342584110BD0020FCE7F7B50F003E
:10073000012803DC1C2000F009FCFEBD01264D68E9
:100740002E4006D1042D04D90F222B681A40092A05
:1007500001D00B20EFE76A681B095410A34200D8B0
:100760005C1E39681E48FFF7C9FF0123019000286D
:1007700013D139681B48FFF7C1FF002811D0002CA6
:100780000DD00123621C013C9C4092005351234335
:100790006B6004E00136B200AB50B442FADA0020DC
:1007A000CBE73B680D20DA07C5D55B10002B11DDC8
:1007B0009C420FDB9B00A200291DEB188918043313
:1007C000994209D10123013C9C40AA181C43536063
:1007D0006C60E4E71220AEE758681860EFE7C046A7
:1007E0006BBA00006FBA0000002310B50C000B704C
:1007F000C30705D50D49421020000AF04DF908E065
:100800000B49002802D0042804D10A4920000AF02C
:1008100063F910BD0428FCD90F2302681340042B90
:10082000F7D102F061FA04490200E5E7C8C200000E
:1008300074BA00007ABA00007FBA0000F0B593B035
:100840000390030002911C20012B1DDD029B01255A
:100850001B681C002C4000D0A8E0042B00D8A5E0A9
:100860001A680F231A40092A48D10194019A029963
:1008700092008A5816002E4005D1042A03D9106828
:100880001840092804D0222000F060FB07002CE06B
:1008900052685210A418019A013201920199039AE8
:1008A0008A42E3D1611C012202F0B4FB071E01D190
:1008B00000271AE064002543456005000835029AC8
:1008C000B300D1584B680A685B1012099A4200D8ED
:1008D000531E002293420BDCDA43D21713409B00D5
:1008E000ED18019B01369E42E9DB380013B0F0BDE4
:1008F00090000C18A46801322C50EBE7042A55D163
:100900002F0026001D00029AB300D058384237D17C
:10091000042835D903682B40042BB4D1FFF730FCF1
:10092000039B01362418B342EDD1200002F0DEFB18
:10093000071EBDD0039B029D9B00EB18041D029374
:1009400001232E681E4222D1042E20D90F223368A3
:100950001340042B0DD13000FFF712FC0190300042
:1009600002F0C2F9019A0100200009F035FD019B57
:10097000E418029B0435AB42E2D100232370B4E7B4
:1009800005A9FFF731FF05A80AF0C6F8C8E705A9D1
:100990003000FFF729FF05A80AF0BEF806000200A4
:1009A00005A9200009F018FDA419E2E7212000F0B4
:1009B000CDFA7DE7F0B50D0095B0002806DC1C20CF
:1009C00000F0C4FA0400200015B0F0BD0C6801214D
:1009D00023000B40009306D1042C04D922680F3366
:1009E0001A40092A01D00B20EAE7626852100392EC
:1009F000002A03DC009802F079FBE3E73F4A01920A
:100A000001280BD06868084208D1042806D902687A
:100A10001340042B02D102F067F9019001980AF00B
:100A20007BF806000F27039B0834013B04935E43C9
:100A3000039B02909B001B19059301232068184219
:100A400051D104284FD903683B40042B52D1FFF702
:100A500097FB059B04343618A342EED1300002F018
:100A600045FB041EAFD02B680593029B002B03D0DF
:100A7000686802F039F90190200002F035F90500AC
:100A8000009B059A9B00D3189F68380002F02CF950
:100A9000012306001F4201D1042F04D807A9380002
:100AA000FFF7A2FE07AE30000AF036F8070002009A
:100AB0003100280009F090FC029BED19002B0AD0B0
:100AC000049B009A934206DD2800029A019909F0DE
:100AD00083FC029BED18009B01330093009A039B5B
:100AE0009342CDD16FE707A9FFF77EFE07A80AF072
:100AF00013F8AEE702F0F8F8F9E7C046CFBD000002
:100B000010B50024A04207DD0B6801341C4003D05F
:100B10005C10E343DB171C40611C0122092002F03A
:100B200079FA002803D0012364001C43446010BDFF
:100B30000B6870B518000125284032D1042B30D93C
:100B40000F241A6849681440092C16D15C681209F0
:100B50002C41A24200D8541E844205DC02200132FE
:100B6000904206DB00200FE085005D19A96001308E
:100B7000F2E7840019510130F2E7032C11D1294228
:100B800003D1132000F0E2F970BD4910FF29F8D815
:100B90001209043392009A189A42E3D9197001336A
:100BA000FAE70B2000F0D2F9DCE700000123F7B5EB
:100BB00000264D680F002B400093B3420DD11E005C
:100BC000042D0AD90F222B681A40092A0FD16A680E
:100BD0001B095610B34200D85E1E3968CB0713D5E7
:100BE0004C10002C01DDA64219DA12202EE0042A56
:100BF00004D12800FFF7C4FA0600EEE7009E032A9E
:100C0000EBD11E09B600E8E72E48FFF777FD002874
:100C100014D009F0DDFE310007F09CFB4C1C009B5A
:100C2000002B4CD1042D4AD92A680F331340092BCD
:100C300010D10134A40064592000FEBD3968224857
:100C4000FFF75CFD34000028E9D1113000F07EF997
:100C50000400F1E7042B2AD1280002F045F8060031
:100C6000FFF7B8FAA042C0DB012C1ADC280002F022
:100C70003BF800903000FFF799FA851B280002F03E
:100C800035FA041ED8D002F02FF80190786802F0EF
:100C90002BF8009B2A00F11A4118019809F09CFBDF
:100CA000CAE73000FFF782FA013C0600DCE7032BBD
:100CB00005D12C19E478023B64001C43BCE70B20EF
:100CC000C4E7C04664BA00006FBA0000F7B54C68CC
:100CD0000F000120210001402AD1042C28D90F2225
:100CE0002368BE681A40092A13D162681B0955108F
:100CF0000191AB4200D85D1E39682848FFF7FEFC21
:100D0000002829D00F2322681340092B19D1012371
:100D100013E0032A0CD1064203D1132000F016F988
:100D2000FEBD72100192FF2AF7D81D09AD00E3E75E
:100D30000B20F3E701339A00A6509D42FADA002017
:100D4000EEE7032BFBD1230001331A1BAA42F6DC8A
:100D50006A461279DA70F7E73968CB0706D5491089
:100D6000002901DD8D4209DA1220D7E70C48FFF790
:100D7000C5FC2900002801D11130CFE70F232268DC
:100D80001340092B03D1013189000E51D7E7032B02
:100D9000D5D16B461B796418E370D0E76BBA0000BD
:100DA0006FBA000010B501240868204216D104284B
:100DB00014D90F2203681A40092A01D1406810BDD6
:100DC000032A03D11809C0002043F8E7042A05D1FB
:100DD00001F08AFFFFF7FEF94000F5E70B2000F075
:100DE000B5F8ECE710B5034A0A21034803F0AAFD61
:100DF00010BDC04614BA00000CBA00000200012069
:100E0000104001D0501070470D22014B1A70FAE7C4
:100E100090020020F0B585B00393019002912C4E12
:100E20002C4B002A02D002223270013A00251A60AF
:100E30001B68F554019B9D4201DB05B0F0BD029A91
:100E4000AB00D058234B1C68C8239B0037191C1BD0
:100E50000123184206D0204A43102100380009F02F
:100E6000E9FD09E01D4A002802D004281BD11C4AD4
:100E70002100380009F0DEFD300009F04DFE154A72
:100E8000039B1060002B0CD0019B013BAB4208DDA3
:100E9000144B984205D8431C136020223254002280
:100EA000F2540135C6E704280FD90F230268134016
:100EB000042B04D101F018FF0B4A0300CDE7092BE6
:100EC00004D14368094A5B10C7E70123084AC4E715
:100ED00091020020B4050020C8C2000074BA0000CE
:100EE0007ABA00001F030000BFC80000E4BC000085
:100EF000F3BC00000123020010B51A4015D10428EC
:100F000001D9026812090B4011D1042901D90B68DB
:100F10001B090024934206D104309B000431C318FE
:100F2000984206D30124200010BD0022EBE70023E5
:100F3000EFE704780A78002C01D1002AF2D00130C2
:100F400001319442ECD00024EDE70000014B187011
:100F5000002070479002002070B501F0D5FC094CCC
:100F60000100251D1F22280009F0DDFD280009F0E1
:100F7000D3FD0423043080080001184320602000C2
:100F800070BDC0466C020020C368F0B59D00836848
:100F900089B05D190300183306930369069A9F0010
:100FA000069B0290DF19436901939B00D3180393BA
:100FB000CD4B1B78002B26D17F222B68CB491C12EE
:100FC00013409B005B58043501929F46029B587862
:100FD00004F094F80023029A137027E0C24B1B78A8
:100FE000002B10D12B68019A1C121340BF4A9B00A2
:100FF0009B580435E9E7069B3A1DD11ABA4BD8290C
:1010000028DD1A221A70029BB74C9B682178019345
:10101000EA1A029B92109B7812021A43029B58789C
:1010200004F074F80023029A23701370029B069A4E
:101030009B680193ED1A029BAD10DD60069BFE1AC2
:10104000029BB6101E61039B9B1A029A9B10536170
:1010500009B0F0BD1B783C60002B01D01700D2E72F
:101060002B6801991C120B40A0499B005B5817008C
:101070000435AAE7069B3A1DD11A9B4BD82902DDFD
:101080001A221A70BFE728681B78291D3860002BC8
:1010900002D017000D00B6E76B6801991C120B40D7
:1010A00092499B005B58170008358EE7069B3A1D56
:1010B000D11A8D4BD82902DD1A221A70A3E7A40099
:1010C0001B782C193C60002B01D017009BE72B6884
:1010D00001991C120B4085499B005B581700043591
:1010E00073E7069B3A1DD11A7F4BD82902DD1A22DD
:1010F0001A7088E77E49A40061581B783960002B7C
:1011000001D017007FE72B6801991C120B4077492B
:101110009B005B581700043557E7043F744B3A684F
:10112000A400E250704B1B78002B00D06BE72B68BB
:10113000019A1C1213406D4A9B009B58043544E7EA
:101140006B4BA400E058FFF759FE043F06003868D7
:10115000FFF754FE36180120654B76000643E65033
:10116000614B1B78002B00D04DE72B68019A1C12B5
:1011700013405E4A9B009B58043526E7069B3A1DA8
:10118000D11A594BD82902DD1A221A703BE706986A
:10119000039C0121A04202D221000C3909681B786E
:1011A0003960002B01D017002DE72B6801991C1224
:1011B0000B404E499B005B581700043505E7069B22
:1011C0003A1DD11A484BD82902DD1A221A701AE7A3
:1011D0000699039881420FD203000C3B1B684549D6
:1011E0005B106418E41AA40023583B603E4B1B7844
:1011F000002B05D0170006E7182119700023F4E72B
:101200002B6801991C120B4038499B005B58170052
:101210000435DAE6069B039A934219D213000C3B7D
:101220001B68344A043FA4185B10E31A039A396818
:101230009B0099502C4B1B78002B00D0E3E62B68C9
:10124000019A1C121340294A9B009B580435BCE6A6
:101250001822254B1A70EDE7069B039A93422DD274
:10126000244B3E1FE31814000C3C04932368049A9B
:101270005B10D31A039A9B009858FFF7BFFD0790A5
:101280003068FFF7BBFD2468049B64101C1B079BA0
:10129000A4001F1801207F00039B0743E75037007D
:1012A000114B1B78002B00D0ADE62B68019A1C1265
:1012B00013400E4A9B009B58043586E618220A4BC1
:1012C0001A70EDE7069B3A1DD11A074BD82902DDAB
:1012D0001A221A7097E60399A40061581B783960A6
:1012E000002B09D017008EE690020020E4BA00001F
:1012F000502D0020FDFFFF3F2B6801991C120B4071
:10130000D7499B005B58170004355EE6043F039BFA
:101310003A68A400E250D34B1B78002B00D072E651
:101320002B68019A1C121340CD4A9B009B58043530
:101330004BE6039BA4001C192368043F38685E1029
:10134000FFF75CFD36180120C64B76001B7806437C
:101350002660002B00D056E62B68019A1C12134021
:10136000BF4A9B009B5804352FE6069BA4003F1BF9
:10137000BC4CBB420CD82378002B00D043E62B6832
:10138000019A1C121340B64A9B009B5804351CE678
:10139000B54801F099FC2378002B00D033E62B6888
:1013A000019A1C121340AE4A9B009B5804350CE670
:1013B000A300ED18002C00DA38E6AA4B1B78002BAE
:1013C00000D020E62B68019A1C121340A44A9B000F
:1013D0009B580435F9E5043F3B68042B04D1A30076
:1013E000ED18002C00DA21E69E4B1B78002B00D074
:1013F00009E62B68019A1C121340994A9B009B58DE
:101400000435E2E5043F3B68042B06D0A200AD188A
:10141000002C02DA002B00D108E6924B1B78002B3F
:1014200000D0F0E52B68019A1C1213408C4A9B00F7
:101430009B580435C9E53A1F13685B10013B002B2C
:1014400006DD01215B00A4000B432D191360EDE5BF
:10145000844B17001B78002B00D0D4E52B68019A31
:101460001C1213407E4A9B009B580435ADE53A00A0
:10147000069B0C32D31AD82B03DD1A22794B1A7033
:10148000C1E5FF2361005B001940FE3BFF3B1943B0
:101490003960029906988968241204916D1A02999C
:1014A000AD1089782D020D4303999D40091A8910CA
:1014B00099401D430B43BB60029B7D609C70E4B26E
:1014C0006A4BE4000392E358029A9360654A1278EB
:1014D000002A03D008331D00039F94E51D00019AE4
:1014E0009B680C351C1213405D4A9B009B58039F60
:1014F0006BE53B1F1C68039A069B93422DD10A2083
:10150000E3070CD4042C13D90F2322681340042BB7
:1015100011D1200001F0E8FB09F0FEFA063064303A
:1015200003F0A0FA00280FD1043D069B03937DE54C
:101530000720042CF3D02000431E9841FA23404298
:10154000FF3318400730EAE7029B2100587803F088
:10155000EFFD0023029A1370E7E7039B039A0C3B0D
:101560001B6802995B109B00D31A0C3B1C601F1D6B
:101570001300083B1B685A108A70D2B23B49D20054
:101580005B0055589B0A029A9B009560ED18039BDF
:10159000069A043B1B685B109B00D3180393314BE6
:1015A0001B78002B00D02EE52B68019A1C121340EB
:1015B0002B4A9B009B58043507E53B1F1868FFF733
:1015C0001DFCA40006003F1B1E2827DC00280DDCA4
:1015D000244B1B78002B00D015E52B68019A1C12B8
:1015E00013401F4A9B009B580435EEE401F07AF942
:1015F000033E361801F076F91D4B801B9842F9D84E
:10160000184B1B78002B00D0FDE42B68019A1C12AC
:101610001340134A9B009B580435D6E40123029AD9
:10162000137001F05FF9029B0A3886195E60FDE4D1
:101630003B1F1868FFF7E2FBA40006003F1B0028D1
:1016400018DC084B1B78002B00D0DCE42B68019AD7
:101650001C121340024A9B009B580435B5E4C04657
:10166000E4BA00009002002005BD000058250020CB
:101670009F860100CA4B984203DD1D22C94B1A7098
:10168000C1E40123029A137001F02CF9FA239B00A4
:101690005E43029B0A3E30185860C7E4A300FF1A5D
:1016A000002320001A003900FFF7B4FBBE4EBF4CE8
:1016B0003168200001F026FDBD4B31681860200024
:1016C00003F0EAFB3168200003F039FD31682000A7
:1016D00001F0B4FDB34B1B78002B00D093E42B68D2
:1016E000019A1C121340B34A9B009B5804356CE4CA
:1016F000AC4BA4001B783F1B002B00D083E42B686D
:10170000019A1C121340AB4A9B009B5804355CE4C1
:10171000029803F00BFAA34B1B78002B00D072E465
:101720002B68019A1C121340A24A9B009B58043557
:101730004BE43B1F1B68002B3ED13B000C3B1B685E
:10174000DA072CD5390001225B1058000839024312
:101750000A60002B44DD012259001143381F01604B
:101760003900083909681141CB1A39000C39096868
:10177000114224D09B189340A4001343039AA35012
:10178000884B1B78002B00D03DE42B68019A1C127B
:101790001340884A9B009B580435FFF716FC042B26
:1017A00006D90F2219680A40092A01D15B68C9E7E6
:1017B00019227C4B1A7026E45B10013BC9E704290F
:1017C00009D90F2208680240092A04D102339B007C
:1017D0005B58A400D2E71922724B1A70FFF713FC72
:1017E0000435CDE7A300069AFB189B1AD82B13DC0F
:1017F0000122631E002C14DC6A4B1B78002B01D0E5
:10180000FFF701FC2B68019A1C121340694A9B00E8
:101810009B580435FFF7D9FB1A22624B1A70FFF769
:10182000F2FB3A601C000437E3E7069A3B1D9B1A63
:101830005C4ED82B03DD1A233370FFF7E4FB069BC5
:10184000039AA40093422AD23B1F1868FFF7D6FAE6
:10185000011E21DD039B0C3B1A68521082421BDBE8
:101860009007801A544B4018C018039B8000C25840
:101870003B1B1A604B4B3F1B1B780437002B01D0DE
:10188000FFF7C1FB2B68019A1C121340494A9B00C9
:101890009B580435FFF799FB20233370EAE71823A0
:1018A000FBE7434BA4001A683B1B1F001A603D4B2B
:1018B00004371B78002B01D0FFF7A5FB2B68019A9A
:1018C0001C1213403B4A9B009B580435FFF77DFBDD
:1018D000A3009C46FE1A002C17DC1C22314B1A7008
:1018E000002333606346FF1A2E4B04371B78002B0E
:1018F00001D0FFF788FB2B68019A1C1213402D4A78
:101900009B009B580435FFF760FB002033685A109A
:101910008300F15801230B4003D10D21214A11709E
:10192000DFE749108A4200DD0A0001308442EFDC23
:10193000012352001343D4E7A3009C46FE1A002C57
:1019400017DC1C22174B1A70002333606346FF1A02
:10195000144B04371B78002B01D0FFF754FB2B6886
:10196000019A1C121340134A9B009B580435FFF741
:101970002CFB002033685A108300F15801230B40E0
:1019800003D10D21074A1170DFE749108A4200DABE
:101990000A0001308442EFDC012352001343D4E7F4
:1019A00080EE360090020020B40500209102002055
:1019B00008000020E4BA0000FCFFFF3F3B00083BAA
:1019C0001868FFF71BFA3B1F06001868FFF716FAA6
:1019D0000023864200DA0433A4003A1B1700136088
:1019E000E34B04371B78002B01D0FFF70CFB2B686F
:1019F000019A1C121340DF4A9B009B580435FFF7E5
:101A0000E4FA3B00083B1868FFF7F8F93B1F0600B3
:101A10001868FFF7F3F9F30FC217B0425341A4005F
:101A20003A1B17009B001360D14B04371B78002B27
:101A300001D0FFF7E8FA2B68019A1C121340CD4A37
:101A40009B009B580435FFF7C0FA3B00083B186821
:101A50003B1F1968A600BE1B0423814202D0042844
:101A600002D80023336016E001231842F9D10F2376
:101A700002681A40042AF4D1033A1142F1D1042930
:101A8000EFD90A681340042BEBD1FFF733FA431E5A
:101A9000984180003060B64BA4001B783F1B043790
:101AA000002B01D0FFF7AFFA2B68019A1C121340EC
:101AB000B04A9B009B580435FFF787FA3B00083B70
:101AC00018683B1F1968A600BE1B0023814202D084
:101AD000042802D80423336016E001231842F9D108
:101AE0000F2302681A40042AF4D1033A1142F1D1BB
:101AF0000429EFD90A681340042BEBD1FFF7FAF958
:101B00004342584180003060994BA4001B783F1B32
:101B10000437002B01D0FFF776FA2B68019A1C12CC
:101B20001340944A9B009B580435FFF74EFA3B0044
:101B3000083B1868FFF762F93B1F06001868FFF7BB
:101B40005DF9F317C20F86425341A4003A1B1700F8
:101B50009B001360864B04371B78002B01D0FFF7E6
:101B600052FA2B68019A1C121340824A9B009B5820
:101B70000435FFF72AFA3B00083B1868FFF73EF9E7
:101B80003B1F06001868FFF739F90023864200DD85
:101B90000433A4003A1B17001360754B04371B78FD
:101BA000002B01D0FFF72FFA2B68019A1C1213406B
:101BB000704A9B009B580435FFF707FA3B1F1B68D0
:101BC000A400043B5A1E93413A1B17009B0013606C
:101BD000674B04371B78002B01D0FFF714FA2B68F2
:101BE000019A1C121340634A9B009B580435FFF76F
:101BF000ECF93B00083B1868FFF700F93B1F0600B3
:101C00001868FFF7FBF832180120A4003B1B1F00E7
:101C1000520002431A60564B04371B78002B01D048
:101C2000FFF7F1F92B68019A1C121340514A9B00EF
:101C30009B580435FFF7C9F93B00083B1868FFF7CC
:101C4000DDF83B1F06001868FFF7D8F8321A0120AC
:101C5000A4003B1B1F00520002431A60444B043790
:101C60001B78002B01D0FFF7CEF92B68019A1C12CC
:101C70001340404A9B009B580435FFF7A6F93B00F0
:101C8000083B1868FFF7BAF83B1F06001868FFF713
:101C9000B5F802000120A4003B1B1F007243520054
:101CA00002431A60324B04371B78002B01D0FFF738
:101CB000AAF92B68019A1C1213402E4A9B009B58CC
:101CC0000435FFF782F93B1F1868FFF797F8061EE7
:101CD00017D11F22264B1A70A4003B1B1F001E6049
:101CE000234B04371B78002B01D0FFF78CF92B68AE
:101CF000019A1C1213401F4A9B009B580435FFF7A2
:101D000064F93B00083B1868FFF778F8310006F0EB
:101D10003BFA012640000643DEE73B1F1868FFF749
:101D20006DF8061E17D11F22114B1A70A4003B1B21
:101D30001F001E600E4B04371B78002B01D0FFF7ED
:101D400062F92B68019A1C1213400A4A9B009B58A7
:101D50000435FFF73AF93B00083B1868FFF74EF8E7
:101D6000310006F0F7FA012649000E43DEE7C046CF
:101D700090020020E4BA00003B1F1868FFF73EF80D
:101D8000C217801850400122A4003B1B1F004000D6
:101D900010431860F64B04371B78002B01D0FFF777
:101DA00032F92B68019A1C121340F24A9B009B588F
:101DB0000435FFF70AF9A300FE1A3068012C24D17C
:101DC000FFF71CF80494079008F002FE0799002919
:101DD00000DC012106F0BEFA049BA400C91801230F
:101DE00049001943E24B3F1B1B7831600437002B3D
:101DF00001D0FFF708F92B68019A1C121340DD4A45
:101E00009B009B580435FFF7E0F8FEF7F7FF0490BE
:101E10007068FEF7F3FF049B0130C31A0793D3E702
:101E2000A300FE1A31002000049301F0A7F9049BDF
:101E30003060FF1ACE4B04371B78002B01D0FFF720
:101E4000E2F82B68019A1C121340CA4A9B009B5867
:101E50000435FFF7BAF83B00083B1868FEF7CEFFE1
:101E60003B1F06001868FEF7C9FF02000120A4000E
:101E70003B1B1F003240520002431A60BC4B043728
:101E80001B78002B01D0FFF7BEF82B68019A1C12BB
:101E90001340B84A9B009B580435FFF796F83B0067
:101EA000083B1868FEF7AAFF06003B1F1868FEF7FC
:101EB000A5FF320002430120A4003B1B1F0052007B
:101EC00002431A60AA4B04371B78002B01D0FFF79E
:101ED0009AF82B68019A1C121340A64A9B009B5843
:101EE0000435FFF772F83B00083B1868FEF786FFE1
:101EF00006003B1F1868FEF781FF320042400120B8
:101F0000A4003B1B1F00520002431A60984B043789
:101F10001B78002B01D0FFF776F82B68019A1C1272
:101F20001340944A9B009B580435FFF74EF83B1F23
:101F30001868FEF763FFC0430122A4003B1B1F008B
:101F40004000104318608A4B04371B78002B01D0E7
:101F5000FFF759F82B68019A1C121340854A9B0021
:101F60009B580435FFF731F83B00083B1868FEF733
:101F700045FF06003B1F1868FEF740FF3200824015
:101F800051000122A4003B1B1F000A431A60784B3A
:101F900004371B78002B01D0FFF735F82B68019A26
:101FA0001C121340734A9B009B580435FFF70DF831
:101FB0003B00083B1868FEF721FF06003B1F18682E
:101FC000FEF71CFF3200024151000122A4003B1B1E
:101FD0001F000A431A60664B04371B78002B01D0A0
:101FE000FFF711F82B68019A1C121340614A9B00FD
:101FF0009B580435FEF7E9FF3B000C3B1868FEF7E1
:10200000FDFE3B00083B06001868FEF7F7FEF117DF
:102010000200C317300006F0EFF93B1F0490059152
:102020001868FEF7EBFE02000498059906F098F98F
:1020300043000120A4003E1B370018434C4B306086
:102040001B780437002B01D0FEF7DDFF2B68019AC7
:102050001C121340474A9B009B580435FEF7B5FFFE
:10206000A300FE1A310020000493FEF749FD049BF3
:102070003060FF1A3E4B04371B78002B01D0FEF76F
:10208000C2FF2B68019A1C1213403A4A9B009B58CE
:102090000435FEF79AFFA300FF1A39002000FEF76F
:1020A00047FD334B1B78002B01D0FEF7ACFF2B68AC
:1020B000019A1C1213402F4A9B009B580435FEF7CF
:1020C00084FFA300FE1A310020000493FEF76EFD8A
:1020D000049B3060FF1A264B04371B78002B01D07D
:1020E000FEF791FF2B68019A1C121340214A9B00B6
:1020F0009B580435FEF769FFA300FF1A3900200042
:10210000FEF7E4FD1A4B1B78002B01D0FEF77BFF96
:102110002B68019A1C121340164A9B009B580435E9
:10212000FEF753FFA300FE1A310020000493FEF7D0
:1021300039FE049B3060FF1A0D4B04371B78002BCF
:1021400001D0FEF760FF2B68019A1C121340094A68
:102150009B009B580435FEF738FF069B3E1DF31A83
:10216000034CD82B08DD1A232370FEF74CFFC04622
:1021700090020020E4BA000000F0BEFB4300012002
:10218000184323783860002B02D03700FEF73BFF5E
:102190002B68019A1C121340F44A9B009B5837008D
:1021A0000435FEF712FF069B3E1DF31AF04CD82BA8
:1021B00003DD1A232370FEF726FF00F093FBED4B9F
:1021C000400018400123184323783860002B02D0C8
:1021D0003700FEF718FF2B68019A1C121340E34AE0
:1021E0009B009B5837000435FEF7EFFE0123A60045
:1021F000BE1B20001A003100FEF70CFEDE4C2068EA
:10220000643002F02FFC002802D1043DFEF70EFFDF
:10221000029B21685A78D94802F09FFF0123029A55
:102220003700137000F05EFBD54B22681B68063246
:1022300053431818029B5860FEF7F8FEA600BE1B19
:102240002000012300223100FEF7E4FDCA4C206883
:10225000643002F007FC0028D7D0C84802F074FDB3
:10226000DCE7A4003E1BFEF777FE3700C04B306072
:102270001B780437002B01D0FEF7C5FE2B68019AAE
:102280001C121340B94A9B009B580435FEF79DFE73
:10229000A4003E1B300000F05EFB3700B44B306002
:1022A0001B780437002B01D0FEF7ADFE2B68019A96
:1022B0001C121340AD4A9B009B580435FEF785FE67
:1022C000A4003E1B300000F048FB3700A84B3060F4
:1022D0001B780437002B01D0FEF795FE2B68019A7E
:1022E0001C121340A14A9B009B580435FEF76DFE5B
:1022F000A300FE1A31002000049300F031FB049B80
:102300003060FF1A9A4B04371B78002B01D0FEF780
:102310007AFE2B68019A1C121340944A9B009B582A
:102320000435FEF752FEA4003F1B380000F04AFBC4
:102330008F4B1B78002B01D0FEF765FE2B68019AAE
:102340001C121340894A9B009B580435FEF73DFE42
:10235000A300FE1A31002000049300F05BFB049BF5
:102360003060FF1A824B04371B78002B01D0FEF738
:102370004AFE2B68019A1C1213407C4A9B009B5812
:102380000435FEF722FEA4003F1B380000F084FB5A
:10239000774B1B78002B01D0FEF735FE2B68019A96
:1023A0001C121340714A9B009B580435FEF70DFE2A
:1023B0000121200000F058FB6D4B1B78002B01D051
:1023C000FEF721FE2B68019A1C121340674A9B00FE
:1023D0009B580435FEF7F9FD0021200000F044FB76
:1023E000634B1B78002B01D0FEF70DFE2B68019A82
:1023F0001C1213405D4A9B009B580435FEF7E5FD17
:10240000A4003E1B300000F069FB3700584B3060E1
:102410001B780437002B01D0FEF7F5FD2B68019ADD
:102420001C121340514A9B009B580435FEF7CDFD0A
:10243000A4003E1B300000F065FB37004C4B3060C1
:102440001B780437002B01D0FEF7DDFD2B68019AC5
:102450001C121340454A9B009B580435FEF7B5FDFE
:10246000A4003F1B380000F027FB414B1B78002BDA
:1024700001D0FEF7C8FD2B68019A1C1213403B4A9D
:102480009B009B580435FEF7A0FDA4003F1B3800BD
:1024900003F04AF9364B1B78002B01D0FEF7B3FD51
:1024A0002B68019A1C121340304A9B009B5804353C
:1024B000FEF78BFDA4003E1B300003F0C7F9370088
:1024C0002B4B30601B780437002B01D0FEF79BFDAF
:1024D0002B68019A1C121340244A9B009B58043518
:1024E000FEF773FDA4003F1B380003F0CDF8204B2E
:1024F0001B78002B01D0FEF786FD2B68019A1C1279
:1025000013401A4A9B009B580435FEF75EFDA40059
:102510003E1B300003F0CEF83700154B30601B78BF
:102520000437002B01D0FEF76EFD2B68019A1C12B8
:1025300013400E4A9B009B580435FEF746FDA3004E
:10254000FF1A3900200001F01BF9094B1B78002B02
:1025500001D0FEF758FD2B68019A1C121340034A64
:102560009B009B580435FEF730FDC046E4BA0000DE
:1025700090020020FEFFFF7FB405002091020020A2
:1025800004000020A300FF1A3900200000F080FFA3
:102590009F4B1B78002B01D0FEF735FD2B68019A6D
:1025A0001C1213409B4A9B009B580435FEF70DFDFF
:1025B000A300FF1A3900200000F07AFF944B1B782B
:1025C000002B01D0FEF71FFD2B68019A1C1213404F
:1025D000904A9B009B580435FEF7F7FCA300FF1AB6
:1025E0003900200000F08CFF894B1B78002B01D0B4
:1025F000FEF709FD2B68019A1C121340854A9B00C7
:102600009B580435FEF7E1FCA300FE1A31002000C0
:10261000049303F0C0F9049B3060FF1A7C4B04372D
:102620001B78002B01D0FEF7EEFC2B68019A1C12E0
:102630001340784A9B009B580435FEF7C6FCA30064
:10264000FE1A31002000049303F0ADF9049B3060C2
:10265000FF1A6F4B04371B78002B01D0FEF7D3FC19
:102660002B68019A1C1213406A4A9B009B58043540
:10267000FEF7ABFCA300FE1A31002000049303F028
:102680009AF9049B3060FF1A614B04371B78002BCA
:1026900001D0FEF7B8FC2B68019A1C1213405D4A6A
:1026A0009B009B580435FEF790FCA300FE1A3100F6
:1026B0002000049302F0A0FF049B3060FF1A544BEB
:1026C00004371B78002B01D0FEF79DFC2B68019A84
:1026D0001C1213404F4A9B009B580435FEF775FCB3
:1026E000A300FF1A3900200000F0D2FF484B1B78EE
:1026F000002B01D0FEF787FC2B68019A1C121340B7
:10270000444A9B009B580435FEF75FFCA300FF1A68
:102710003900200000F01CFF3D4B1B78002B01D03E
:10272000FEF771FC2B68019A1C121340394A9B007A
:102730009B580435FEF749FCA300FE1A3100200027
:10274000049300F073FE049B3060FF1A304B043793
:102750001B78002B01D0FEF756FC2B68019A1C1247
:1027600013402C4A9B009B580435FEF72EFCA30017
:10277000FF1A3900200000F0E9FF254B1B78002BE1
:1027800001D0FEF740FC2B68019A1C121340214A2D
:102790009B009B580435FEF718FC069B029AFB1A17
:1027A0009B101361A300FF1A3900200002F0DEF82D
:1027B000174B1B78002B01D0FEF725FC2B68019AE4
:1027C0001C121340134A9B009B580435FEF7FDFB77
:1027D000069B029AFB1A9B101361A300FE1A31009C
:1027E0002000049302F0C2F8049B3060FF1A084BEB
:1027F00004371B78002B01D0FEF705FC2B68019AEB
:102800001C121340034A9B009B580435FEF7DDFB66
:1028100090020020E4BA00000023F7B55A1E01928E
:10282000002B07DA00F0C2FF02F094FB02F0ECFC90
:102830001923019300263000194B1968B14212DDAB
:10284000184B1A6801328A420FDAF0241A601D68A8
:10285000154F6C43E35D002B1FD0E419022B06D10A
:102860002000FEF791FB019BD8E70022EDE7012B4A
:102870000DD1002801D100F035F8F0226A43BB18D1
:102880005B680A49C31A8B4201D80223BB54F02368
:102890005D43054BEB5C022BE2D00136CCE7C04632
:1028A000B805002000000020F81B00209F860100D2
:1028B00000207047002070470020704700207047BC
:1028C00001220020054B06491A615850043103309B
:1028D00058500831801858501A60704700800040E6
:1028E000040500000122034B1A64A822D200985864
:1028F0007047C0460080004010B5FFF7F3FFFA2193
:10290000890005F0B7FB10BD0048704758BD0000B6
:102910001D20704770B5054E0400335C0D008B42DE
:1029200002D003F057FF355570BDC046BC050020EE
:1029300070B50024064D635D012B05D100212000F8
:1029400003F048FF0023635501341D2CF2D170BD04
:10295000BC05002070470D2070473B2070470000E9
:10296000F8B501240B6806000D00234204D10D20A8
:10297000FEF7ECFA2000F8BD5B102000052BFAD81A
:102980000E4A9B009C580E4F3B5D002B05D000214A
:10299000200003F01FFF00233B55012E06DD6B686E
:1029A000042B03D10221200003F014FF200003F0C8
:1029B000BFFD012440002043DDE7C04640BD0000CC
:1029C000BC050020F8B501260568354202D04468F0
:1029D000344203D10D20FEF7B9FAF8BD6D101C2D5D
:1029E000FBD80A4F7B5D012B04D03100280003F097
:1029F000F1FE7E55064964108C4202DCE143C917A2
:102A00002140280003F01AFEE7E7C046BC0500207D
:102A1000FF03000070B501240D68254204D10D208C
:102A2000FEF794FA200070BD6D101C2D17D80024FD
:102A3000012804DD4C68043C63425C416400094E9B
:102A4000735DA34204D02100280003F0C3FE745537
:102A5000280003F0F3FE03000420012BE3D0002044
:102A6000E1E7C046BC05002070B504000D001C283D
:102A70000ED8084E335C012B04D0012103F0AAFECE
:102A800001233355290020004D1EA94103F0C0FE4B
:102A900070BDC046BC050020036810B5DA0703D43A
:102AA0000D20FEF753FA10BD4168581004394A4210
:102AB0005141FFF7D9FFF6E737B569460A00064BE3
:102AC00030CB30C203680220042B02D100F0F0FCAE
:102AD00037BD00F015FDFBE718BD000010B5084C30
:102AE0006379002B05D00021052003F073FE00233D
:102AF0006371052003F0A2FE43425841800010BDDF
:102B0000BC05002010B5084CE37A002B05D000214D
:102B10000B2003F05FFE0023E3720B2003F08EFE18
:102B200043425841800010BDBC05002070477047EB
:102B300010B5034A0421034801F004FF10BDC0464C
:102B400020BD0000F8C30000E12170B5490214481F
:102B500003F0E6FAFFF7B4FE0A2003F0E3FC0023DB
:102B6000FF21104A995401331D2BFBD10122002073
:102B70000D4B01001A6004230C4A0D4D1468002C03
:102B8000FCD02C680002013B20431160002BF5D1E2
:102B90000122084B1A6003F07FFC00F053FF70BD68
:102BA000801B0020BC05002000D0004000D1004068
:102BB00008D5004004D00040F8B50B4E07003000A7
:102BC0000D0003F0F5FA0400A84200DD2C003D00E2
:102BD000EB1B9C4205DD300003F0F4FA2870013550
:102BE000F6E72000F8BDC046801B002010B50100AC
:102BF000014803F09DFA10BD801B002010B5054C64
:102C0000200003F0A3FAE1212000490203F088FA32
:102C100010BDC046801B0020C3070CD4064B1B68A8
:102C2000834208D8054B1B68984204D8031F1B68D1
:102C3000002B00D018007047E4050020E0050020BC
:102C40000023012210B50A48990001334250642B39
:102C5000FAD1084C084B00211A602000074A07F0FF
:102C6000D7FB074B074A6360074B1A6010BDC0468D
:102C7000502D0020E805002008000020D4090000A5
:102C800030270000EC050020DC05002010B5044BC7
:102C9000044A1A60044B054A1A60FFF7D1FF10BDC1
:102CA000E4050020E8050020E0050020BC0F00201E
:102CB000044B1B68186800090238C343DB1718402F
:102CC0007047C046DC05002000B59BB002000549F6
:102CD00001A807F0E1FE01A802F052F802F094FA10
:102CE000FCE7C046BFBD00000A4BC20704D404285D
:102CF00004D8094B00D0094B180070470F22036815
:102D00001A40031D042AF7D0054B092AF4D0054BBD
:102D1000F2E7C046A5BD00007ABA000074BA000010
:102D2000B8BD0000AFBD00000020064A0649131FD1
:102D3000186013681B0902339B00D2188A42F6D32D
:102D40007047C046EC050020BC0F0020F7B50F24EB
:102D50000126304B304A1968304B314D18681368E2
:102D60001F002740072F25D813681B0902339B003B
:102D7000D218AA42F3D300242A4EA500AD19286820
:102D8000FFF74AFF01342860642CF6D1264C2068F6
:102D9000FFF742FF2060254C2068002802D0FFF793
:102DA0003BFF20600025224B1B680093009B9D4247
:102DB00013DBF7BD1B099B00D3189A42D4D01F68C0
:102DC000374208D1B94206D2B84204D3043F3F6823
:102DD000002F00D01F60043BEFE7F0236B43154A40
:102DE0009B181A78002A01D10135DFE71F693C23BF
:102DF00000266B43DB199B0001930136BB1BF3D408
:102E0000019BB4001C1B0B4B1C19A069FFF704FFAE
:102E1000A061F2E7E4050020EC050020E0050020B9
:102E2000BC0F0020502D002008000020BC0F002007
:102E3000B8050020F81B0020F7B50124204244D13A
:102E4000224B1B689C4698423FD3214B1B68019341
:102E500098423AD8031F1B68002B36D10200036842
:102E600000941B09002B0FD10099131F1960904289
:102E70002BD015682B1F1B68990069180C68013B43
:102E800014600A602A00EDE79D0055192968009C2E
:102E9000214218D18C4516D8019C8C4213D30E1FA9
:102EA0003468002C0FD10F680F343C40072C07D931
:102EB0002F60151F2B600B680A601B090A00D1E701
:102EC00000993160CEE7013BCCE7F7BDE405002077
:102ED000E00500200D49F0B50B000F260C4D1868D9
:102EE0001C1F276802090232002F0BD000208B42E2
:102EF00000D0080020609000091892009B18AB4297
:102F0000EDD3F0BDB0431860F7E7C046EC050020F4
:102F1000BC0F0020F8B5114C26000F2233681F09A2
:102F200013420DD07D1CAD00A64204D02A00310012
:102F3000200007F05AFA00226319043564191A6058
:102F40000237BF00064BF6199E42E6D31B1B9B10AF
:102F5000013B1B012360034B1C60F8BDEC05002006
:102F6000BC0F0020DC050020F0B59BB0FFF7BAFCD9
:102F700000240700204AA300D0580134FFF75CFF6B
:102F8000642CF7D11D4B1868FFF756FF1C4B1868CF
:102F9000002801D0FFF750FF00261A4B1B689E4205
:102FA00016DBFFF797FFFFF7D1FEFFF7B3FFFFF741
:102FB00099FC154BC21B1B6814491B6801A81B090F
:102FC000023B07F069FD01A801F0DAFE1BB0F0BD7D
:102FD000F02575430E4BED182B78002B01D10136EF
:102FE000DBE72B695C1E002CF9DBA300EB1898696A
:102FF000FFF722FF013CF6E7502D002008000020DB
:10300000BC0F0020B8050020DC05002085BD0000B5
:10301000F81B0020F7B5164D4F1C2B6806001B68E7
:103020000C0001921B099F420ADBFFF79DFF2B68F2
:103030001B681B099F4203DB0A20FDF787FFFEBDCB
:103040002868A71CBA00DB1B81181B010B602960D4
:103050000021031F19600F231E4003002401264393
:1030600040C3083A9A189A42E9D9019902C3FAE78B
:10307000DC050020F7B503000122134004000D0019
:103080000193002B2AD1164B1B68834226D8154B7F
:103090001B68834222D90F23134F38600068184001
:1030A000FFF7B8FF019B3C68061E3B6016D0236803
:1030B00004301B099D4200DD1D00AA00211D251FB3
:1030C00007F08AF9FFF730FE2E60FFF73FFE00237E
:1030D0002B6022680F339A43226034002000FEBD2B
:1030E000E4050020E0050020BC0F0020032304308D
:1030F00010B5C11719400918891000220420FFF7E4
:1031000089FF10BD70B5050008000C00FFF7EEFF49
:103110000023002804D170BDE95CC218117101338D
:10312000A342F9DBE343DB171C400023041923719E
:10313000F1E7000010B501240B681C4016D05C10AC
:10314000200005F0B5FA0B4905F080F907F066F8A4
:1031500003F0B8FC0022084B06F01AFA03F05AFC00
:1031600006F0ECFF43000120184310BD0D20FDF7D1
:10317000EDFEE5E7D30237390000D040086870B5AE
:1031800001240500254006D1042804D90F23026834
:103190001340042B03D00E20FDF7D8FE70BDFFF7BF
:1031A000A3FD03782900233B5A4253411022C01843
:1031B00007F068FD80239B05C218044B9A4201D991
:1031C0001420E9E740002043E8E7C046FFFFFF3F47
:1031D00010B5034A0221034801F0B4FB10BDC046FC
:1031E000D8BD0000D0BD00000020704710B51E20E3
:1031F000FDF7ACFE10BD10B51E20FDF7A7FE10BDFB
:1032000010B51E20FDF7A2FE10BD10B51E20FDF763
:103210009DFE10BD10B51E20FDF798FE10BD10B527
:103220001E20FDF793FE10BD10B51E20FDF78EFE8B
:1032300010BD10B51E20FDF789FE10BD70470000BF
:1032400010B5034A0921034801F07CFB10BDC046BC
:10325000F8BD000040BE00000120034B1860034B86
:103260001B68834018437047E00F0020C00F002008
:10327000F0B5EFF310810123194083F31088134C4C
:10328000134AA4461268134E013A9340124F134A50
:10329000002B17D0146803420FD03D682C60C04645
:1032A000C046C046C046C046C046C046C0460C4C9C
:1032B0001568246825605B08EAE765462C60146899
:1032C0003460F8E781F31088F0BDC046080500506F
:1032D0000C0000200C050050CC0F0020D40F002063
:1032E000C80F002030B585B001AD0C22064928007A
:1032F00007F072F80024285D01210134FFF70AFB72
:103300000C2CF8D105B030BDCCBE0000F7B56A4634
:10331000394B01AD13801C239370384B2B800A234B
:10332000AB70FFF7DFFA364B364CC0182368984273
:1033300001D2002323602668002E3DD16B469F5D9D
:1033400001213800FFF7E6FA01360021380003F0CA
:103350005FFA032EF2D10026AF5D01213800FFF79E
:10336000D9FA01360121380003F052FA032EF3D1C5
:10337000C8200138C046C046C046C046C046C04608
:10338000C046C046C046C046C046C046F1D1002136
:103390002878FFF7BFFA68780021FFF7BBFAA87812
:1033A0000021FFF7B7FAFFF79DFAFA2300251B016A
:1033B000C01820602800FEBDFFF794FA236800259E
:1033C0009842F7D3032003F0B3F80600042003F07B
:1033D000AFF836180A2003F0ABF80B4B9B1B181AFA
:1033E0000A4BA84206DB18600023094A23601360D9
:1033F0000125DFE71D60F7E71A1B0000030400004A
:1034000010270000D80F0020E3030000C00F0020A9
:10341000E00F002010B50124044002D04410200029
:1034200010BD0D20FDF792FDF9E700000868F8B522
:10343000C3071AD5FFF7EEFF0300203B5E2B23D80E
:103440000520012258430023104E451DA84217D0E5
:1034500005211024375C3C4200D09B1801395200F2
:1034600064100029F7D10130F0E704280CD90F22AD
:1034700003681A40042A07D11B0905D00079DBE74D
:1034800001205B001843F8BD0120FCE7D8BE000016
:103490000022054B10B51A60044B1B68934201D003
:1034A00002F0EEFA002010BDDC0F0020A41A00206C
:1034B00070B508680D00FFF7ADFF04006868FFF7FE
:1034C000A9FF621E0100042A14D8451E042D11D83C
:1034D00005236B439B18012215009D402B000648D5
:1034E00005682B430360054B1B68002B02D02000AE
:1034F00002F0C7FA002070BDDC0F0020A41A0020E3
:1035000070B508680D00FFF785FF04006868FFF7D5
:1035100081FF621E0100042A13D8451E042D10D815
:1035200005236B439B1801229A4007480368934385
:103530000360064B1B68002B03D00022200002F022
:10354000A0FA002070BDC046DC0F0020A41A0020A5
:10355000F0B5050089B008680C00FFF75BFF069026
:10356000022D36DD6068FFF755FF0190A068FFF778
:1035700051FF04000127231D661E0793731C02934D
:10358000079B9E4235D0052373430593019B019D04
:1035900005330493049BAB421ED0042E16D86B1E39
:1035A000042B13D80122059B2349013B5B199A4048
:1035B0009446224A0B681068069A3A4003920DD04E
:1035C00062461A430A60012200280DD17F000135AE
:1035D000E0E701240194CDE7029ECFE762469343E2
:1035E0000B600028F2D0039A0299280002F049FAF1
:1035F000ECE7019B1E1D042E1AD8012C18D10025C2
:1036000005273B0021006B439B1999400B000A4A98
:10361000013511689943094B11601B68002B05D0D7
:10362000019B0022581D290002F02BFA052DE8D13C
:10363000002009B0F0BDC046DC0F0020A41A002015
:1036400010B5041E10DA00240A4BA400E25801232E
:103650009340094A09491360094A1160094A0A4915
:1036600011600A4A136010BDFFF752F9A042EADD6B
:10367000EAE7C04650CB0000D40F002008050050F8
:10368000CC0F0020C80F00200C050050180500507A
:103690002B4BF7B51B680C00002B03D101204042D7
:1036A000FFF7CEFF24680126250035401AD0FF22FF
:1036B0006310120260121040DAB21043FF221B02A4
:1036C0001204134018431F4B1B68202B06D1B44033
:1036D0001D4BA40EA400E35800021843FFF7C8FDD9
:1036E0000020FEBD042CFBD90F2322681340092BB8
:1036F000F6D1FF2763683F025B100193019B9D4257
:10370000EEDAAB00E3189B68334216D05A10581219
:10371000D1B238400843FF21120209040A40104385
:10372000084A1268202A06D15B009B0E06499B00BE
:10373000020258581043FFF79BFD0135DEE7C046F3
:10374000D40F00200C000020B4C000000200086864
:1037500010B5C3070FD540101823012A03DD4A68AE
:10376000042A00D10833054A1360FFF7F3F8FFF786
:1037700067FF002010BD01204042EDE70C00002053
:10378000086810B5C30703D5FFF744FE054B186062
:10379000054B1B68002B03D0024B186802F072F92E
:1037A000002010BDDC0F0020A41A00207FB5A04C23
:1037B0002368002B0AD19F4A1268002A06D19E4B2B
:1037C0001B68002B01D0FFF7A1FD7FBD9B4D2A6830
:1037D000002A26D1984A1268002A1BD0FFF796FDCE
:1037E0000028F2D0FFF77EFD924B24681A681C6017
:1037F000002A16D0002C14D101AD0C2290492800CB
:1038000006F0EAFD285D00210134FFF783F80C2C57
:10381000F8D1DAE7874A1268002AE5D1002BE3D015
:10382000E0E700211A2002F0F3FF00211B2002F044
:10383000EFFF00211C2002F0EBFF2E68012E5CD070
:10384000022E00D1A2E0002E50D101363100794C79
:1038500003202368994302F0DBFF04202168014024
:103860004B42594102F0D4FF102123680A2019402D
:103870004B42594102F0CCFF8021236809011940D5
:103880004B425941062002F0C3FF80212368090200
:1038900019404B425941072002F0BAFF80212368AA
:1038A000490219404B425941092002F0B1FF8021E1
:1038B0002368890219404B425941192002F0A8FFA0
:1038C00080212368C90219404B425941182002F057
:1038D0009FFF802321681B0319404B425941172049
:1038E00002F096FF31001A2002F092FF2B680321AC
:1038F000581C04F02FFD296067E702214D4C17206A
:10390000236819404B42594102F082FF0821236885
:10391000182019404B42594102F07AFF8021236858
:10392000C90019404B425941042002F071FF802127
:103930002368490119404B4259410A2002F068FFAF
:1039400080212368C90119404B425941032002F0EC
:103950005FFF80212368890319404B4259410920A8
:1039600002F056FF802321681B0419404B42594145
:10397000192002F04DFF3100062002F049FF31000E
:10398000072002F045FF31001B20ADE72021294C24
:103990001720236819404B42594102F039FF40215A
:1039A0002368182019404B42594102F031FF802111
:1039B0002368192019404B42594102F029FF802108
:1039C0002368490019404B425941092002F020FF69
:1039D00080212368890019404B425941072002F099
:1039E00017FF80212368890119404B425941062065
:1039F00002F00EFF80212368490319404B425941D0
:103A00000A2002F005FF80212368C90319404B42B8
:103A10005941032002F0FCFE802321685B04194019
:103A20004B425941042002F0F3FE01211C205BE7C8
:103A3000DC0F0020D00F0020E00F0020C40F00207A
:103A4000CCBE0000012010B54042FFF7F9FD10BDCB
:103A500010B5034A0921034800F074FF10BDC046A9
:103A6000B4C10000FCC1000030B502248025094B20
:103A7000094AED009C505C59002CFCD0A124E400C4
:103A8000884202D30021995030BD8025ED001851A5
:103A90004019F5E700E001400405000010B50028DA
:103AA00006D1C020B02140028902FFF7DDFF10BD22
:103AB000B02080218002C902F7E70000434258414C
:103AC000064B40421840B0239B02C01803680020F8
:103AD0001A0E532A01D11B02180A704700C0FEFFBC
:103AE00030B501248025054B054AED009C505C59FA
:103AF000002CFCD001600021995030BD00E0014055
:103B00000405000043425841074B40421840B0238F
:103B10009B02C018A62310B50902DB05090A194348
:103B2000FFF7DEFF10BDC04600C0FEFF70B50124E8
:103B300080250D4B0D4EED009C515C59002CFCD0A6
:103B4000002902DC00229A5170BD557814782D02AC
:103B500025439478013924042543D478043224067B
:103B60002C4310C0ECE7C04600E001400405000013
:103B700070B505004B680A009C1C2100A400FFF7EB
:103B8000D5FF281970BD0000134B1B68002B0CD00B
:103B90008022B023D2029B0200280BD11A1D5B6841
:103BA0001B0E522B00D110007047B022C02392028E
:103BB0005B02F1E782420DD903681B0E522B09D13B
:103BC000436802339B00C018824203D903681B0E6E
:103BD000522BE9D00020E7E7E410002070B5002068
:103BE000FFF7D2FFFF260500002801D1280070BD95
:103BF00003681C143440FFF7C7FFDA2CF4D105002A
:103C0000F2E700008022F0B55200A1B00021674821
:103C100006F0FEFB802200215200654806F0F8FB0A
:103C2000644BFF271B681A00049353425A4110004B
:103C30000592FFF733FF049C0020631E9C415E4BFE
:103C400064421C405D4BE418FFF7C8FF0600002EDD
:103C50002DD10498FFF732FF411C0598FFF752FF62
:103C6000059A574D534B2C601A60FEF7C7FF514B16
:103C700064201B68A0215A4253414F4A5B421340C3
:103C8000B0222C6892029B18E41A6043490204F0A7
:103C90007BFAA0225202030000924A49220007A8A0
:103CA00006F0FAFE07A801F06BF821B0F0BD32680B
:103CB000131412123A403B4003921A000A3A092A9E
:103CC00049D83A4B039A995C002931D110223E48D9
:103CD00006F09EFB35002B6803991A123A40914278
:103CE00009D11A143A400B2A27D0132A2DD00A2AB8
:103CF00001D1354B1D602800FFF746FF051EEAD1B4
:103D0000314B196800290FD02000FFF731FF040064
:103D10002D4B5B195968002903D02000FFF728FFBD
:103D2000040004350C2DF3D1204B0121039A995442
:103D30003000FFF729FF060089E73B40022BDADC61
:103D4000214A9B00D3185D60D5E7102200211E4850
:103D500006F05EFBCFE71A00153A082AE8D8144AA5
:103D60000399525C002AE3D13500152B00D01500D1
:103D7000300003681A143A40152A0FD01D2A00D1CA
:103D80000025FFF701FF0028F3D1002D04D020000B
:103D90002900FFF7EDFE0400054BC6E7039A1B124E
:103DA0003B409A42EDD10500EBE7C046E40F00200E
:103DB000EC100020E410002000C0FEFF04C0020050
:103DC000E810002095C20000E02E0020F0B5002091
:103DD000B7B00024FFF7D8FE270005002600002D0D
:103DE0002ED1284D2868FFF769FE32003B00019074
:103DF0000094254904A806F04FFE04A800F0C0FF77
:103E0000224B64201C682B68A0215A425341204A4F
:103E10005B421340B02292029B18E41A60434902AD
:103E200004F0B2F9A02252020300009219492200C4
:103E300004A806F031FE04A800F0A2FF37B0F0BDE0
:103E4000FF226B6829689C460233FF180B1201366B
:103E500013409C4200DA1C00FF200A140240039227
:103E60006246014001920091039A0B4904A806F0B2
:103E700013FE04A800F084FF2800FFF785FE05006C
:103E8000ADE7C046E410002006C30000E8100020A3
:103E900000C0FEFFB0C20000F2C2000070B50020FA
:103EA000FFF70CFE04000120FFF708FE844200DA51
:103EB00004000A4B1D686A42554128001D60FFF747
:103EC000EDFDA0226B4252021340054A28009B18C8
:103ED000044A611C1360FFF715FE70BDE41000205A
:103EE00004800100E8100020F8B50020FFF7E6FD8F
:103EF00007000120FFF7E2FD3E00204D0643204C65
:103F00000DD18021C020C9024002FFF7ADFD012183
:103F10003000FFF7F7FD1B4B2E6023601DE087424A
:103F200009DD0023B0212B60164B89022360236832
:103F30000020012517E0012380212B60124BC902CC
:103F40002360F4E7120E522A08D0002800D0236024
:103F50000E4800F015FFFFF7A1FFF8BD28005A68D2
:103F6000023292009B188B4205D21A68561CE9D186
:103F70000028F2D0D1E72160EFE7C046E41000202E
:103F8000E81000200480010004C00200CBC2000041
:103F9000F0B585B0039203220333DC17294D14409A
:103FA000E4182B68284F5A42534180225B42D202C8
:103FB000A4103B409B18A21C0291244E910000913A
:103FC0000190316800980A18934215D2FFF71AFE43
:103FD0002B685A42534180225B421F40D202BF18D5
:103FE0003368009A9B189F4206D2194800F0C8FE19
:103FF0000025280005B0F0BD029B356819066B4608
:104000001A7BA423DB051343FF222F00090C19435D
:10401000019B12041B04134019432800FFF760FDA5
:104020000837281D21003760FFF75AFD002C04D007
:104030000A9A21003800FFF779FD009B083BFF1822
:104040003760D6E7E410002000C0FEFFE810002033
:104050006FC2000010B5FFF7D5FD10BD70B59AB066
:10406000FFF742FFFF221E4CD2000021200006F085
:10407000CFF9FF25FFF7B2FD0026002814D102007A
:10408000C300E3580130591E8B41D218FF28F7D1E5
:10409000144901A806F000FD01A800F071FE1248C5
:1040A00000F06EFE1AB070BD03681A142A400A2A86
:1040B0000AD11A122A40FF2A03D0D200A1180B718C
:1040C000A050FFF761FDD8E7132AFAD11B122B404D
:1040D000FF2BF6D0DB00E2181671E650F1E7C04680
:1040E000582500203BC300004FC300000021094BAE
:1040F000094A59600131516059680029FCD00021FA
:104100001961012393600222044B8131FF315A501F
:104110001A607047FC1000400010004000E100E011
:104120000222064B0121DA670022054B5A61054A3B
:1041300011615A69002AFCD07047C04604E100E0D2
:10414000FC1000400010004010B5044C2378002BF8
:1041500001D0FFF7E5FF0020207010BDED11002019
:104160000120024B1B685B0018437047701200204F
:1041700003480368002B02D11422037102607047C8
:10418000082F00200120024B1B685B00184370477A
:104190001000002070B504000D001600FEF7ACFB07
:1041A0008023012200215B055B6E6270E270020ACF
:1041B000A271020CE2711A0A60716372000EA2729F
:1041C0001A0C1B0E26702571A1702072E2722373E7
:1041D00070BD0000124B10B51B68124C5A1C0FD05A
:1041E000114C002B0CD0114C012B09D0104C022B80
:1041F00006D00D4C042B03D00E4C052B00D10B4CDC
:1042000021000D4806F080FC200006F085FC03002C
:10421000042204339B0809481B011343036010BDAB
:1042200014000020D7C30000D0C30000E2C3000088
:10423000E7C30000DCC30000F42E0020F02E0020B5
:1042400070B5214C2278002A3DD1204B01215A60C3
:104250008022D20511605A68002AFCD00022072073
:104260001B4B1C4901255A500439585008315A50EB
:1042700019481A4958501A491A485A501A495A5056
:10428000A622D2009D50082218495A500431585095
:1042900002201749585017491748585017480439F1
:1042A0005850182016495850C12189005A500539D4
:1042B000FF395858921802435A501249124A9950DD
:1042C000FFF714FF257070BDED110020FC000040C9
:1042D000001000400C050000746962751C050000A8
:1042E00024050000200004022C0500001405000035
:1042F000340500003C050000FFFF00002110010014
:1043000054050000EE1100200405000070B50E4BAE
:1043100006001B78002B01D1FFF792FF00200B4D08
:104320002C7884420ED00A4B202219780323091BD3
:104330001940084B4901C918300006F04DF801201A
:10434000013C2C7070BDC046ED110020741200209D
:10435000EC110020EE110020002370B588B09842C7
:1043600027DD0D6801262C0034409C4221D123001A
:10437000042D1ED90F222B681A402300092A18D1B8
:104380006A681F2A15D96846FFF7C0FF2300002876
:104390000FD06B4619783300A14203DB6B461B5DDF
:1043A0005B003343A200AA1801349360202CF2D1A1
:1043B0000423180008B070BD70B5414B8AB01B785B
:1043C000002B01D1FFF73CFF02AD2800FFF79EFF55
:1043D000002802D100200AB070BD2B780B2BF9D930
:1043E0006B78012BF6D1EB78012BF3D10023354EFE
:1043F000354C336023712B79344A1360002B0ED176
:10440000152169444A780B7812021A438B781B04F1
:104410001A43CB781B0613433360002318E0012BAB
:1044200020D1152169444A780B7812021A438B78FF
:104430001B041A43CB781A211B06134333600E2347
:104440006A7C6944934200DD130000229A4232D113
:1044500004200021E21804339B101B010343117157
:104460002360B8E7022B03D16A7B10331621E8E7FB
:10447000042B0DD1152108226944684605F0ACFFD4
:104480000098019902F036FA05F058FE3060C4E752
:10449000052BC2D1152108226944684605F09CFF0E
:1044A0000098019902F026FA05F048FE30606A7D16
:1044B0000A231E21C5E78D5CA01805710132C5E7EE
:1044C000ED11002070120020082F002014000020A1
:1044D00010B5134B04001B78002B01D1FFF7B0FE81
:1044E000FFF71EFE00200F4A0F49104B5450586032
:1044F0000130106058680028FCD00020186101309D
:10450000906018690028FCD0094B0A481B785B01B1
:104510001B185350FFF704FEFFF7E8FD10BDC0461F
:10452000ED1100200010004004050000FC100040C8
:10453000EC110020EE11002010B588B000281DDD20
:104540000A68012113000B4018D1042A16D90F2044
:1045500014682040092811D150681F280ED99800EE
:10456000101880680024084201D04010C4B2684688
:10457000C4540133202BF2D1FFF7AAFF002008B06A
:1045800010BD000010B5002813DD0C68E30710D53E
:104590006410532C0DD8084B1B78002B01D1FFF76A
:1045A0004FFEFFF7BDFDA123044ADB00D450FFF707
:1045B0009DFD002010BDC046ED1100200010004000
:1045C00010B500280EDD0C68E3070BD56410FF2C36
:1045D00008D8054B1B78002B01D1FFF731FE034AA9
:1045E000034BD450002010BDED11002000100040FE
:1045F0002405000013B5002814DD0C68E30711D56D
:10460000094B64100093094B0193072C0AD8084BFF
:104610001B78002B01D1FFF713FE6B46054A195793
:10462000054BD150002016BDE2ECF0F4F8FC00047C
:10463000ED110020001000400C05000070B588B09E
:10464000002820DD0124086804401CD104281AD960
:104650000F2302681340042B15D1FEF745FB06001B
:1046600006F05AFA0500122800D912252A00022164
:104670000D326846FFF78EFD6B465D73A54205DC83
:104680006846FFF725FF002008B070BD2300325DAB
:104690006B449A730134F1E7F0B50D008BB001283B
:1046A00032DD08680122040014402DD104282BD9E2
:1046B0000F2301680B40042B26D16B68134223D0D3
:1046C000FEF712FB6E6807007310019306F024FAE0
:1046D00005000E2800D90E252A000121113202A85A
:1046E000FFF758FD6A46127902AB5A7302AA731299
:1046F0009373019B76141B0ED67313745574A542E5
:1047000005DC02A8FFF7E4FE00200BB0F0BD3A5D27
:1047100002A963189A740134F1E730B589B0002812
:1047200014DD0C68E30711D5102268460021FFF75D
:1047300031FD6B466A4665105D73684663122D0E47
:1047400064149373D4731574FFF7C2FE002009B08C
:1047500030BD0000174B184A5968002903D00021CA
:10476000596001319160196900291FD0002018613A
:104770008023DB00D3581149012B18D1A923DB007A
:10478000D3585B420B600E490B78032B01D80133E1
:104790000B7003200B490B78013303400B700A495F
:1047A0005B015B180949535001239360704708600F
:1047B000FAE7C046FC100040001000401000002046
:1047C00074120020EC110020EE11002004050000FE
:1047D00010B5034A0E21034800F0B4F810BDC046DE
:1047E00060C3000057C30000044A05491368C85459
:1047F00001339B059B0D13607047C0469016002047
:104800009012002070B5114C114A2368834202DCDB
:104810000023236016E0155C411C2E00FA3E012E99
:1048200005D899420FDA555C013D1F2D01D90800CA
:10483000ECE70100151A565C6E5401318B42FADC2C
:10484000181A206070BD1570FAE7C0469C1A002047
:104850009C16002010B5FEF745F8064B1A688242F8
:1048600001D900221A601B68C31A0348984280418C
:10487000404210BD8C120020204E000010B5094CA3
:10488000094A23681268934200D110BD074AD05CE0
:10489000FEF7ACF90028F8D0236801339B059B0D87
:1048A0002360ECE794160020901600209012002060
:1048B00010B50400064B074A1B6812689B1ADB43BD
:1048C0009B059B0DA34200DB10BDFFF7D7FFF1E76F
:1048D0009016002094160020F7B505005668019147
:1048E000B000441C06301700FFF7E2FFFB20FFF783
:1048F0007BFF1C20FFF778FFE8B2FFF775FFE0B2FF
:104900002412FFF771FFE0B2FFF76EFF6B461879D4
:10491000FFF76AFF0025AE4200DCF7BDAB00FB18D5
:104920009C680135E0B2FFF75FFF2012C0B2FFF7CD
:104930005BFF2014C0B2FFF757FF200EFFF754FFB4
:10494000E9E7000070B5074E3368092B08DC0C2539
:104950005D43054C0133285164196160A2603360E6
:1049600070BDC046981600202C2F0020F0B587B0EF
:1049700002900C00012803DC1B20FCF7E7FA45E05D
:10498000244B08680093C30709D4042807D90F23D0
:1049900002681340042B02D1FEF7A6F900901D4BCC
:1049A00060680193C30709D4042807D90F2302685C
:1049B0001340042B02D1FEF797F901900027164B04
:1049C0001B680493049BBB42D6DD0C267E43134B2D
:1049D0000099F618306806F08DF8051E05D1736849
:1049E000B6680593059B9D4201DB0137EAE7306815
:1049F0000199039606F07EF80836002808D12100B8
:104A00000298039B083102385B68984707B0F0BDF5
:104A10000135E7E7CFBD0000981600202C2F0020BD
:104A200010B5FCF7DFF9FFF713F8FEF781F8FEF792
:104A3000CFFBFEF705FCFFF7CBFE00F049FE01F0CF
:104A400023F810BD962210B512010021034805F08D
:104A5000DFFC0022024B1A6010BDC046F81B00208C
:104A6000B8050020064B074A1B6812689B1ADB43F7
:104A70009B059B0D0122834200DC00221000704741
:104A80009016002094160020F8B505000C001600C2
:104A90001F1E0ED10320FFF7E5FF002808D0FA20E3
:104AA000FFF7A2FEE8B2FFF79FFEE0B2FFF79CFE21
:104AB000F8BD501DFFF7D6FF0028F9D0FB20FFF707
:104AC00093FEE8B2FFF790FEE0B2FFF78DFEF0B282
:104AD000FFF78AFE3012C0B2FFF786FE3C00E31BF0
:104AE0009E42E5DD2078FFF77FFE0134F7E7000006
:104AF00070B50024F0250B4B1B68A34202DCFFF7C6
:104B0000A1FF70BD2B006343074A9B181A78002A47
:104B100005D05978002311201A00FFF7B5FF0134A2
:104B2000E9E7C046B8050020F81B0020F8B50700EB
:104B30000024F0252B0063430C4A01349E18B74231
:104B400011D0317800290BD00133D15C0023112022
:104B50001A00FFF799FF2A000021300005F058FCE9
:104B60000A2CE7D1F8BD024B1C60F9E7F81B0020C6
:104B7000B8050020F0B5150001222F005E4C17404B
:104B8000A54401900291002F11D005AB1A706A1054
:104B90005A70120E1A710522691299706D140299D9
:104BA000DD70FFF771FFCF239B009D44F0BD042D06
:104BB0001ED90F232A681340042B25D1023B04AAD7
:104BC00028001371FEF790F8040005F0A5FF4B4B89
:104BD000984200D91800B84204DC421C05AB029987
:104BE0000198DEE701377B1EE35C05AAD355F2E7A7
:104BF000042D7CD1032304AA043D13716B425D4153
:104C000005AB55710222EAE7092BCCD1042205AB92
:104C10001A706A68511000916946521209789A70A8
:104C2000009A59701F2A01DD202200926A461278EC
:104C300006ACDA70009BBB4202DC05ABE21ACEE7A1
:104C40000126BB00EB189868064006D1042837D926
:104C50000F2302681340022B0CD101232370431051
:104C6000637042121B0E4014A270E0702371053471
:104C70000137DFE7042B21D1023B2370FEF734F824
:104C8000039005F049FFA31C0C2809D860708642E8
:104C900001D19C19ECE7039A925D9A550136F6E72B
:104CA0000C226270039A925D9A550136092EF9D151
:104CB0002E23E372237363730E34D9E7012B07D1DC
:104CC0000323043823704342584160700234CFE715
:104CD000092B09D1053B23704368E6705A105B121B
:104CE0006270A3700434C3E726700134C0E7002D5E
:104CF00000D058E77EE7C046C4FCFFFF2303000056
:104D000070B502000024F0210D4E080060438019A8
:104D10004578954203D001340A2CF6D170BDF022BB
:104D2000002105F075FB074A1368013BA34200D13F
:104D30001460002329001A001120FFF7A5FEEDE7FB
:104D4000F81B0020B805002010B5B2B002236A4657
:104D50000400137005F0E0FEC72800D9C720002327
:104D6000984207DC421C6B46FE211420FFF78CFEA4
:104D700032B010BD694601335A1EA25CCA54EFE737
:104D800030B5B3B002236A460500137005F0C4FEC7
:104D90000400C72800D9C72400239C420BDC200054
:104DA0003230FFF785FD621C6B46FF211420FFF7B0
:104DB0006BFE33B030BD694601335A1EAA5CCA543B
:104DC000EBE70000F7B5234B06001B68F0210093CA
:104DD0000023009A9A4211DC0024F0231A00624357
:104DE000019201991C4A55182F78002F12D00134D6
:104DF0000A2CF3D11948FFF7C3FF29E00A005A43F0
:104E0000154882185078B04202D11278002A1FD17A
:104E10000133DEE7F0223900280005F0F9FA022319
:104E20000D4A0199EB6053540D4AF1008A58009BDA
:104E30006E70AE70AA602F616F61A34202DC054BF9
:104E400001341C60002331001A001020FFF71CFE03
:104E5000F7BDC046B8050020F81B0020D1C80000EF
:104E60005825002010B5FFF743FEFF24084AE30051
:104E70005B429B18074AD35C043B012B03D8E043F9
:104E8000C0B2FFF79FFF013C002CEFD110BDC04620
:104E9000FC07000058250020F7B50F00FF247F25F0
:104EA00001901E4AE300D31A1D4A9A181278062A66
:104EB00001D0032A20D1FF22D2009B1818688368F2
:104EC0002B401C2B18D1C3681A002A40042A13D186
:104ED00002692A40192A0FD11B0A01339B000C30AA
:104EE000C018FDF701FF03780600002B10D005F075
:104EF00013FE0023B84209D0013C002CD1D1F7BDEC
:104F0000019AF15CD25C9142F6D101339F42F7DC09
:104F1000E043C0B2FFF756FFEEE7C0465825002039
:104F2000FC07000070B50500FF24084AE3005B425F
:104F30009B18074AD35CAB4203D1E043C0B2FFF7F2
:104F400041FF013C002CF0D170BDC046FC070000C1
:104F500058250020F7B5FDF7C5FC514B1A68824271
:104F600001D900221A601A684E49821A8A4200D872
:104F700083E01860FDF7C0FC071E00D10137002058
:104F8000FDF7ACFD01900020FDF7BCFD019B0090FA
:104F9000454C464D002B14D02368002B00D07AE0FE
:104FA0002B682760002B00D171E0414B01261B7854
:104FB000002B63D10920FFF7B5FF3E4B1E703C4B21
:104FC0001E70009B002B12D02B68002B0FD1236882
:104FD0002F60002B1ED0374B01261B78002B52D19F
:104FE0000920FFF79FFF334B1E70314B1E70236863
:104FF000002B0FD02F4E3278002A0BD19F4200D2C7
:1050000027602368FB1A312B04D90720FFF78AFF9A
:10501000012333702B68002B0FD0254E3278002AE5
:105020000BD1BB4200D92F602B68FF1A312F04D956
:105030000820FFF777FF012333702368002B0CD083
:10504000019B002B09D11B4E3378002B02D1072086
:10505000FFF768FF0023236033702B68002B0CD010
:10506000009B002B09D1124C2378002B02D1082081
:10507000FFF758FF00232B602370F7BD0720FFF7D1
:1050800051FF0C4B9CE70820FFF74CFFADE7009B5E
:10509000002B9CD1ABE7009A002A95D1AAE7C04625
:1050A000881200200F2700007812002080120020B4
:1050B000841200207C12002037B500240500FFF781
:1050C00017FD01A80194FDF7F7FC21002000FEF771
:1050D000DFF9FEF76BFBFDF729FDFDF728FDFEF775
:1050E000B1FCFDF725FCA54204D0FDF7A9FD02485F
:1050F000FFF746FE37BDC046C2C80000002310B50A
:1051000001001A001120FFF7BFFC10BD07B56B4668
:10511000197069465A7013128B701314120ECB70EB
:105120000A716B46010005221320FFF7ADFC07BD95
:1051300010B50A0001001220FFF71CFD10BD70B56C
:10514000050008000C003230FFF7B2FB2B002200F4
:1051500000211B20FFF798FC70BD10B50C00030068
:10516000110014202200FFF78FFC10BD012370B541
:10517000FF24084A41185B42884201D3D84370BDDE
:1051800006781D0A234073409B009B5801306B40FA
:10519000F2E7C046A4C40000002313B501930B4BF3
:1051A000C2000400D058002805D043680830990098
:1051B000FFF7DCFF01900920FFF77AFB01AB042227
:1051C00021001720FFF760FC13BDC04658250020C2
:1051D00070B506000020FEF7D7FC0024FF2500284C
:1051E00001D1200070BD03681A142A40152A07D186
:1051F0001B122B40B34200D10400FEF7C5FCEEE7C2
:105200001D2AFAD10024F8E7F0B580279DB0FFF7FA
:1052100035FBAD4CAD4D2068FF00391A4019FDF744
:10522000CBFC23680600C3182360002B0ED11DB0F1
:10523000F0BD2068391A2818FDF7BEFC2368060067
:105240001B182360FDF74EFBA14B1860002EF0DC0D
:105250002B78FA2B00D013E12368022B07DCFFF731
:10526000F9FA0028E3D00120FFF7CCFADFE76878ED
:10527000AC78023818281FD802F0F2FE0D2024283E
:105280002B341E3E6872768CDEEF1E1E1E1E1E1E06
:105290001E1E1E1EFD00FF2C0ED02000FFF730FD4D
:1052A00000228C4BE100CA505B181A712100009259
:1052B00013001320FEF76CFE0320D5E72000FFF754
:1052C00081FDF9E72000FFF71BFDF5E7FFF7CAFDB9
:1052D000F2E7FFF70DFC0020FFF7EEFE7E48FFF738
:1052E0004FFDE9E7632CE7D87C4BA200D2582100A0
:1052F0001520FFF73FFCDFE700242000FFF768FFE1
:10530000061E03D10134642CF7D1D5E7083005F02F
:1053100003FC05000530FFF7CBFAFB20FFF764FA2A
:105320001D20FFF761FAE0B2FFF75EFAE8B2FFF77F
:105330005BFA2812C0B2FFF757FA3700BB1B9D4239
:10534000E0DD387AFFF750FA0137F7E700211D203A
:1053500000910B000A00FEF71BFEFDF771FCABE7A6
:105360002000FFF719FFA7E7FDF7CEFA03AC5C4A70
:10537000642100905B4B200005F05CFB02232000C1
:10538000237005F0C9FB2300020000211620FFF75F
:105390007BFB91E700244F4AE300D558002D28D02D
:1053A0006B689E00701DFFF783FA2B00002532000A
:1053B000083321000120FFF767FB0020FEF7E4FB24
:1053C0002F002E00002818D1002F04D03A00012110
:1053D0002000FFF781FA002D04D02A0002212000CE
:1053E000FFF77AFA002E04D0320000212000FFF7E8
:1053F00073FA0134FF2CCED15EE7FF2103681A1245
:105400000A40A24209D11A140A400B2A08D10B40C3
:105410000CD0012B0CD0022B0CD0FEF7B5FBD1E742
:10542000132AFAD100252F002E00F6E70600F4E734
:105430000700F2E70500F0E70024FFF759FB220020
:10544000210000942300DA20FEF7A2FDFF222100B4
:10545000D200204804F0DCFF7FE7012C02D1FEF7E8
:10546000B5FC29E7022C02D1FEF7F4FD24E7012068
:10547000FFF722FE20E7002321001A001A2086E70A
:10548000FB2B00D0EFE62268042A00DCE7E62E7949
:10549000E878154B360206439E4200DDE3E6331DF5
:1054A0009A4200DCDBE6EB5CFE2B00D0DBE66B789F
:1054B000AC78711E1B2B6BD018D8012B2BD0082B6E
:1054C0003DD0701DD0E6C0469C1A00209C160020DE
:1054D0008C12002058250020A4C80000502D002068
:1054E000BBC80000B6C80000F60300001D2B60D04A
:1054F00052D31E2BE5D1012CE3D10029E1DD6B79DC
:10550000002B03D01C00322B00DD322464235C43CB
:10551000344B1C60D5E7FF2CD3D02000FFF7F0FB05
:105520006D79314AB31E009221002A000A20FEF74D
:105530002FFD2E4BE400E0501B191D71C1E7632CB9
:10554000BFD86A79022A13D0032A1BD0012AB8D106
:10555000E979AB79090219432B7AA4001B0419439A
:105560006B7A1B060B435B001343214AA350A8E749
:105570000029A6DDB11E1C48FDF7C4FD1C4BA4008C
:10558000E0509EE7AB79A4005A1E93419B00ECE7E4
:105590001848FFF781FC94E7FF2C92D06A79022A21
:1055A0008FD811490B2000912100B31EFEF7F0FCAB
:1055B00087E70B00632900DD6323002203A89342E1
:1055C0000ADCD9430022C917194041180A70013377
:1055D000009021001520E9E7A9184979815401328A
:1055E000EDE7C04604000020A21600205825002048
:1055F000502D0020A11600200122094B1A60094AF3
:105600001368002BFCD00322074B1B68D8171040EF
:10561000C018012380100638400018437047C04668
:1056200000C0004000C1004008C500400120704794
:1056300010B5064C200000F0A5FA0549200000F046
:10564000C9FA0122034B1A6010BDC046A81A0020F7
:10565000801A0600A01A002010B501210D20FDF7C8
:1056600059F901210E20FDF755F900210F20FDF712
:1056700051F9044C200000F011FC1021200000F032
:1056800029FC10BD601B002010B504680D20E30745
:1056900003D56410FF2C03D91720FBF757FC10BD6E
:1056A000FFF7DAFFE1B2024800F036FC0020F6E72F
:1056B000601B002010B5FFF7CFFF0021034800F06A
:1056C0002BFC43000120184310BDC046601B002086
:1056D00010B5034A08210348FFF734F910BDC0464E
:1056E000E8C8000028C900000D4B70B51B68040015
:1056F0000E001500002B01D1FFF79AFFE1B2094C13
:10570000200000F0FEFAF1B2200000F001FAE9B248
:10571000200000F0FDF9200000F05EFB70BDC046E7
:10572000A01A0020A81A002010B501240368234203
:1057300005D04168214202D08268224203D10D2067
:10574000FBF704FC10BD5810802801D91520F7E79D
:105750004910FF2901D91620F2E75210FF2A01D97A
:105760001720EDE7FFF7C0FF0020EBE7F7B50124B6
:105770002300A0421DDD0D682C421AD01A4B254192
:105780001B684C68002B01D1FFF752FFE9B20127DB
:105790002500164E3D40300000F0B3FA002D0AD02F
:1057A0003C413000E1B200F0B3F9300000F014FBEE
:1057B00000231800FEBD042CF7D90F2322681340E4
:1057C000092BF2D163685B100193019BAB42ECDDC6
:1057D000AB00E3189968394204D04910C9B23000CF
:1057E00000F096F90135F0E7A01A0020A81A002071
:1057F000144B70B51B6805000E00002B01D1FFF79C
:1058000017FF114CEDB22900200000F07AFAF1B236
:10581000200000F07DF90021200000F07DFA002832
:1058200001D0404270BD01222900200000F064FA3E
:10583000200000F05EF90028FAD0200000F05EF9A8
:10584000F0E7C046A01A0020A81A002010B50124D5
:105850000368234202D04168214203D10D20FBF7A7
:1058600075FB10BD5810802801D91520F7E74910A5
:10587000FF2901D91620F2E7FFF7BAFF40002043C5
:10588000EFE70000002370B5344D0400EB56013300
:105890000BD10D211D20FFF7ABFF5A2814D1012297
:1058A0002A212A703D38FFF71FFF0023EB56022BF9
:1058B0002AD0032B49D0012B4CD121001D200124DB
:1058C000FFF796FF644225E00F211920FFF790FFB4
:1058D000332805D102235F222B7020211A38E2E7FA
:1058E0000D211E20FFF784FFC7280AD103230022C1
:1058F0002A21A9382B70FFF7F7FE1B222A211E2030
:10590000D1E700232B70D0E7012C13D129211920D6
:10591000FFF76EFF7F2801DD0138FF3803007F337A
:1059200001DA7F20404264237F21584302F02CFC9F
:10593000604370BD032C0BD12B211920FFF758FFBA
:10594000043CE7E72D211920B9E721001E20B6E726
:10595000052CF7D0012400206442E4E71800002061
:1059600070B50120FFF78EFF04000320FFF78AFFC8
:1059700005000520FFF786FF6D436443404364192B
:10598000201804F011FC01F0E5F804F0D7FB430007
:105990000120184370BD10B50120FFF773FF4300CD
:1059A0000120184310BD10B50320FFF76BFF430023
:1059B0000120184310BD10B50520FFF763FF430019
:1059C0000120184310BD0000F8B501231C009842C7
:1059D00034DD0F683B4231D04E6835001D402DD17B
:1059E000042E2BD90F2231680A40092A26D1736868
:1059F0005C10202C00DD2024114B1B68002B01D1F2
:105A0000FFF716FE7F10F9B20E4F2200380000F0AB
:105A100073F9A5420FDA380000F06BF80028FAD0CD
:105A2000380000F06BF80122AB004000F31810437F
:105A30009860AD18EDE70120640004432000F8BD34
:105A4000A01A0020A81A00200020704701207047EB
:105A500000207047002070470120704700207047E9
:105A600000207047002070470020704700207047DA
:105A700000207047002070470020704700207047CA
:105A8000704770477047000010B5034A0E21034865
:105A9000FEF758FF10BDC04678C90000E8C90000F5
:105AA00010B5FDF751F8FDF7F1F8FEF7B9FF04481E
:105AB000FFF766F9FEF7D2FAFFF7D4F910BDC0463A
:105AC00071CA000010B5FCF7A7FE10BDF8B50500BF
:105AD0000E0017000024BC4208D02B68315D1B6803
:105AE00028009847002801D00134F4E72000F8BDD1
:105AF000704710B51C3000F061FA10BD10B51C30B5
:105B000000F04EFA10BD10B51C3000F05DFA10BD6B
:105B100070B5437E0D00002B01D1002070BD6430B4
:105B2000040000F05AFA0028F7D12000290000F004
:105B300028FA0120F2E70000F7B50193FA230025C7
:105B400004009B0083600D4B4560083303601C30EC
:105B50000F00160000F00AFA2000643000F006FA88
:105B6000074A2761B600B35820006375019B9B006C
:105B70009B586576A576A375FEBDC0468CCA00000D
:105B800050CB00000123A022C375837D0E49C13391
:105B9000FF33D2059B009950437DC133FF339B00F7
:105BA0009950CC220169094B5204CA50052201695F
:105BB000243BCA50827D01690833CA500269417D85
:105BC000034BD1507047C0460C060000240500006E
:105BD0000C050000A022002310B50469D200A350D8
:105BE0000A4CA1420FD90A4C8C425B4109495B42E5
:105BF0000B40CD21C9045B18046907496350052196
:105C00000369995010BDCC235B04F5E7A086010021
:105C100090D00300000098FD24050000F7B50400B3
:105C200000200D000193824265D01600402A00D961
:105C3000402627001C37380000F0AEF9B123226956
:105C4000DB00D55080220123216992008B50A27E77
:105C5000002A03D122691362226913600025731E92
:105C6000AB4207D1019B002B04D080220221236983
:105C700092009950012223691A622369FC33DA6881
:105C8000002A02D19A6A002AF9D09A6A002A0BD116
:105C9000DA60A3232269DB00D1583800C9B201358C
:105CA00000F06FF9B542DAD3019B2269002B0FD1C6
:105CB0001300FC339B6A002B0AD10133A376D36116
:105CC0002369FC33DA6C002AFCD00022DA640AE093
:105CD00000230121A37651611A002369FC339968DE
:105CE0000029FCD09A602369FC339A6A002A01D00B
:105CF00000229A62E8B2FEBD10B50123FFF78EFFC5
:105D000010BD0300AC3310B504001970643000F00E
:105D100043F90123637610BD0023020070B5AC3255
:105D200043760D001178B12204000069D200815041
:105D30008022216992008B5022690133136222690B
:105D4000936026006436300000F038F9002812D045
:105D5000300000F025F91E4B2269D0502369FC3336
:105D60001A6A002A02D19A6A002AF9D09A6A002A8D
:105D700001D11A62E5E723690122002D0DD1190036
:105D8000FC31896A002908D1DA612369FC33DA6CB5
:105D9000002AFCD00022DA6407E05A612369FC3350
:105DA0009A68002AFCD000229A6000202369FC3304
:105DB0009A6A82420BD098622169064A8B588B50AE
:105DC0001800022B03D0181F431E9841033070BDEA
:105DD0001C050000C404000010B50121FFF79CFF62
:105DE00010BD000010B51323142202490248FFF72A
:105DF000A3FE10BD00400040A81A002070B5002589
:105E000004AC24780573A94205D10A4B0A4A232120
:105E10000A4804F073FA01600949920052589B0045
:105E200002715B58A400837163588560437102233B
:105E3000C37170BDACCA000011CB0000BACA00002B
:105E400050CB0000037B002B04D1437383730361A9
:105E500001330373704700001FB50191A021002496
:105E60000068C900D2B24450012A10D0A24209D021
:105E7000032A0AD0074A8350074B019AC2500123D4
:105E800043501FBD02221343F4E70422FBE706221E
:105E9000F9E7C046540500002405000010B50400D1
:105EA000FFF7D0FFA1222368A179D2009950617930
:105EB000064A20009950217904329950044B196800
:105EC0005A689B68FFF7C8FF10BDC0460C0500006C
:105ED000741B00204BB2002B0FDB80233F290FD80F
:105EE0001F290FD80F290FD807290FD803290FD83A
:105EF0001B060168074A8B50704780239B04F8E714
:105F0000DB04F6E71B05F4E75B05F2E79B05F0E72A
:105F1000DB05EEE7240500000368074A99501A00E4
:105F2000FC32D1680029FCD0A321C90058580023B5
:105F3000C0B2D3607047C0461C05000007B5802280
:105F4000074BD2051A6000229A6002321A710F23A1
:105F50000C3200930349023B0348FFF74FFF07BD94
:105F6000741B002000300040601B002010B5402250
:105F70000021040004F04CFA002320002364636431
:105F800010BD10B53F24026C531C2340446C9C424E
:105F900001D08154036410BD00230364436470473F
:105FA000436C026C934206D03F21C25C01330B402C
:105FB00043641000704701204042FBE7036C406CD3
:105FC000181A00D540307047436C026C934201D0E0
:105FD000C05C704701204042FBE73F22036C406CED
:105FE00001331340181A43425841C0B270470000B1
:105FF00003210A4802680A430260094802680A430A
:1060000002600849084A094B9B1A03DD043BC85843
:10601000D050FBDC00F012F8FAF776F824050040C7
:1060200054050040A4D000000000002050020020D1
:10603000FEE7FEE7FEE7FEE7FEE7FEE72D4B10B5C5
:106040001A68D2B2012A0FD12B4A126812070BD15B
:106050002A4AE0241168F0220800104021422DD184
:106060002749096811422CD01A68D2B2012A12D1EC
:106070002149096809070ED1F0202049096801402B
:10608000402908D11E490968014204D18020C1215C
:10609000C005C90042501B68DBB2012B0DD1164B65
:1060A0001B681B0709D1154B1A68F0231A40A02A58
:1060B0000FD1134A12681A420ED010BD3028CFD02B
:1060C000D2E7104A104911608021104A090211607C
:1060D000CAE7D02AF1D1ECE70D4B1A68012A04D0A7
:1060E0000C4A1A601A68012AFCD1C0220A4B1A60B5
:1060F000E3E7C046E00F00F0E40F00F0E80F00F027
:10610000EC0F00F004050040DFFF07C0186C0040F2
:1061100000EC06407593000014EC06400120704727
:1061200010B503681322DB69984710BD7047000063
:10613000054B0269D1500369FC331A6A002AFCD06E
:10614000002201201A6270471C050000030010B5F0
:106150005C331A781F231A401E3B19009140114AE4
:10616000D167C222042104699200A15002695360E0
:106170000269D360A02300220169DB00CA50012319
:106180000169094A5B428B500169084A8B500169D9
:106190000C3A8B50016908328B501430FFF7FCFE2B
:1061A00010BDC04604E100E00C050000140500002D
:1061B00010B51430FFF702FF10BD10B51430FFF713
:1061C00003FF10BD10B51430FFF7EAFE10BD00004C
:1061D000030070B55E331A780469724BE250030015
:1061E0005D331A780469704BE250030061331C7808
:1061F00002696E4B012C00D09EE005005F352E78C1
:10620000A225ED005651020060321578A1220669E0
:10621000D200B5500269D4509623DB00994200D8D1
:106220008CE096231B01994200D88AE096235B01FB
:10623000994200D888E096239B01994200D885E0D6
:10624000E1239B01994200D882E09623DB01994229
:1062500000D880E0E123DB01994200D87DE096235D
:106260001B02994200D87AE0E1231B02994200D830
:1062700077E096235B02994200D874E0E1235B0249
:10628000994200D871E0E1239B02994200D86EE068
:10629000474B994200D86CE0E123DB02994200D8D9
:1062A0006AE0E122002312038A425B41414A5B42D9
:1062B0001340802252059B1801693F4A8B50A0234E
:1062C00004220169DB00CA5000210369FC33D96054
:1062D0000369FC331962012301690B6001698B605A
:1062E000C1210469890062501F215C3002780A4094
:1062F00093406231314AFF31535000214156002909
:106300003CDA0F230B40083B2D4C9B089B001B19CC
:1063100003242140A140FC348C40DD69A5432C00BE
:10632000C0258D4029002143D9611F2301781940E0
:106330001E3B8B40136070BD00246CE79E23DB0284
:10634000BAE79D231B03B7E71E4BB5E71E4BB3E728
:10635000EC239B03B0E71D4BAEE71D4BACE71D4B99
:10636000AAE71D4BA8E71D4BA6E71D4BA4E71D4B55
:10637000A2E78023DB049FE71B4B9DE78C080F4BB4
:10638000A400E41803230B40FF21C025DB00994043
:10639000AD0066598E433100C0269E4033000B434A
:1063A0006351C2E70C050000140500006C050000F5
:1063B00090D0030000D0BEFE2405000000E100E004
:1063C00000ED00E000B013000050270000A04E00D8
:1063D00000F0750000509D0000F0EB0000903A01C5
:1063E00000E0D70100B0AF0300705F07F7B500937E
:1063F00008AB1B7800250193FA2304009B008360FF
:106400000E4B45600833036014300F001600FFF791
:10641000ADFD23005C3327611E70009B084A9B0082
:10642000995823005D331970019B20009B009A58F6
:1064300023005E33DD701A70FEBDC046D4CB000071
:1064400050CB0000036910B51A00FC32D26804007A
:10645000002A0AD0A322D20099581430C9B2FFF7FB
:1064600090FD00222369FC33DA6010BD10B50248AC
:10647000FFF7E8FF10BDC046801B0020162307B5BC
:10648000022200930249013B0248FFF7AFFF07BD1C
:1064900000200040801B002010B5002801D004F02F
:1064A00073FA10BD7047000010B500F011F8FFF747
:1064B000F9FF012000F000FAFFF7F2FAFFF702FB04
:1064C000024B002BFAD000E000BFF7E7000000000D
:1064D000C420114B80001A5810491140C0221202EA
:1064E0000A431A50C0218022490092025A501A6071
:1064F0008023A3220021DB05D20099500122F9302C
:106500009A60074BFF301950C120023180001950AA
:10651000403019501A60704700E100E0FF00FFFFB3
:1065200000100140014B18607047C0466400002015
:10653000F7B5002320285AD8384B8000C258042AC7
:106540005BD007D8022A54D055D80423012A09D099
:1065500000234CE0062A54D051D31A2A53D00223E8
:106560001B2AF5D12E4A116808294ED909294FD086
:106570000A240226A02001252A4AC00015502A48D4
:106580002A4D07681C20BF00074029480197006872
:106590005759009027481B0207401F43C02300980B
:1065A0009B020340FF2057515759000207401F43E9
:1065B000019B1F43009B58016023184007433E4343
:1065C000565101251C4B156058680028FCD000204E
:1065D0005860A1230125DB00D3585560A025ED00AC
:1065E00050511BB2A14202D015D2611ACB40180003
:1065F000FEBD0823B6E71023B4E72023B2E740230B
:10660000B0E78023AEE70123ACE708240026B1E71A
:106610000C000126AEE7091B8B40E8E750CB0000D9
:1066200060000020007000401C00002004050000F5
:1066300020000020FF00FFFFFC700040F0B5202884
:106640005BD8364B8000C258354B1E68002E30D1C7
:10665000C227344BBF00D859334C03250440C02017
:1066600000022043D851C0248020640080001851CB
:106670002E4F18602E4B803CD859FF3CA043D85178
:106680000437D859A8432043D8510837D8590C3576
:10669000A8438446072065462843D851A820C00057
:1066A0001E50C1208026800076021E501C601C4BAC
:1066B0001C60142500202B001E4C2E00464336592A
:1066C000771C1BD14343E250A0230325C132FF3284
:1066D0009200DB05D550184B1A68082A14D11423F0
:1066E0004343E3189A6812485132FF3292005960CE
:1066F0001150DA68C1239B00C250F0BD9642E1D030
:1067000001300328D9D1F8E7082A02D9083AD14044
:10671000E5E708239A1A9140E1E7C04650CB000014
:10672000E41B002000E100E0FF00FFFF0405000083
:106730000090004024000020640000202149F0B5B2
:106740004A6C2148002A14D0A025A1260023012448
:10675000ED05F600C258571C06D0C7187F68002FF9
:1067600002D027009740AF5114333C2BF2D10023C5
:106770004B64A0230121DB0500260F009C46142357
:106780004B43C3181A1F1268104C0E4D9200141977
:106790005219526C002A10D01A00143A1268551C73
:1067A00009D0103B1B68FF2B05D03B00934065468A
:1067B0001A00074BEA50FC34666401310429DED12B
:1067C000F0BDC046FC900040240000200090004036
:1067D0000C05000000B5202810D80C4A8000835812
:1067E00003290BD8A0220800C133FF33D2059B0038
:1067F00001F036FC020905070021D15000BD0C2133
:10680000FBE70421F9E70321F7E7C04650CB00007E
:1068100020280AD8074B8000C25801239340A022A9
:10682000D205002902D1044953507047A121C90063
:10683000FAE7C04650CB00000C0500000300002022
:10684000202B0AD8A021A222C905D2008858034AC9
:106850009B009B58D84001231840704750CB000044
:10686000F7B506000D000C008B180193019B671B08
:106870009C4207D0336821781B6830009847013468
:106880000028F3D13800FEBD0849094A094B10B56C
:106890001B688858FA22190A1B0618439200002325
:1068A00001F0AAFD4904C00B084310BD00100140CF
:1068B00004050000E81B002070B5041E09D0FFF796
:1068C000E3FF050000F014F8FFF7DEFF401BA042D5
:1068D000F8D370BD0022044B9A60044A1368013358
:1068E000DBB213607047C046FC100140E81B00207B
:1068F00070470000F0B5C64600B5CB0F9846404A39
:106900004B005B0D9A1882B00D000400132A2FDC97
:10691000002A49DB3B4F17413E000E40064323D07F
:106920007F08390029400C430AD03749BD438C46C3
:1069300063445C425C418023DB021341E4071D4356
:106940004146CE0031492B008E192200346875680B
:106950002000290001F0F6FE0090019100980199B5
:1069600022002B0003F086F802B004BC9046F0BD74
:10697000332A08DD8023DB009A42F5D102000B00A8
:1069800001F0E0FEF0E7224A9446012263445242BD
:10699000DA400242E8D052080242D1D09443802229
:1069A000D2051A411443CBE74B005B080343DBD00D
:1069B0000B031B0B1C436342234380244D0C240315
:1069C0001B0B23406D042B4319004346DA000F4B89
:1069D0009B181C685D6802000B002000290001F074
:1069E000B1FE009001910098019922002B0003F064
:1069F00041F842464B005B08D60733431900B3E722
:106A000001FCFFFFFFFF0F00EEFBFFFF08CC0000C3
:106A1000EDFBFFFFF8B5274A4B005B0D9A180C0001
:106A20000700132A10DC002A36DB234B13410B42EC
:106A30003AD0802424031441002064189C430600AB
:106A4000250030002900F8BD332A0EDD8023060022
:106A5000DB000D009A42F4D102000B003800210047
:106A600001F070FE06000D00EBE7144D0600AC4689
:106A7000012563446D42DD40AC4663460D00034290
:106A8000DFD033239A1A323B93401818874200D93B
:106A90004C1C63469843D2E7C90FCC070020531C17
:106AA000CDD1074B1C43CAE706000D000028C0D11A
:106AB000C7E7C04601FCFFFFFFFF0F00EDFBFFFF34
:106AC0000000F03F30B5214A4B0087B05B0893428D
:106AD0001EDD1F4A934205DD02000B0002F0CAFFD3
:106AE00007B030BD02AA00F095F803231840049ABD
:106AF000059B012813D002281DD0002814D002982D
:106B0000039900F06FFB80231B069C466144E7E776
:106B1000002300220093002301F0DEF8E0E7029852
:106B2000039900F05FFBDBE70124029803990094CE
:106B300001F0D2F8D4E7012402980399009401F0FF
:106B4000CBF880231B069C466144C9E7FB21E93F43
:106B5000FFFFEF7FF0B54746CE4680B58DB004000D
:106B60000D0000F067FA294B06001B780F005BB29E
:106B70009846013310D022002B002000290003F09A
:106B8000C1FA8146002807D10022002320002900F5
:106B900001F00AFC002806D1300039000DB00CBC11
:106BA00090469946F0BD01230293194B0694079530
:106BB00003934B460A93434604940595002B15D046
:106BC000002300221900100002F0D8F84346089074
:106BD0000991022B0ED103F0AFFB212303600A9B26
:106BE0000193002B0CD1089E099FD5E700230024B8
:106BF0000893099402A801F0C1F90028EFD1EAE74F
:106C000003F09AFB0A9B01930360ECE76800002005
:106C100018CC0000F0B54E464546DE465746E0B576
:106C2000E14B4C008FB09046894664089C4200DCE2
:106C300087E0DE4B9C4222DCDD4A002900DC92E04A
:106C4000DC4B02F017FFDB4B06000F009C4200D12B
:106C50007EE1D94AD94B02F00DFF02000B004146FC
:106C600030000A604B60390002F004FFD34BD24A77
:106C700002F000FF434601259860D9606BE0D04BDD
:106C80009C4200DC8FE0CF4B9C4200DD55E1CE4AB8
:106C9000231592469A4451460905631A19001D00AE
:106CA000040003F04BFA03F07FFA02000B0020000F
:106CB00029000892099302F0DDFE0022C34B02F086
:106CC00067FC0F00060003F039FA03F06DFA0400C8
:106CD0000D0002000B00300039000A940B9502F001
:106CE000C9FE0022B94B02F053FC002200230C9095
:106CF0000D9101F053FB002800D192E10023002206
:106D00002000290001F04AFB434243410133B04ACD
:106D100041460192022208A80092524600F07CFBF4
:106D20004B460500002B16DA802243461206944695
:106D300042465B68454263445360D3686344D36012
:106D400009E00B00020041460A604B60002200236C
:106D500000258A60CB6028000FB03CBC9046994665
:106D6000A246AB46F0BD934B01F0ECFC914B060004
:106D70000F009C4200D13DE18F4A904B01F0E2FCB4
:106D800002000B00414630000A604B60390002F0FF
:106D900071FE894A894B01F0D5FC012543466D42BD
:106DA0009860D960D7E701F049F88A4A8A4B060013
:106DB0000F0002F0EDFB0022884B01F0C3FC03F052
:106DC000BDF9050003F0F0F9794A7A4B049005917A
:106DD00002F0DEFB02000B003000390002F04AFE38
:106DE000754A06000F0004980599744B02F0D0FB19
:106DF000029003911F2D00DCC7E0029A039B300034
:106E0000390002F037FE83468A4653465B0024155C
:106E10005B0DE31A102B6CDD04980599D322674BA8
:106E2000520502F0B5FB02000B003000390002925F
:106E3000039302F01FFE0A0001001300069107925F
:106E400002003900300002F015FE029A039B02F0A6
:106E500011FE06000F0004980599614A614B02F08B
:106E600097FB32003B0002F005FE069E079F0B00D9
:106E70000200390030000292039302F0FBFD4B0048
:106E80005B0D83468A46E41A312C32DD049805995D
:106E9000B822544B920502F07BFB03000C00020069
:106EA000029303940B000698079902F0E3FD020099
:106EB0000B0006000F000698079902F0DBFD029A0E
:106EC000039B02F0D7FD484A02900391049805996C
:106ED000464B02F05DFB029A039B02F0CBFD0200E1
:106EE0000B00300039000292039302F0C3FD834689
:106EF0008A465A465346414630000A604B60390084
:106F000002F0B8FD029A039B02F0B4FD44460B0068
:106F10000200A260E3604B46002B00DB1BE75B46F0
:106F2000236080231B065344636080231B069C461A
:106F30006144A060E1606D420DE70B00020002F0C9
:106F400099FD434600259860D9601860596002E7B2
:106F5000D3221A4B520502F08DFD214A214B0D0020
:106F6000040002F087FD02000B00414620000A6089
:106F70004B60290002F07EFD1A4B194A02F07AFD9F
:106F8000434601259860D960E5E602000B00300019
:106F9000390002F06FFD6B1E154A9B009B5883461B
:106FA0008A46A342A5D130E7FB21E93F7BD90240C5
:106FB00000004054FB21F93F3163621A61B4D03DB7
:106FC000FB213941FFFFEF7FEAFBFFFF000070412B
:106FD000A0CC000083C8C96D305FE43F0000E03FF3
:106FE0007370032E8A19A33BC14920259A837B39EC
:106FF00020CC0000D3220C4B520501F0A3FB0B4A1E
:107000000B4B04000D0001F09DFB02000B004146FC
:1070100020000A604B60290002F02CFD034A044B5B
:10702000B9E6032373E6C04661B4D03D7370032E06
:107030008A19A33BF8B54746CE46674B80B50A0090
:107040000F00190005003940994200D19BE004006F
:107050000100002F69DD3F1500D1B4E05F4B120342
:107060009C468023120B5B0313435B00CA0F6744EB
:107070009B184A00F80703D5D20F5B009B188A00C3
:1070800079108C46002180201624894680030D1833
:107090009D4202DC29185B1B8144D50F5B00013C3B
:1070A0005B1952004008002CF1D10020804680205E
:1070B00020250027000609E08B425CD0D40F5B003E
:1070C000013DE31852004008002D16D0C4198B4230
:1070D000F2DD27180E00002C49DB5B1AA242894121
:1070E00049425B1A121BD40F5B00013D8044310002
:1070F000E31852004008002DE8D113434ED1434617
:107100005B0837494A468846494652104244C907F7
:1071100002D5802109060B4361460F05BD181800F2
:1071200029000CBC90469946F8BD7B005B080343E0
:107130003900002BF5D0002F3CD1E30A153A640545
:10714000002BFAD08020400303423FD1002700E00B
:107150000F005B00791C0342FAD0250020208D40EF
:10716000401A2900D71B2200C2401A4376E7FE438B
:10717000F60F8E19B1E79442A0D82718002CF6DB41
:107180001E000023AEE702003B002800390002F099
:10719000FFF92A003B0001F0D5FAC2E7434601336C
:1071A00003D0434601335B08ABE701239846002335
:1071B000C144A6E73B00020002F05CFC02000B00A9
:1071C00001F0DCFDADE713000022BBE70127210041
:1071D00020207F42C6E7C0460000F07F01FCFFFF91
:1071E0000000E03FF0B54746CE4680B587B000923C
:1071F0000193754B4F00814688467F089F4263DCB0
:1072000002F09CFF002800D1D4E04A46434648469D
:10721000414602F0BDF904000D006C4A6C4B02F0CF
:10722000B7F96C4A6C4B01F08DFA22002B0002F08A
:10723000AFF96A4A6A4B02F01DFC22002B0002F0F3
:10724000A7F9684A684B01F07DFA22002B0002F092
:107250009FF9664A664B02F00DFC22002B0002F0FB
:1072600097F9644A644B01F06DFA22002B0002F09A
:107270008FF9029003910022604B2000290002F058
:1072800087F9029A039B06000F002000290002F0F4
:107290007FF9009A019B04000D004846414602F028
:1072A00077F902000B002000290002F0E3FB020046
:1072B0000B003000390002F0DDFB02000B00002063
:1072C0004F4902F0D7FB70E002000B0002F060F9BA
:1072D00004000D003D4A3E4B02F05AF93D4A3E4B38
:1072E00001F030FA22002B0002F052F93B4A3C4BED
:1072F00002F0C0FB22002B0002F04AF9394A3A4B57
:1073000001F020FA22002B0002F042F9374A384BF4
:1073100002F0B0FB22002B0002F03AF9354A364B5E
:1073200001F010FA2B00220002F032F9354B0290E6
:1073300003919F429FDD344B00229F423DDC334945
:1073400000207B182E4916001F0002F093FB0490CA
:1073500005910022294B2000290002F019F9320082
:107360003B0002F087FB029A039B06000F002000FF
:10737000290002F00DF9009A019B04000D00484617
:10738000414602F005F902000B002000290002F03E
:1073900071FB02000B003000390002F06BFB0200B1
:1073A0000B000498059902F065FB07B00CBC9046F1
:1073B0009946F0BD00201249F7E7154B00260492CC
:1073C0000593144FC5E7C046FFFF3F3ED43888BE43
:1073D000E9FAA8BDC4B1B4BD9EEE213EAD529C8079
:1073E0004F7E923E9015CB19A001FA3E7751C116FF
:1073F0006CC1563F4C5555555555A53F0000E03FD3
:107400000000F03F3233D33F0000E93F0000E0FFCF
:107410000000E73F0000D23FF0B5DE464E4645464D
:107420005746E0B5DC4CA5440D9114001900A49A10
:107430000993DA4B9200D6584D1E03901821E01E96
:107440000696029500F0A0FEC3430100DB17194029
:107450004B1C9A009B1ADB001B190B9105934C1BCC
:10746000771918D4A59BA5009C463F1922AE654408
:10747000013707E0286802F097FE013403C604359F
:10748000BC4208D0002CF5DA00200021013403C6EC
:107490000435BC42F6D1069B002B01DA00F0FDFB5F
:1074A000069B03990133DB009A46099BDA00944658
:1074B00000920022914672AA0492B94A614493460E
:1074C00088469AAB63449B44029B002B00DABCE1E4
:1074D0005D4600260027039C4D442A686B6803CC58
:1074E00002F056F802000B003000390001F02AF9D2
:1074F000083D06000F004445EFD1049B4B441E603D
:107500005F6008239C46E144D145DDD10EA80421EB
:107510008446494261448C46069A93009C446146E5
:1075200084460A910399083B63448C460C93009B64
:10753000009263449B46009A0498D10003008C4655
:10754000634408911E685F68002A33DD95498046D0
:107550008C466244D300984470AB9A460EAB994671
:107560000022914B3000390002F012F802F0E6FDE3
:1075700002F01AFE00228D4B04000D0002F008F804
:1075800002000B003000390002F074FA02F0D6FD60
:107590004B4601C39946434620001A685B682900A0
:1075A00001F0D0F808235B429C46E04406000F003F
:1075B000D045D5D1059B30001A003900984600F01F
:1075C000DFFCFF2300229B0504000D0001F0E0FF1B
:1075D00000F038FC0022764B01F0DAFF02000B00CD
:1075E0002000290002F046FA0D00040002F0A6FD7A
:1075F000814602F0D9FD02000B002000290002F0B4
:1076000039FA060040460F00002800DCEEE0009B3F
:1076100018215A1E92000EAB9B58091A1D000D41ED
:10762000A9448D405D1B0EAB9D5017231B1A1D41B5
:10763000002D2DDD01239C46009BE144002B00DC46
:107640001CE20E9C0123002C00D0B5E0009A012A18
:1076500009D099000EAA54580133002C00D0ACE098
:10766000009A9A42F5D1059B002B0EDD012B00D12B
:10767000A8E1022B09D1009B0EA95A1E92000EAB65
:107680009B5807939B029B0A8B50022D00D1C1E0AF
:10769000002300223000390000F080FE009B00280B
:1076A00000D194E2069A591E8A4210DC414A0A9897
:1076B00094460EAA6344944600229B0063441C68CF
:1076C000043B22438342FAD1002A00D0C0E0069B4B
:1076D0000EAA013B9B00D358002B00D0B3E001223F
:1076E0000C9B043B596801320029FAD0009B9C4650
:1076F0006244110007921A0001338B4246DC0B985A
:1077000063468046A59C4344A046099C9B00A14635
:107710004A449844D30022AA9146049A9944944634
:10772000089BA59A63448446614494469A468B001C
:10773000634400934346586802F036FD4B46186098
:107740005960029B002B24DB4D46039C002600273A
:1077500001E0286869680CCC01F01AFF02000B00F8
:107760003000390000F0EEFF083D06000F005C45D8
:10777000EFD153469E60DF6004239C460433E0440F
:107780009C46009BE144E2449845D3D1079B00937B
:10779000D1E600260027ECE794FDFFFFE8CD0000CE
:1077A00018FEFFFFFFFFFF1F0000703E000070414A
:1077B00000002040FFFFFF3F002180225204141BE5
:1077C0000EAA5450009999420EDD0EA884469B00E3
:1077D0000EAA8900D25861446344CF4800E01A6879
:1077E000821A04C38B42FAD101243CE7059B002B8B
:1077F00006D1009B0EAA013B9B00D558ED1517E75B
:107800000022C64B300000F0EDFD002800D024E13E
:1078100000253DE732003B000020C14902F02AF973
:1078200006000F00002C00D132E7059A0020BC4969
:1078300000F0A6FB02000B003000390002F01AF93C
:1078400006000F0024E7012250E70026002754E637
:107850004B46059A079388468B000EA9CB58183AD9
:1078600008950592002B0DD18C464146AD4B434403
:107870009B006344043B58680139183A0028F9D04A
:1078800088460592059A0020A54900F079FB4346F9
:1078900004000D00002B00DA05E29E000EAB9C46B2
:1078A0004346DB0066449C46059370AB9946049FB3
:1078B00067440097306802F077FC22002B0001F04B
:1078C00067FE002238607960974B2000290001F0A4
:1078D0005FFE083F04000D00043EB945EAD14AAB03
:1078E00003939B4600239A46069B4246994643468D
:1078F0000132029204934B46002B00DAAAE080206A
:107900008A4B009D9846C00589490026002700241F
:1079100008E008239C460835E044544511DC434602
:10792000186859682A686B6801F032FE02000B0083
:107930003000390000F006FF013406000F00A145B9
:10794000E7DA5B46C0C39B4601239C46009BE244AA
:10795000083B0093029B9A45CDD1049B9846A49B7B
:10796000022B00DD8EE0002B37DC1FD1059B0027AA
:107970001D00039B00249C461E006544083E2A68A7
:107980006B683800210000F0DDFE083D07000C00A8
:10799000AE42F4D1089B002B03D080231B069C46EB
:1079A00064443A0023000D990A604B600720079B4E
:1079B00018409B239B009D443CBC90469946A246A0
:1079C000AB46F0BD009B0EA95A1E92000EAB9B5811
:1079D00007935B025B0A8B5057E64346002B00DAA5
:1079E00070E100200021DB004AAAD61848AF3268B7
:1079F0007368083E00F0A6FEB742F8D1089B002B42
:107A000000D025E10B0002004A984B990D9C2260A2
:107A1000636002F02FF8434607000C00002B13DDD3
:107A200001254CAEB14638002E0021004C460136EF
:107A30000CCC00F087FEA146B045F7DA089B0700A2
:107A40000C00002B00D015E13A0023000D998A604C
:107A5000CB60ABE70026002773E701239C46009B21
:107A6000E1440225002B00DDEBE532003B00002065
:107A70002B4901F0FFFF06000F0009E60024F2E5A4
:107A80004AAB0393A49B032B00D08FE74346002B04
:107A900000DC14E1039ADB009B46130091465B4433
:107AA0001E685F68234B43440293DB00994448AB54
:107AB0009A464B465C681B681800210032003B0068
:107AC0000090019100F03EFE04000D0002000B004A
:107AD0000098019901F0CEFF3B00320000F032FE29
:107AE0004B469860D9601C605D6008235B429C46F1
:107AF000E14426002F00CA45DBD14346012B00DCC0
:107B0000E3E0039A13005B441E685F68029BDB009E
:107B100099464A44904610E0FFFFFF000000E03F16
:107B20000000F03FFFFFFF3F0000703EA8CD0000C7
:107B3000FB21F93FFFFFFF1F984643465C681B6827
:107B40001800210032003B000090019100F0FAFD86
:107B500004000D0002000B000098019901F08AFF5B
:107B600032003B0000F0EEFD4346039A9860D96076
:107B70001C605D60083B26002F009A42DCD14D4618
:107B80009446002600244746083565442A686B68F9
:107B90003000210000F0D6FD083D06000C00AF4289
:107BA000F4D1039B4A9F5D689968D868089B002BB5
:107BB00065D08022120694460D9B6544604464445F
:107BC0001F605D609960D8601E615C61EEE69A4658
:107BD0004B460793059B30005A423900089500F048
:107BE000CFF900223A4B06000F0000F0FBFB002803
:107BF00024D0384B00223000390001F0C9FC02F0DB
:107C00009DFA52460400950002F0CEFA0022304B55
:107C100001F0BEFC02000B003000390001F02AFF29
:107C200002F08CFA0EAA50510122059B52441833DF
:107C30009046059393000EAAD45023E65346300095
:107C400039009C0002F07AFA0EAB1851D04619E6C2
:107C500080230D9A1B06CB18106053600B000200A6
:107C60004A984B9901F006FF434607000C00002B91
:107C700000DDD5E680231B069C466444E4E62B0029
:107C80003A000D9D2A606B600A000300AA60EB6059
:107C9000320023002A616B6188E6099BDB000093B8
:107CA00072AB049332E4A49B022B00DDE8E6002BC8
:107CB00000DD92E600D079E6002700246AE600267F
:107CC00000246EE70020002198E60026340068E7D3
:107CD000000070410000703EF0B5CE46474680B5CA
:107CE00087B000920193474A4B00814688465B0863
:107CF000934207DC4146484602F020FA4146031E03
:107D0000484666D04A4643464846414601F040FC54
:107D100004000D0002000B004846414601F038FC0B
:107D2000394A3A4B06000F002000290001F030FCD0
:107D3000374A384B01F09EFE22002B0001F028FC50
:107D4000354A364B00F0FEFC22002B0001F020FCEF
:107D5000334A344B01F08EFE22002B0001F018FC58
:107D6000314B324A00F0EEFC0E9B02900391002B47
:107D700034D00098019900222D4B01F009FC029AA1
:107D8000039B049005913000390001F001FC0200D2
:107D90000B000498059901F06DFE22002B0001F004
:107DA000F7FB009A019B01F065FE224A04000D00DA
:107DB000214B3000390001F0EBFB02000B002000EA
:107DC000290000F0BFFC02000B004846414601F0CC
:107DD00051FE07B00CBC90469946F0BD02000B0066
:107DE0002000290001F0D4FB124A134B01F042FE9F
:107DF00032003B0001F0CCFB4A46434600F0A2FCB7
:107E0000E7E7C046FFFF3F3E7CD5CF5A3AD9E53D74
:107E1000EB9C2B8AE6E55A3E7DFEB157E31DC73E3B
:107E2000D561C119A0012A3F1111813FA6F8101197
:107E30000000E03F495555555555C53F49004B0891
:107E400019007047474AF0B54F4691464B005B0D0D
:107E500099444646D6464A46C0B505000C000E0079
:107E600088460700132A27DC002A4BDB3E4B1341D0
:107E70009A460B0052461340034318D03B4A3C4BF2
:107E80002800210000F05EFC0022002300F0A0FA90
:107E9000002847D0002C04DA80234A465B031341B4
:107EA00098444646534600279E43380031001CBC88
:107EB00090469946A246F0BD332A08DD8023DB00B8
:107EC0009945F4D102000B0000F03CFCEFE7294A91
:107ED0009446012263445242DA4092460242E6D07E
:107EE000224A234B2800210000F02CFC0022002312
:107EF00000F06EFA002815D0002C1EDB53464646D3
:107F00009F430FE0194A1A4B2800210000F01AFC89
:107F10000022002300F05CFA002803D0002C04DBD0
:107F20000027002638003100C1E7640064082543BB
:107F30000027002DF6D0104EF4E74B46142B0BD043
:107F40003422D21A012393405D19BD4208D2012385
:107F50009C462F00E044D1E7133B9C46E044CDE72C
:107F60002F00CBE701FCFFFFFFFF0F009C7500888F
:107F70003CE4377EEDFBFFFF0000F0BF00207047C0
:107F80004B0070B55B0D14000A00002B1AD14B009A
:107F90005B08034315D0234B002201F0F9FA224B72
:107FA0009C422DDB0A004B005B0D363B1F4DE31856
:107FB000AB422ADC002B0DDD1D4C1B0522401A4371
:107FC000110070BD1B4DAB42F0D102000B0000F060
:107FD000B9FBF6E71D00353519DA174B02009C4254
:107FE00009DD0B001548164900F032F8134A144B0E
:107FF00001F0CEFAE5E70B001248134900F028F82B
:10800000104A114B01F0C4FADBE70200E9E7084C23
:10801000363322401B051343190000220B4B01F09D
:10802000B7FACEE700005043B03CFFFFFE07000068
:10803000FFFF0F80FF07000050C300009C75008801
:108040003CE4377E59F3F8C21F6EA5010000903C56
:1080500030B54A00DB0FDB0752081A43110030BD70
:1080600002B4714649084900095C49008E4402BCCB
:108070007047C046002243088B4274D303098B42E9
:108080005FD3030A8B4244D3030B8B4228D3030CE8
:108090008B420DD3FF22090212BA030C8B4202D38A
:1080A0001212090265D0030B8B4219D300E0090AB2
:1080B000C30B8B4201D3CB03C01A5241830B8B42BB
:1080C00001D38B03C01A5241430B8B4201D34B03A4
:1080D000C01A5241030B8B4201D30B03C01A524109
:1080E000C30A8B4201D3CB02C01A5241830A8B428E
:1080F00001D38B02C01A5241430A8B4201D34B0277
:10810000C01A5241030A8B4201D30B02C01A5241DA
:10811000CDD2C3098B4201D3CB01C01A524183098E
:108120008B4201D38B01C01A524143098B4201D3C8
:108130004B01C01A524103098B4201D30B01C01AF3
:108140005241C3088B4201D3CB00C01A524183086D
:108150008B4201D38B00C01A524143088B4201D39A
:108160004B00C01A5241411A00D2014652411046FA
:108170007047FFE701B5002000F0F0F802BDC046EF
:108180000029F7D076E7704703460B437FD40022DF
:1081900043088B4274D303098B425FD3030A8B429B
:1081A00044D3030B8B4228D3030C8B420DD3FF2205
:1081B000090212BA030C8B4202D31212090265D0D3
:1081C000030B8B4219D300E0090AC30B8B4201D386
:1081D000CB03C01A5241830B8B4201D38B03C01ACD
:1081E0005241430B8B4201D34B03C01A5241030B44
:1081F0008B4201D30B03C01A5241C30A8B4201D3F5
:10820000CB02C01A5241830A8B4201D38B02C01A9F
:108210005241430A8B4201D34B02C01A5241030A16
:108220008B4201D30B02C01A5241CDD2C3098B42FB
:1082300001D3CB01C01A524183098B4201D38B0178
:10824000C01A524143098B4201D34B01C01A52411B
:1082500003098B4201D30B01C01A5241C3088B4260
:1082600001D3CB00C01A524183088B4201D38B004B
:10827000C01A524143088B4201D34B00C01A5241ED
:10828000411A00D201465241104670475DE0CA0FC4
:1082900000D04942031000D34042534000229C4684
:1082A00003098B422DD3030A8B4212D3FC2289018E
:1082B00012BA030A8B420CD3890192118B4208D364
:1082C000890192118B4204D389013AD0921100E0C6
:1082D0008909C3098B4201D3CB01C01A52418309DA
:1082E0008B4201D38B01C01A524143098B4201D307
:1082F0004B01C01A524103098B4201D30B01C01A32
:108300005241C3088B4201D3CB00C01A52418308AB
:108310008B4201D38B00C01A5241D9D243088B4201
:1083200001D34B00C01A5241411A00D201466346A4
:1083300052415B10104601D34042002B00D5494208
:10834000704763465B1000D3404201B5002000F047
:1083500005F802BD0029F8D016E770477047C046FF
:10836000D0400B1C1141203A03D49C4613411843C2
:1083700063465242934018437047C0468446101CDF
:1083800062468C46191C634600E0C0461FB501F0EA
:1083900097F8002801D40021C8421FBD10B500F095
:1083A000EFFF4042013010BD10B501F089F8002800
:1083B00001DB002010BD012010BDC04610B501F04A
:1083C0007FF8002801DD002010BD012010BDC0464F
:1083D00010B501F011F8002801DC002010BD0120CB
:1083E00010BDC04610B501F007F8002801DA0020E2
:1083F00010BD012010BDC046F0B5CE46474615045D
:108400002D0C2E0080B50704140C3F0C9946030C6C
:108410007E435D43674363437F19340CE4199C46F4
:10842000A54203D980235B029846C4444B4643438C
:108430005143250C36046544360C2404A4195B19F9
:10844000591820000CBC90469946F0BDF0B54E4638
:1084500057464546DE46E0B543025B0A450083B019
:108460000F1C99462D0EC60F002D57D0FF2D24D07E
:108470008020DB00C0041843002381469A469B46B7
:108480007F3D7C027A00FB0F640A120E984623D0CF
:10849000FF2A4BD0E30080240020E4047F3A1C43F1
:1084A000AD186B1C47460193534677403A000F2B9B
:1084B00048D87D499B00CB589F46002B00D085E0D3
:1084C00008339A46063B9B467C027A00FB0FFF2549
:1084D000640A120E9846DBD1002C00D090E0524680
:1084E00001231A4392460120DBE74C465846170009
:1084F000022824D0032800D1CFE000220023012845
:108500004DD15802D205400AFF071043384303B04B
:108510003CBC90469946A246AB46F0BD002B5BD1D1
:1085200004239A46033B00259B46AAE7FF35002C0F
:1085300060D1524602231A4392460220B1E7FF223D
:108540000023DEE74B461B0C9C464B462604360CAC
:10855000180461463300220C6446000C43434E432A
:108560005043544380191A0C1218964203D98021A3
:1085700049028C4664441B041B0C1004C018830180
:108580005E1EB341800E1843130C1B199B0103435D
:108590001C00230179D5012362081C401443019A71
:1085A0007F32002A4DDD630704D00F232340042BC4
:1085B00000D00434230103D53C4B019A1C40803287
:1085C000FE2ABCDCA3015B0AD2B29AE70C239A46CE
:1085D000093BFF259B4654E7180001F071FE4A460F
:1085E000431F76259A4000236D4291462D1A9A46E4
:1085F0009B4646E7524603231A439246032050E720
:10860000200001F05DFE431F2D1A9C40763D0020A6
:1086100047E780230027DB03FF2272E7424666E735
:108620004C463200584662E780234A46DB031A4232
:1086300022D01C4220D123435B025B0A4746FF2223
:108640005FE701239A1A1B2A21DC23000199D340FA
:108650009E318C401A0023005C1EA34113435A072D
:1086600004D00F221A40042A00D004335A0111D436
:108670009B015B0A002244E780234A46DB03134345
:108680005B025B0A3700FF223BE7019587E7002288
:10869000002336E70122002333E78023DB03234353
:1086A0005B025B0AFF222CE7F8CD0000FFFFFFF71B
:1086B00070B500283DD0C317C5185D40C40F280011
:1086C00001F0FEFD9E22121A962A07DCD2B208287B
:1086D00033DD083885406802400A23E0992A0BDD23
:1086E000052329001B1AD94003001B339D402B0092
:1086F0005D1EAB4119430D00052801DD431F9D4060
:108700002B000F490B406E0709D00F263540042D72
:1087100005D004335D0102D59F220B40121A9B0144
:10872000580AD2B24002D205400AE407104320435F
:1087300070BD002400220020F4E76802400AF1E73F
:10874000FFFFFFFBF0B54F464646D6460C00090337
:10875000C0B5490A470F5E0039431F03DB0F9C4633
:1087600065007B0A570F1F436D0DE40F760DA14680
:10877000C000B846D200AB1B64457BD0002B5FDD48
:10878000002E00D0A4E03E00164300D112E15E1E90
:10879000002E00D09EE1871A4346B8428041012551
:1087A000C91A4042091A0B0200D431E149024E0AAB
:1087B000002E00D16EE1300001F082FD0300083B85
:1087C0001F2B00DD61E120223900D21A9E40D140EA
:1087D0009F400E439D4200DD51E15D1B6B1C1F2B32
:1087E00000DD7CE12021C91A3D0030008F40884027
:1087F000DD40791E8F41310007222843D9400025F2
:1088000007433A40002A09D00F233B40042B05D0F0
:108810003B1DBB42BF417F42C9191F000B0200D460
:1088200026E26A1CC64B55056D0D9A4200D106E141
:10883000C44AFF080A40530752023B43120B8EE022
:10884000002B00D0B8E06B1C5B055B0D012B00DC3E
:1088500030E1871A4346B842B641CB1A76429E1B96
:10886000330200D54CE13B003343A1D10022002468
:10887000002570E0002B00DCE5E0002E00D183E055
:10888000AF4EB54260D0802636043743B846382B09
:1088900000DC3EE1434613431F007A1E97413F1818
:1088A00087428041404209180B0200D4B0E0A44B3B
:1088B00001359D4200D1C3E0A24A7B080A40012154
:1088C0000F401F435108D30707221F433A4099E73F
:1088D0009B4EB54238D0802636043743B846382BF5
:1088E00000DDDCE01F2B00DC30E11E004746203EAF
:1088F000F740BC46202B04D04026F31A46469E4043
:108900003243170063467A1E97411F43CCE0002B89
:1089100000D104E24346134300D159E14B07C0089C
:1089200018438023C9081B03194208D04546ED08A7
:108930001D4204D14346D008590708432900420F7D
:10894000C9007F4D1143C0004B07CA087C49C008CD
:1089500003438D4268D012036D05120B6D0D00218B
:1089600012031800130B0A0D12051A43764B2D053E
:1089700013402B435B00E4075B08234319001CBC36
:1089800090469946A246F0BD3E00164312D05E1EA8
:10899000002E00D000E187188742804141444042C8
:1089A000091801250B0233D5022585E764463300FB
:1089B000414610001D00C7E7002D00D0DAE00C0092
:1089C0000443F3D05C1C00D19FE15D4CA64200D172
:1089D0002FE1DB43382B00DD66E11F2B00DD83E157
:1089E00020240500E41A0F00DD40D940A040434692
:1089F000A7405B1A441EA04198462F433843171ADC
:108A0000BA42924143465242991A64463500CAE638
:108A100007223A40002A00D0F6E64B07CA08484928
:108A2000FF083B438D4296D11900114300D19EE1CE
:108A3000802109030A431203120B414D8FE71500F1
:108A4000002200238BE7002B00D0C7E06B1C5F05E2
:108A50007F0D012F00DCF1E0394DAB4200D1B9E0D0
:108A600085180A008542894142444942511807222B
:108A7000CF076D082F4349083A401D00C2E6072280
:108A80003049ED1A31403A40BCE63E002838864075
:108A900000279FE6380001F013FC20308EE64346A5
:108AA00013431F007A1E9741C71BB84280414042C2
:108AB000091A78E60E003B0006431343002D61D1EE
:108AC000002E00D0F4E0002B00D11BE164463900F9
:108AD000100039E71A4FBB427AD03300FFE630006E
:108AE0001F3DE840202B03D04021CB1A9E40374346
:108AF0007B1E9F41072207433A400021002589E75A
:108B0000171A4346BA42B641591A76428E1B64463A
:108B10004EE61F2B00DDADE020264746F61AB74093
:108B2000B9461700B246DF404E463E433700564630
:108B3000B240561EB24117434246DA408918AEE6AB
:108B4000FF070000FFFF7FFFFFFF0F802026474643
:108B5000F61AB740B9461700B246DF404E463E43CC
:108B600037005646B240561EB24117434246DA40DD
:108B7000891A99E77F4CA6425BD0802424045B428B
:108B8000214327E7002E0CD1002B00D1CBE0644617
:108B900039001000774DD7E6764FBB4218D033002E
:108BA00075E6002B14D04B07C00818438023C90872
:108BB0001B03194207D0FC081C4204D17907D008D6
:108BC0000843E14621004C46420FC9001143C00052
:108BD000684DB9E61D0000220023C0E6002D5BD1E0
:108BE0000D00054300D1E2E65D1C00D1B0E0614D0F
:108BF000AE421FD0DB43382B71DC1F2B00DD96E02B
:108C000020250F00ED1AAF40B9460700AA46DF4005
:108C10004D463D432F005546A840D940451EA8412A
:108C200088440743BF18974292415142414435005E
:108C30003AE6644635004146100085E60B000343E2
:108C4000002D00D063E6002BF5D04346134300D13E
:108C50007AE687188742804107224144404209183A
:108C60003A400B0200D4D5E6434B01351940C9E523
:108C7000380069E61E004746203EF740BC46202BE0
:108C800004D04026F31A46469E40324317006346FE
:108C90007A1E97411F4302E6364DAE42CAD0802568
:108CA0002D045B422943A6E70843411E8841A6E6FE
:108CB000002B00D148E6871A4346B842B641CB1A8A
:108CC00076429E1B33024BD5171A4346BA42924155
:108CD000591A5242891A072264463A4092E50143E2
:108CE0000F00791E8F419DE71C000F00203CE740DC
:108CF000202B03D04024E31A99400843411E8841A9
:108D000038437CE60022002425E6171A4346BA427F
:108D10009241591A5242891A6446350043E5414648
:108D20001000144D10E680220024120380E61D007E
:108D30000F00203DEF40BC46202B03D04025EB1A0E
:108D40009940084307006346781E87411F4369E73F
:108D5000871897429B4141445B42C9183500A3E5FF
:108D60003B003343CED0072231003A4052E6002385
:108D70001A00F4E5FF070000FFFF7FFFF0B557463C
:108D8000DE464E464546E0B5834607000E034800E2
:108D900085B092461C00360B400DCD0F002800D147
:108DA0009DE0954B984239D08023F6001B041E436A
:108DB000924A7B0F334399469446030063440093E1
:108DC00000230026FF00029323031B0B9846630039
:108DD000E40F52465B0D019400D1B3E086498B420B
:108DE00000D19EE04246D100802212040A4351463F
:108DF000490F11438B46814952468C460099634482
:108E0000CB1A0021D20000932B0063409A460F2E0C
:108E100000D905E17A4BB6009B599F465B46334328
:108E2000994600D0B8E0022308260027009002935C
:108E3000CAE7CB463A0002990195019B9A4602295E
:108E400027D0032900D180E2012944D06D49009B3D
:108E50008C4663441C00002C38DD530700D013E21D
:108E6000D2085B46DB0109D55946674B19408B4652
:108E70008021C9008C46009B63441C00634B9C42CC
:108E800007DC5B4664055F075B0217431B0B620D43
:108E900002E000230027584A00211B031C0B0B0D86
:108EA0001B05234314055A4A380013401C435346FC
:108EB0006400DB0764081C43210005B03CBC9046FD
:108EC0009946A246AB46F0BD0122524201231B1B2C
:108ED000382B00DCADE1002200230027DCE75B46F5
:108EE000334399465ED0002E00D18AE1300001F074
:108EF000E7F903000B3B1C2B00DD7BE11D22D31A9D
:108F00005A460100DA4008398E4013005F46334369
:108F100099468F403F4B00261B1A00930023029373
:108F200052E7414653460B433B499B468C46009BC8
:108F3000634400935B46002B3BD1022300221E4377
:108F4000022161E7434613439B4637D04346002B3B
:108F500000D162E1404601F0B3F903000B3B1C2B4A
:108F600000DD53E102004146083A914088461D2148
:108F7000CB1A5146D9400B0041460B439B46534602
:108F800093401A00009B25499C46604403008C4690
:108F900063440093002137E70323B14600900C2679
:108FA000029311E700230093013304260027029364
:108FB0000AE70323C3461E43032125E701331E436B
:108FC0000022012120E700239A46802300271B036B
:108FD000094A61E7802349461B03194200D1E2E0B8
:108FE0005946194200D0DEE00B431B0317001B0B50
:108FF000A246014A50E7C046FF07000001FCFFFF00
:1090000038CE0000FF030000FFFFFFFEFE07000058
:10901000FFFF0F800DFCFFFF01F8FFFFF3030000CF
:10902000D94500D9CBE000D1C6E03C004846002736
:10903000009B013B00935B46160E1B021E4313026E
:10904000984633041B0C9946310C0191FFF798F8B0
:109050004A4642430B04210C050019438A4207D9B2
:109060008919013D8E4203D88A4201D9851E89198A
:10907000881A0199FFF784F809048C464A462104AE
:1090800064464243090C030021438A4204D98919EA
:10909000013B8E4200D8F1E02D041D43AB46434610
:1090A000891A4246280C12041D0C5B46140C22003F
:1090B0001B041B0C5A4303946B43444302956843BF
:1090C0001B19150CEB189C4203D980246402A4469A
:1090D00060441C0C15041B042D0C20185D198142E2
:1090E00077D373D00C1AA24A7D1BAF42BF4194467E
:1090F000009B7F426344E01B1C00864200D1DBE002
:109100000199FFF73DF84A4642430B04290C07003A
:1091100019438A4207D98919013F8E4203D88A42EE
:1091200001D9871E8919881A0199FFF729F80904BE
:109130004A46894629044D464243090C0300294307
:109140008A4207D98919013B8E4203D88A4201D944
:10915000831E89193F04891A3A00039F1A43380075
:1091600013041B0C584381460298150C6F4343436C
:1091700045434846000C8446DB1963449F4203D9AB
:10918000802040028446654448461F0C00041B04AE
:10919000000C7D191818A94200D284E000D17FE0AC
:1091A00001231A4357E680234A461B0313431B033C
:1091B0001B0BAA466F4A6FE6BA4200D935E74B4609
:1091C000DC0758087B081C43FF0734E70024AF4244
:1091D00089D247444745A4415B466442A4196418B8
:1091E000013BA6421ED2A0426DD800D1B6E0241A9F
:1091F0009B4678E703005A46283B9A400027914651
:1092000088E6584601F05CF8203072E603005246CA
:10921000283B9A4093460022B4E6504601F050F8AD
:1092200020309AE6A642E2D1B845DCD9341A9B46F2
:1092300059E71F2B65DC504C0099A4465C466144FD
:1092400008008C4011008240D940501E82410C43DE
:1092500014435A46DA401300620709D00F22224015
:10926000042A05D02200141D9442894149425B180A
:109270001A0262D50122002300270DE68A4200D897
:109280000AE7831E891907E70F231340042B00D137
:10929000E6E5171D9742924153429B44FA08E0E5E8
:1092A000002800D1D7E57118531EB14227D3A94237
:1092B00015D358D01A0073E7002B00DC04E6012315
:1092C00000229B44CDE502234744474589415B4248
:1092D0009C46494289190C19E344241A03E7434682
:1092E0005F0047459B41B8465B429E19023A891987
:1092F000A94200D054E7404500D051E7ABE51A0041
:10930000F6E71F215F4649420C1BE740202B07D0A0
:109310001A49009B8C46634418005B4683401A43FD
:10932000501E82413A4307270023174009D00F21DE
:10933000002311401400042995D122005F075B022D
:109340001B0BD20817430022A6E5802359461B03B6
:109350000B431B0317001B0B064A9DE5BD42B2D809
:109360009B460024BFE68045B9D31A00C3E7C04638
:10937000FF030000FF0700001E0400003E04000081
:10938000F0B54F464646D6468446C0B58046194E8F
:1093900018030F034D00000B5C0082463F0B6D0D60
:1093A000C90F9146640DDB0F0120B5420AD0B442CB
:1093B00003D0A54201D157450CD01CBC904699461C
:1093C000A246F0BD66463E43F7D1AC42F5D15446C5
:1093D0001443F2D10120C845EFD1994207D0002DA6
:1093E000EBD163461F433800471EB841E5E7002034
:1093F000E3E7C046FF070000F0B54F464646D646B5
:109400004D00C0B50E03C90F8A462C491F035C00EE
:109410008046360B6D0D91463F0B640DDB0F8D4280
:109420001ED08C4216D0002D1ED130438446002C15
:1094300001D13A4323D06246002A1AD09A4529D056
:10944000514602200139084001381CBC904699461B
:10945000A246F0BD39001143E5D002204042F4E7B6
:109460003043FAD1AC420FD0002C0FD13A43E7D0B1
:109470000CE00122013B934318000130E5E763460D
:109480000020002BE1D0DBE73A43E6D19A45D7D163
:10949000A542D5DCA54205DBBE42D1D808D00020CC
:1094A000BE42D2D250460123013898430130CCE766
:1094B000C845C5D80020C845F4D3C6E7FF0700005B
:1094C000F0B54F464646D6464D00C0B50E03C90F0F
:1094D0008A462E491F035C008046360B6D0D91466F
:1094E0003F0B640DDB0F8D4218D08C4211D0002D44
:1094F00018D130438446002C1ED13A431CD1634618
:109500000020002B30D0514602200139084001389C
:109510002AE039001143EAD0022025E03043FBD194
:10952000AC4226D0002C26D13A4324D15146022009
:1095300001390840013817E06246002A0FD09A45E9
:10954000E1D1A54205DBBE42DDD819D00020BE42E4
:109550000AD25046012301389843013004E0012229
:10956000013B9343180001301CBC90469946A2462B
:10957000F0BD3A43D0D19A45C5D1A542C3DCE0E75E
:10958000C845C0D80020C845E3D3EDE7FF07000079
:10959000F0B55746DE464E464546E0B583460600E2
:1095A0000F03480087B092461D003F0B400DCC0FC3
:1095B000002800D16FE0DE4B984238D08023FF00B6
:1095C0001B041F43730F3B430193DA4B002799465B
:1095D00000239B46F60081442B0369001B0B524677
:1095E0009846490DED0F002900D185E0D04B9942F6
:1095F00000D173E04346DA0080231B041343524634
:10960000CC48520F84461343524600206144D20096
:1096100089442100694000918C46012149448A46D1
:109620000F2F00D990E0C449BF00CF59BF465B4619
:109630003B43019300D06AE10223082700268146BC
:109640009B46C9E732005846019B614600910228BB
:1096500000D175E0032800D1FEE1012800D02CE103
:1096600000230027002600253F032A0D3F0BB348A7
:1096700012053A4302401B051343009A5B00D107D1
:109680005B080B433000190007B03CBC904699467C
:10969000A246AB46F0BD5B463B43019300D12FE1B0
:1096A000002F00D1A5E1380000F00AFE03000B3BBB
:1096B0001C2B00DD96E11D22D31A5A460100DA4028
:1096C0005E4608398F4013008E403B4301939C4B0C
:1096D00000271B1A994600239B467DE741465346C7
:1096E0000B4393498C46E144002B00D01AE102223F
:1096F0000220174300228CE7134300D10DE14346BB
:10970000002B00D181E1404600F0DAFD02000B3A67
:109710001C2A00DD72E10100434608398B4098465F
:109720001D239A1A5346D3401A0043461343524608
:109730008A404946081A824989468144002068E7E0
:109740007B4B002700268EE7140C1204120C11002C
:10975000370C3604350C794328008C462E006043C4
:109760006044834656432100300C80465846794376
:1097700040440291844506D98846802149028C469E
:10978000E044414602913604010C360C00048B463D
:1097900081191E0C1B041B0C0391190079438C4684
:1097A000280075436544A8465843050C4544774353
:1097B000A94203D9802149028C466744290C8C4672
:1097C00039000004000C2D042D186144AB440591B0
:1097D0005946049101990F043F0C080C390051437C
:1097E0004243904602008C46090C8B4662437C4300
:1097F00044445C44A04503D9802149028846424440
:10980000210C884661460904090C8C4639005943ED
:10981000434370437E430F0CF6182404BE1964447E
:1098200042448C46B34203D980235B0298464044AD
:10983000029B61469846049B370443449B46AB45D4
:10984000AD416B420D0405992D0C8C467F19674480
:10985000FD18A8465D462D19A542A44193466442D1
:10986000A446C344DC448F42BF4198459B41934585
:109870009241A445A4415B427F421F43360C5242B1
:109880006442BF192243BF18624638184302D20D02
:10989000039913436A020A43501E82416146ED0D4B
:1098A0002A434E023243D90100D4B3E001265008C6
:1098B00032400243DE0732435B08224C5444002C02
:1098C00062DD510709D00F201040042805D0101D7B
:1098D0009042924152429B180200D90104D5802443
:1098E0001948E400034054441848844200DD27E747
:1098F0005E075B02D2081F0B630516435B0DB2E6E1
:10990000002399460133042700269B4664E603237F
:10991000019781460C279B465EE6012201201743F2
:10992000002276E6032303201F43434671E6C04628
:10993000FF07000001FCFFFF78CE0000FFFF0F8053
:109940000DFCFFFFFF030000FFFFFFFEFE0700000E
:109950000023802700933F030026434B83E6019BAF
:109960003200A446584670E6AC466EE68027019960
:109970003F0339422DD03B422BD11F433F033F0BC6
:1099800000951600384B6EE601252D1B382D00DDA5
:1099900066E61F2D40DC35481C005044160082400E
:1099A0008440EE40501E824134431443EB40620732
:1099B00009D00F222240042A05D02200141D94420F
:1099C000804140421B181A023ED501230027002681
:1099D00049E68027019B3F031F433F033F0B009451
:1099E000214B40E603005A46283B9A40002601924C
:1099F0006DE6584600F064FC203057E603005246FE
:109A0000283B9A401300002293E6504600F058FC91
:109A100020307BE6CA4650E71F201E004042041B50
:109A2000E640202D03D0124C5444A3401A43501E4C
:109A30008241324307260027164009D00F20002319
:109A4000104014000428B9D122005E075B021F0BEE
:109A5000D2081643002306E680273F031F433F0337
:109A60003F0B1600004BFEE5FF0700001E04000040
:109A70003E040000F8B557464E464546DE460C000B
:109A80000903E0B5490A460F5F0031431E03DB0FAF
:109A9000760A9B46530F3343C84E6500C000E40F5F
:109AA000D2006D0DA24681467F0D9C469046B7427E
:109AB00000D1B9E05B46012673409B46EE1BA345EF
:109AC00000D183E0002E63DD002F00D0B1E06346BB
:109AD000134300D123E1731E002B00D0BAE1861A94
:109AE0006346B04280410125C91A4042091A0B025F
:109AF00000D447E149024B0A98464346002B00D167
:109B000089E1404600F0DCFB0300083B1F2B00DD31
:109B10007CE120223000D21A4146D0409940020018
:109B20009E400A439D4200DD6AE15D1B6B1C1F2BBA
:109B300000DD94E1202110003500C91A8E40DA4082
:109B40008840DD40711E8E41110007222843002508
:109B500006433240002A09D00F233340042B05D09E
:109B6000331DB342B641764289191E000B0200D460
:109B70003DE26A1C914B55056D0D9A4200D119E1E9
:109B80008F4AF6080A40570752023743120B9BE0F0
:109B9000002E00D0C5E06E1C7605760D012E00DC8F
:109BA00048E16746861ACB1BB042BF417F42B846A8
:109BB0001F004346FF1A3B00B8461B0200D55FE179
:109BC00037439AD100220024002579E0002E00DCE2
:109BD000FAE0002F00D18DE0784B9D4267D08023C2
:109BE00067461B041F43BC46382E00DC52E1634627
:109BF00013435A1E93411E18864280414042091861
:109C00000B0200D4BEE06D4B01359D4200D1D2E085
:109C10006B4A73080A4001210E401E435108D307C6
:109C200007221E43324095E71E00164300D045E749
:109C300040E7624B9D423AD0802367461B041F4396
:109C4000BC46382E00DDEBE01F2E00DC3AE133008D
:109C50006746203BDF403B00202E05D04027BF1B3E
:109C60006646BE40324390464646721E9641334396
:109C7000DAE0002B00D114E26346134300D168E11F
:109C800080234E07C008C9081B030643194208D0A9
:109C90006046C008184204D163460100D2085E073E
:109CA0001643F3009946C900720F444D11434B46C9
:109CB000DE08424B4F073743CA089D4200D16EE091
:109CC00012036D05120B6D0D00211203130B0A0D0B
:109CD00012051A433B4B2D0513402B435B00E40751
:109CE0005B082343380019003CBC90469946A246C5
:109CF000AB46F8BD6346134311D0731E002B00D052
:109D000007E18618864280416144404209180125D6
:109D10000B0237D502257BE73E00614691463500B0
:109D2000C5E75C46002D00D0E1E00B000343F3D013
:109D3000731C00D1ACE1214B9F4200D13AE1F343C7
:109D4000382B00DD6FE11F2B00DD8CE120250E009C
:109D5000ED1AAE40B0460600AA46DE404546354301
:109D60002E005546D940A8406346451EA8415B1ABF
:109D70009C463043161AB242924163465242991AA7
:109D80003D00B4E607223240002A00D0E4E60B4B47
:109D9000F6084F073743CA089D4200D090E73B00C2
:109DA000134300D1A6E180231B031A431203120BB5
:109DB000024D89E715000022002785E7FF07000014
:109DC000FFFF7FFFFFFF0F80002E00D0C7E06B1C5E
:109DD0005E05760D012E00DCF0E0C84DAB4200D1EF
:109DE000B9E085180A008542894162444942511808
:109DF0000722CE076D082E43490832401D00A9E610
:109E0000BF49ED1A114007223240A3E6320028383C
:109E10008240002686E6300000F052FA203073E6D9
:109E2000634613435A1E9341C61AB04280414042D2
:109E3000091A5CE60E00674606431743002D5ED103
:109E4000002E00D0F3E0002F00D11EE15C466146F9
:109E500091462CE7A94FBE427BD01E00F1E61000D0
:109E60001F3DE840202B03D04021CB1A9A401643D7
:109E7000731E9E410722064332400021002583E7DE
:109E8000161A6346B2428041591A40420B1A98464C
:109E90005C4632E61F2E00DDABE02027BB1B9A4656
:109EA00063465746BB40994613004F46F3401F4355
:109EB0003B005746BA40571EBA4113436246F24030
:109EC000891898E62027BB1B9A4663465746BB4035
:109ED000994613004F46F3401F433B005746BA4094
:109EE000571EBA4113436246F240891A9CE7834BDE
:109EF0009F425FD080252D047342294320E7002E26
:109F00000CD1002F00D1D0E05C46614691467B4DDC
:109F1000CDE67A4FBE421CD01E0065E6002F18D059
:109F2000C0084E0706438020C9080003014208D03C
:109F30006346DC08044204D12100DA46D2085E07F9
:109F40001643F300994601245346C900720F11438A
:109F50001C406A4DABE61D0000220027B4E6002D30
:109F600059D10B00034300D1D6E6731C00D1B2E0F7
:109F7000624B9F421ED0F343382B6FDC1F2B00DD5A
:109F800097E020250E00ED1AAE40B0460600AA4626
:109F9000DE40454635432E005546A840D940451E73
:109FA000A8418C440643B6189642924151426144FE
:109FB0003D0025E63D006146914678E60B000343EF
:109FC000002D00D055E6002BF5D06346134300D199
:109FD0006DE686188642804161444042091800229D
:109FE0000B0200D4D0E6464B01351940B2E5B1462C
:109FF0005DE633006746203BDF403B00202E05D066
:10A000004027BF1B6646BE40324390464646721EFE
:10A0100096413343EFE5394B9F42CBD080252D0449
:10A0200073422943A8E70843411E8841A2E6002F56
:10A0300000D13CE66346861ACF1AB0429B415B4290
:10A04000FB1A98461B024ED5161A6346B24292413D
:10A05000591A5242891A5C4600227BE501430E00E0
:10A06000711E8E419FE71D000E00203DEE40B04660
:10A07000202B04D04025EB1A9940084381464846DE
:10A080004346411E8841184374E60022002417E627
:10A09000161A6346B2429241591A5242891A3D0039
:10A0A00025E561469146154D01E680220024120304
:10A0B00079E61D000E00203DEE40B046202B04D076
:10A0C0004025EB1A9940084381464E464346711E8F
:10A0D0008E411E4367E7861896429B4161445B426E
:10A0E000C9183D008CE547463743CED0072241468C
:10A0F000324049E600273A00E6E5C046FF07000087
:10A10000FFFF7FFF70B50C4E0D031C0349005B0081
:10A110002D0B490D240B5B0DB14208D006490020E0
:10A120008B4203D114432000441EA04170BD05435F
:10A130000120002DFAD1F1E7FF07000030B5144DE2
:10A140000A034B00120B5B0DC90F0024AB4211DD5B
:10A15000104CA34210DC8024640322430E4CE41A0A
:10A160001F2C0CDD0D48C31ADA4013005C42002995
:10A1700000D11C00200030BD094BCC18FAE7094D76
:10A18000E040AC4663449A4013000343EEE7C04608
:10A19000FE0300001D04000033040000130400004F
:10A1A000FFFFFF7FEDFBFFFF70B500282DD0C31729
:10A1B000C5185D40C40F280000F082F8154B1B1A2B
:10A1C0005B055B0D0A2815DD0B38854000222D0349
:10A1D0002D0B002110002D030A0D2D0B12052A4313
:10A1E0000D4D1B052A4013435B00E4075B08234326
:10A1F000190070BD02002900153291400A000B21A0
:10A20000081AC5402D032D0BE3E700240023002589
:10A210000022DEE71E040000FFFF0F804100090E50
:10A220004B1C70B5DBB24602750AC40F012B14DD5E
:10A23000E0239B006D07360BCB1800210A0D280088
:10A2400012051C4D32435B052A405B0813435B003B
:10A25000E4075B082343190070BD002914D1002DC9
:10A260001ED0280000F02CF80A281CDC0B232A0042
:10A270001B1ADA40030015339D400F4B12031B1AC3
:10A280005B05160B5B0DD8E7002D06D0320B802640
:10A2900036036D071643094BCFE7084B0026CCE782
:10A2A00000230026C9E703002A000B3B9A40002543
:10A2B000E3E7C046FFFF0F8089030000FF070000AF
:10A2C0001C2101231B04984201D3000C10391B0AE6
:10A2D000984201D3000A08391B09984201D30009AA
:10A2E000043902A2105C40187047C0460403020201
:10A2F00001010101000000000000000030B51C0059
:10A30000094B05001B6885B0D868084B002A01D1AD
:10A31000074B1A000292019300912B00220005497D
:10A3200000F026F800F08EFD6C000020B8CE000092
:10A33000CFBD0000C5CE0000014B18687047C04675
:10A340006C000020084B10B50400002B02D0002147
:10A3500000E000BF054B1868836A002B00D09847C7
:10A36000200001F045FBC04600000000F4CE0000D4
:10A370000EB403B5010003AB044804CB006801939D
:10A3800000F076F802B008BC03B018476C0000205B
:10A3900070B500260C4D0D4C641BA410A64209D1CB
:10A3A000002601F027FB0A4D0A4C641BA410A642AC
:10A3B00005D170BDB300EB5898470136EEE7B30006
:10A3C000EB5898470136F2E73C0200203C0200209F
:10A3D0003C0200204C020020002310B59A4200D11C
:10A3E00010BDCC5CC4540133F8E710B5884202D9E3
:10A3F0008B18984203D3002307E08B5C8354013A07
:10A40000FBD210BDCC5CC45401339A42FAD1F8E7B8
:10A4100003001218934200D1704719700133F9E715
:10A42000936810B5013B9360002B04DA9469A34252
:10A4300007DB0A2905D01368581C10601970080042
:10A4400010BD00F033FC0100F9E7F8B506000F007D
:10A450001400D518AC4201D1002007E021783A0061
:10A460003000FFF7DDFF0134431CF3D1F8BD0000DD
:10A47000F0B59FB002900F0016000593002805D09C
:10A4800083690493002B01D100F0DCFD7B4B9F42DC
:10A490005BD1029B5F68BB891B0762D53B69002BC0
:10A4A0005FD0002306AC6361203363761033A3765C
:10A4B00035002B78002B01D0252B5CD1AB1B0493EE
:10A4C0000CD0320039000298FFF7BFFF431C00D1C7
:10A4D000C4E06269049B9446634463612B78002B5B
:10A4E00000D1BBE0012200235242626002A9543233
:10A4F00052186E1C2360E360A3601370A36531786B
:10A5000005225F4800F0BCFE751C002835D122688A
:10A51000D30604D5532302A95B1820211970130711
:10A5200004D5532302A95B182B21197033782A2BE9
:10A530002CD0350000210A20E3682A786E1C303ABE
:10A54000092A64D900292ED026E04E4B9F4202D121
:10A55000029B9F689FE74C4B9F429CD1029BDF6808
:10A5600099E73900029800F0F7FB002899D0012004
:10A5700040421FB0F0BD01359BE7414B2268C01A35
:10A5800001238340134323602E00B8E7059B191D68
:10A590001B680591002B01DB099304E05B42E3603B
:10A5A0000223134323602B782E2B0AD16B782A2B9E
:10A5B00035D1059B02351A1D1B680592002B2BDB3C
:10A5C0000793324E29780322300000F059FE00280C
:10A5D00006D04023801B834022680135134323604B
:10A5E000297806222A486E1C217600F049FE0028B0
:10A5F0003AD0284B002B25D10722059B07339343E4
:10A60000083305936369039A9B18636150E74343DA
:10A6100001219B18350090E701235B42D0E700231E
:10A620000A201A000135636029786E1C3039092927
:10A6300003D9002BC5D00792C3E742430123521828
:10A640003500F1E705AB00933A00134B2100029867
:10A6500000E000BF0390039B0133D3D1BB895B06AD
:10A6600000D584E70B9884E705AB00933A000A4BCA
:10A670002100029800F080F8ECE7C0464CCF0000C3
:10A68000F8CE00006CCF00002CCF0000FECE000002
:10A6900002CF0000000000004BA40000F7B5150039
:10A6A00001938A680B6900900C00934200DA130052
:10A6B00022002B6043321278002A01D001332B6034
:10A6C00023689B0602D52B6802332B60062723687C
:10A6D0001F4027D0230043331B785A1E9341226822
:10A6E000920630D42200019943320098089EB04768
:10A6F000431C25D0062320682A68E1680340002512
:10A70000042B03D18D1AEB43DB171D40A36822698C
:10A71000934201DD9B1AED180027BD4220D1002095
:10A7200010E00137E3682A689B1ABB42D2DD2200A1
:10A730000123193201990098089EB047431CF0D1BB
:10A7400001204042FEBD3020E11843310870210055
:10A750005A1C45310978A218433202331170C1E7FF
:10A76000220001231A3201990098089EB047431C29
:10A77000E6D00137D1E70000F0B589B004920A00B5
:10A7800043320593039002920A7E0C000E9B6E2AC0
:10A7900000D186E01FD8632A33D008D8002A00D120
:10A7A0008CE0582A4DD0250042352A7030E0642ACA
:10A7B00001D0692AF7D1196825680A1D280629D50C
:10A7C00008681A60002803DA2D23029A40421370A9
:10A7D0006B4E0A274FE0732A74D008D86F2A1FD017
:10A7E000702AE0D1202209680A43226003E0752A1A
:10A7F00016D0782AD7D12200782145321170614EC7
:10A8000022E025001A684235111D196013682B706B
:10A81000012365E008681A606906D3D500B2D1E764
:10A8200019682568081D186008682E0605D5544E5D
:10A8300008276F2A1BD00A2719E06D06F7D580B2CA
:10A84000F5E745314E4E0A7018682268011D006810
:10A850001960150621D5D30702D520231A4322609B
:10A860001027002803D1202322689A432260230066
:10A87000002243331A706368A360002B58DB042264
:10A88000216891432160002854D1029D002B5AD0A9
:10A890002500337842352B7055E05506DBD580B264
:10A8A000D9E71A680D68101D4969186013682E06EB
:10A8B00001D5196002E06D06FBD519800023029DC9
:10A8C00023614FE01A68111D196015680021626844
:10A8D000280000F0D5FC002801D0401B60606368B0
:10A8E00023610023029A13703CE023692A00049933
:10A8F0000398059DA847431C3ED023689B0715D4A9
:10A90000079BE068984239DA180037E022000123FB
:10A91000193204990398059EB047431C2CD0013589
:10A92000E368079A9B1AAB42F0DCE9E70025F7E7FA
:10A930000028ADD0029D3900FDF722FC735C013D7B
:10A940002B700028F7D1082F09D12368DB0706D523
:10A9500063682269934202DC3023013D2B70029B25
:10A960005B1B2361059B07AA00932100049B0398AE
:10A97000FFF794FE431CB8D10120404209B0F0BD5E
:10A9800009CF00001ACF00000D4B70B51C68050000
:10A99000A36B002B0FD1182000F056FC094BA063CD
:10A9A0000360094B01224360084B83600B238381C2
:10A9B0000023026143610022A36B1D615A6170BDD7
:10A9C0006C0000200E33CDAB34126DE6ECDE0500DA
:10A9D000124B10B51C68A36B002B0FD1182000F090
:10A9E00033FC0F4BA06303600E4B012243600E4B00
:10A9F00083600B238381002302614361A46B0B4AB4
:10AA0000206961690A4BFDF7F7FC012200238018D9
:10AA10005941206161614800400810BD6C00002070
:10AA20000E33CDAB34126DE6ECDE05002D7F954C78
:10AA30002DF451580CB430B5164B9DB00C1E1D684A
:10AA400008DA8B2301202B6040421DB030BC08BCCB
:10AA500002B01847822302A99B008B810023029039
:10AA600008619C4200D0631E8B604B6101235B42F6
:10AA7000CB81209A21AB2800019300F03DFD431CBF
:10AA800001DA8B232B60002CDFD00023029A137095
:10AA9000DBE7C0466C0000200EB400B50B499CB04B
:10AAA0001DAB02900690079104910948094904CB17
:10AAB0000591006802A9019300F01EFD0023029A8F
:10AAC00013701CB008BC03B01847C046FFFFFF7FDF
:10AAD0006C0000200802FFFF020010B51378541C20
:10AAE000002B05D1CC5CD4540133002CFAD110BD1D
:10AAF0002200F3E702780B78002A03D001300131FD
:10AB00009A42F7D0D01A704703000A7801311A70C0
:10AB10000133002AF9D170470023C25C0133002AB7
:10AB2000FBD1581E704730B50500002A00D130BD5A
:10AB30000C78013A6B1C2C700131002C05D19A184D
:10AB40009A42F4D01C700133FAE71D00EDE710B50E
:10AB50000378002B0FD10B785A4253415B421840C7
:10AB600010BD0023CA5C002AFAD0C45C944201D113
:10AB70000133F7E701300378002BF2D11800EFE73B
:10AB8000F0B51F000E0087B00590019102920C985D
:10AB9000347800F0EAFA082200194378751C134053
:10ABA00036D12D2C36D1B51C74780126002F62D0F9
:10ABB000102F09D1302C07D120222B789343582B0A
:10ABC00054D110276C7802352D4B3900F31818003A
:10ABD0000393FDF7D5FA04910121002349420200B5
:10ABE0008C4618002100303909291AD80C00A742D8
:10ABF00023DD591C09D06346824206D302D1049951
:10AC0000A14202DB0123784320182C780135E9E7C3
:10AC10002E00BCE72B2C01D01E00C7E7B51C7478B2
:10AC2000FAE721004139192901D8373CDFE7210033
:10AC30006139192901D8573CD9E75A1C08D1059A1E
:10AC400023331360029B0398002B09D107B0F0BD9A
:10AC5000002E00D04042029A002AF7D0002B01D0EB
:10AC60006B1E0193029B019A1A60EFE73024002FBC
:10AC7000AAD10827A8E7302C9ED00A27A4E7C0460F
:10AC8000FFFFFF7F37B51300064A05001068046A0E
:10AC9000002C00D1044C0A0000942900FFF770FF3B
:10ACA0003EBDC0466C000020D0000020F8B5050075
:10ACB0000E001400002804D08369002B01D100F09D
:10ACC000C1F9224B9C422DD16C68A369A360A38972
:10ACD0001B0731D52369002B2ED023682269F7B2D8
:10ACE000981A6369F6B2834205DC2100280000F05F
:10ACF0003BF9002826D1A3680130013BA3602368FB
:10AD00005A1C22601F706369834204D0A389DB0749
:10AD10001AD50A2E18D12100280000F025F90028A4
:10AD200012D00FE00A4B9C4201D1AC68CDE7094B31
:10AD30009C42CAD1EC68C8E72100280000F00CF85A
:10AD40000028CAD0012676423000F8BD4CCF000062
:10AD50006CCF00002CCF0000364B70B51D6806008C
:10AD60000C00002D05D0AB69002B02D1280000F0AB
:10AD700069F9314B9C420FD16C680C23E25E93B2AF
:10AD800019072DD4D90611D4092301203360373394
:10AD90001343A381404270BD284B9C4201D1AC6853
:10ADA000EBE7274B9C42E8D1EC68E6E75B0713D55D
:10ADB000616B002908D023004433994202D030004F
:10ADC00000F06AFA002363632422A3899343A381DA
:10ADD00000236360236923600823A2891343A381AE
:10ADE0002369002B0BD1A0218022A3898900920026
:10ADF0000B40934203D02100300000F0E1F9012321
:10AE0000A289134011D00023A36063695B42A36150
:10AE1000002023698342BED10C23E25E1306BAD51B
:10AE200040231343A3810138B5E7920700D4636937
:10AE3000A360EDE76C0000204CCF00006CCF000059
:10AE40002CCF000010B5062000F090FC012000F08F
:10AE5000CFFD0000F7B58A8905000C00130760D408
:10AE60004B68002B04DC0B6C002B01DC0020FEBDCA
:10AE7000E76A002FFAD000232E682B6080235B0145
:10AE8000216A1A4034D0606DA3895B0706D56368D8
:10AE9000C01A636B002B01D0236CC01A0200216A18
:10AEA00000232800E76AB847A189431C06D12B6814
:10AEB0001D2B30D82B4ADA40D3072CD500236360F2
:10AEC00023692360CB0405D5431C02D12B68002BDA
:10AED00000D16065616B2E600029C7D02300443328
:10AEE000994202D0280000F0D7F900206063BEE745
:10AEF00001232800B847431CC6D12B68002BC3D0C0
:10AF00001D2B01D0162B01D12E60AFE74023A28963
:10AF10001343A381ABE740230B430120A3814042AD
:10AF2000A5E70F69002FA1D00B680F60DB1B019311
:10AF30000023920700D14B69A360019B002B00DC2A
:10AF400094E7019B3A00216A2800A66AB0470028CE
:10AF500003DC4023A2891343DFE7019B3F181B1A40
:10AF60000193EAE7010040200B6970B505000C0071
:10AF7000002B01D1002070BD002804D08369002B74
:10AF800001D100F05FF80B4B9C4209D16C680C2298
:10AF9000A35E002BEED021002800FFF75BFFEAE75D
:10AFA000054B9C4201D1AC68F1E7044B9C42EED1C9
:10AFB000EC68ECE74CCF00006CCF00002CCF000019
:10AFC000002310B504000360436083608181436601
:10AFD000C281036143618361190008225C30FFF77D
:10AFE00017FA054B24626362044BA362044BE362CD
:10AFF000044B236310BDC046ADB70000D5B70000B9
:10B000000DB8000039B8000010B5024900F08CF806
:10B0100010BDC04669AF000070B568254A1E554393
:10B020000E002900743100F081F9041E08D00021BF
:10B030002A00016046600C30A0606832FFF7E8F932
:10B04000200070BD836913B50400002B28D18364F0
:10B05000C3640365134B144A1B68826201939842D0
:10B0600001D101238361200000F020F860602000FE
:10B0700000F01CF8A060200000F018F80022E0604A
:10B0800004216068FFF79CFF01220921A068FFF7F7
:10B0900097FF02221221E068FFF792FF0123A361CC
:10B0A00013BDC046F4CE000009B00000F8B51C4B3B
:10B0B00007001E68B369002B02D13000FFF7C2FF02
:10B0C0004836B4687368013B04D53368002B07D059
:10B0D0003668F6E70C22A55E002D0DD06834F2E745
:10B0E00004213800FFF798FF30600028F0D10C23CE
:10B0F00004003B602000F8BD20000A4B6566256017
:10B100006560A560E36025616561A561082229008D
:10B110005C30FFF77DF96563A563A564E564E9E745
:10B12000F4CE00000100FFFFF7B504000700002681
:10B1300001914834002C01D13000FEBD6368A56840
:10B140000093009B013B009301D52468F2E7AB8993
:10B15000012B08D90E22AB5E013304D02900380040
:10B16000019B984706436835EBE7EC300068704771
:10B1700070B50E001D000E23C95E96B014000029A4
:10B1800007DA00232B60B3891B0611D48023DB0070
:10B190000FE06A4600F088FB0028F2DBF022019BFA
:10B1A00012021340054A9B185A4253412B60EDE7A7
:10B1B00040230020236016B070BDC04600E0FFFFB2
:10B1C000F7B502268B8905000C00334206D0230018
:10B1D00047332360236101236361F7BD01AB6A46F6
:10B1E000FFF7C6FF00990700280000F09FF800282D
:10B1F00008D10C22A35E9A05EFD4032293431E4389
:10B20000A681E4E70F4BAB628023A2892060134341
:10B21000A381009B20616361019B002B0DD00E2355
:10B22000E15E280000F052FB002806D00322A3892B
:10B2300093431A0001231343A381A0893843A081BB
:10B24000CBE7C04609B0000010B5034B01001868F9
:10B2500000F06CF810BDC0466C00002082B00029E0
:10B2600000D101A9101E06D0002B06D013780B6068
:10B270001078431E984102B0704702204042FAE71E
:10B28000C9B28218904201D10020704703788B42E6
:10B29000FBD00130F6E7000070B50500002910D0A2
:10B2A0000C1F2368002B00DAE418280000F034FBA0
:10B2B0001D4A1368002B05D163601460280000F05C
:10B2C0002CFB70BDA34209D9216860188342F3D1D9
:10B2D00018685B6841182160EEE713005A68002A7D
:10B2E00001D0A242F9D919685818A0420BD12068A0
:10B2F0000918581819608242E0D110685268411844
:10B3000019605A60DAE7A04202D90C232B60D5E716
:10B3100021686018824203D1106852684118216088
:10B3200062605C60CAE7C046EC1B0020032370B576
:10B33000CD1C9D43083506000C2D1ED20C25A942BC
:10B340001DD8300000F0E8FA254A146821000029D1
:10B3500019D1244C2368002B03D1300000F0CAF926
:10B3600020602900300000F0C5F9431C2BD10C23CC
:10B370003000336000F0D1FA03E0002DDFDA0C2357
:10B380003360002070BD0B685B1B19D40B2B03D9F5
:10B390000B60CC18256003E04B688C420DD1136024
:10B3A000300000F0BAFA200007220B30231D904332
:10B3B000C31AE7D05A42E250E4E763600C00EFE7BB
:10B3C0000C004968C3E70323C41C9C43A042E1D09E
:10B3D000211A300000F08EF9431CDBD1C7E7C046CC
:10B3E000EC1B0020F01B0020F8B507000D00160034
:10B3F000002905D11100FFF799FF04002000F8BDD6
:10B40000002A03D1FFF748FF3400F7E700F086FA7F
:10B410002C00B042F2D231003800FFF787FF041E43
:10B42000ECD029003200FEF7D7FF29003800FFF7E3
:10B4300033FFE3E7F0B58E6885B007000C00039298
:10B4400001939E423CD890238A89DB001A4234D073
:10B450000325096923685B1A0293636902985D43B7
:10B46000EB0F5D19019B6D1001331B18AB4200D926
:10B470001D00530532D529003800FFF757FF061E7F
:10B4800009D10C233B6040230120A2894042134391
:10B49000A38105B0F0BD029A2169FEF79DFFA38943
:10B4A000144A1A4080231343A381029B2661F61895
:10B4B00026606561019EED1AA560019B9E4200D940
:10B4C000019E320003992068FEF78FFFA3680020D9
:10B4D0009B1BA36023689E192660DAE72A003800C8
:10B4E000FFF782FF061EE0D121693800FFF7D4FE86
:10B4F000C7E7C0467FFBFFFFF0B59FB00290059302
:10B500008B890F0016001B0611D50B69002B0ED17D
:10B510004021FFF70BFF38603861002805D10C236C
:10B52000029A013813601FB0F0BD40237B610023F5
:10B5300006AC6361203363761033A37635002B7835
:10B54000002B01D0252B46D1AB1B04930CD032002D
:10B5500039000298FFF76EFF431C00D1AEE062692C
:10B56000049B9446634463612B78002B00D1A5E0D3
:10B57000012200235242626002A9543252186E1C0A
:10B580002360E360A3601370A365317805225448FB
:10B59000FFF776FE751C00281FD12268D30604D55C
:10B5A000532302A95B1820211970130704D55323D4
:10B5B00002A95B182B21197033782A2B16D035007D
:10B5C00000210A20E3682A786E1C303A092A4ED9F5
:10B5D000002918D010E00135B1E7414B2268C01AAC
:10B5E00001238340134323602E00CEE7059B191DE2
:10B5F0001B680591002B01DB099304E05B42E360CB
:10B600000223134323602B782E2B0AD16B782A2B2D
:10B6100035D1059B02351A1D1B680592002B2BDBCB
:10B620000793304E297803223000FFF729FE0028C7
:10B6300006D04023801B83402268013513432360DA
:10B640002978062228486E1C2176FFF719FE00286B
:10B650003CD0264B002B25D10722059B0733934373
:10B66000083305936369039A9B18636166E7434354
:10B6700001219B183500A6E701235B42D0E7002398
:10B680000A201A000135636029786E1C30390929B7
:10B6900003D9002BC5D00792C3E7424301235218B8
:10B6A0003500F1E705AB00933A00114B21000298F9
:10B6B00000E000BF0390039B0133D3D1BB890B98FB
:10B6C0005B0600D42FE7012040422CE705AB009336
:10B6D0003A00074B21000298FFF74EF8EAE7C04610
:10B6E000F8CE0000FECE000002CF000000000000F7
:10B6F00035B40000002370B5064C05000800236037
:10B7000000F060F9431C03D12368002B00D02B60AC
:10B7100070BDC046A42F002070B504000D001F2985
:10B7200004D9162303600120404270BD436C002BF6
:10B7300004D08A009B181A68002A08D1200000F063
:10B7400031F82A000100200000F01AF8EDE700208F
:10B75000012AEAD0511C03D1162301302360E4E70B
:10B76000002428001C6090472000DEE710B5034B42
:10B7700001001868FFF7D0FF10BDC0466C00002024
:10B78000002370B5064C050008001100236000F08E
:10B7900001F9431C03D12368002B00D02B6070BD3E
:10B7A000A42F002010B500F0E5F810BD70B50C0016
:10B7B0000E25495F00F0BAF8002803DB636D1B1803
:10B7C000636570BDA389024A1340A381F9E7C046AF
:10B7D000FFEFFFFFF8B51F008B8905000C00160076
:10B7E000DB0505D50E23C95E0022022300F080F898
:10B7F000A389054A28001340A38132000E23E15E8D
:10B800003B0000F02BF8F8BDFFEFFFFF70B50C0018
:10B810000E25495F00F06CF8A389421C03D1054A4C
:10B820001340A38170BD802252011343A381606540
:10B83000F8E7C046FFEFFFFF10B50E23C95E00F02A
:10B8400021F810BD0B1E04D0FF2A04D98A230360FF
:10B850008B3B180070470A700123FAE770B50500AA
:10B86000080011000022064C22601A0000F0B8F80F
:10B87000431C03D12368002B00D02B6070BDC04651
:10B88000A42F0020002370B5064C0500080023609B
:10B8900000F060F8431C03D12368002B00D02B601C
:10B8A00070BDC046A42F0020002370B5064C0500D3
:10B8B00008001100236000F055F8431C03D12368F1
:10B8C000002B00D02B6070BDA42F0020002370B58A
:10B8D000064C05000800236000F054F8431C03D117
:10B8E0002368002B00D02B6070BDC046A42F002021
:10B8F00070B50500080011000022064C22601A00F5
:10B9000000F050F8431C03D12368002B00D02B60BB
:10B9100070BDC046A42F0020704770470B1F1B68E6
:10B92000181F002B01DA0B58C018704770B50500BE
:10B93000080011000022064C22601A0000F03AF8BC
:10B94000431C03D12368002B00D02B6070BDC04680
:10B95000A42F002058220120014B40421A6070475A
:10B96000A42F002058220120014B40421A6070474A
:10B97000A42F002058220120014B40421A6070473A
:10B98000A42F00205822024B00201A607047C046A6
:10B99000A42F002058220120014B40421A6070471A
:10B9A000A42F002058220120014B40421A6070470A
:10B9B000A42F002058220120014B40421A607047FA
:10B9C000A42F0020044A1368002B00D1034B181841
:10B9D000106018007047C046F41B0020A82F0020FC
:10B9E00058220120014B40421A607047A42F0020CA
:10B9F000FEE7C046F8B5C046F8BC08BC9E46704796
:10BA0000F8B5C046F8BC08BC9E46704764617461D6
:10BA10000000000088BA0000EB01000091BA0000AD
:10BA20001704000099BA00002D070000A0BA00001A
:10BA30003D080000A5BA0000DF020000B0BA000017
:10BA400083040000B5BA0000B5090000C1BA0000C7
:10BA50001B020000CBBA000035060000D9BA000076
:10BA6000A105000072616E646F6D00616C6C006C0A
:10BA70006173740066616C7365007472756500258E
:10BA80002E3135732E2E2E006D616B654C697374EB
:10BA9000006164644C6173740064656C6574650076
:10BAA0006A6F696E00636F707946726F6D546F00D4
:10BAB00066696E64006A6F696E537472696E67734B
:10BAC00000756E69636F6465417400756E69636FBC
:10BAD0006465537472696E6700667265654D656D65
:10BAE0006F727900CC0F0000DC0F0000F60F000031
:10BAF00074100000AC100000E21000001A110000E9
:10BB0000401100007C110000BE1100001412000062
:10BB100058120000C41200000C1300003213000081
:10BB20006A130000B0130000D613000004140000D4
:10BB3000361400006E140000F2140000BA15000064
:10BB4000301600009C160000F016000010170000D0
:10BB500032170000E41700002A180000A2180000A5
:10BB6000CC0F0000CC0F0000D018000038190000E6
:10BB7000BC190000021A00004A1A0000BC1A00009A
:10BB80002E1B0000761B0000BC1B0000F21B0000F7
:10BB9000381C00007E1C0000C61C00001A1D00009E
:10BBA000781D0000B61D0000201E0000561E00007B
:10BBB0009E1E0000E61E00002E1F0000681F0000F1
:10BBC000B01F0000F81F0000CC0F0000CC0F0000D9
:10BBD000CC0F000060200000CC0F00009620000079
:10BBE000C2200000F820000024210000CC0F00003B
:10BBF000CC0F0000CC0F0000CC0F00005A21000039
:10BC0000A6210000CC0F0000CC0F0000EC210000AA
:10BC10003C22000062220000CC0F0000CC0F00008C
:10BC2000CC0F000090220000C0220000F022000093
:10BC3000262300005023000086230000B0230000CC
:10BC4000D8230000002400003024000060240000FD
:10BC50008A240000B4240000E42400000E25000023
:10BC6000CC0F0000CC0F0000CC0F0000CC0F000068
:10BC7000CC0F00003E25000084250000B025000008
:10BC8000DC250000082600003E2600007426000087
:10BC9000AA260000E02600000C270000382700003C
:10BCA0006E270000CC0F0000CC0F0000CC0F00006E
:10BCB000CC0F0000CC0F0000CC0F0000CC0F000018
:10BCC000CC0F0000CC0F0000CC0F0000CC0F000008
:10BCD000CC0F0000CC0F0000CC0F00009A27000012
:10BCE000D0270000282564206974656D206C697375
:10BCF000742900286F626A65637420747970653AEC
:10BD00002025642900537461636B20756E6465722D
:10BD1000666C6F7700000000070000000300000061
:10BD200062BD0000B52800006ABD0000B92800000F
:10BD300073BD0000B12800007CBD0000BD280000DC
:10BD400000000000010000000200000003000000ED
:10BD5000040000000A0000006D6963726F3A6269B6
:10BD60007400686173546F6E6500706C6179546F14
:10BD70006E6500686173536572766F007365745306
:10BD80006572766F00474320746F6F6B20256420C7
:10BD900075736563733B2066726565202564207743
:10BDA0006F726473003C496E74656765723E003C57
:10BDB0004F626A6563743E003C4C6973743E000DCB
:10BDC0000A564D2050616E69633A2025730D0A00B2
:10BDD0006D69736300000000E8BD00007D31000064
:10BDE000F1BD000035310000686578546F496E740C
:10BDF0000073696E0000000044BE0000E9310000DD
:10BE00004CBE0000ED31000056BE00000B320000B9
:10BE10005FBE0000153200006ABE00001F32000045
:10BE200076BE00002932000087BE000033320000D9
:10BE30009DBE0000F7310000B6BE000001320000D8
:10BE40006E65740068617357694669007374617246
:10BE500074576946690073746F7057694669007753
:10BE6000696669537461747573006D7949504164F2
:10BE70006472657373007468696E67446573637296
:10BE8000697074696F6E00636C6561725468696E85
:10BE9000674465736372697074696F6E0061707076
:10BEA000656E64546F5468696E6744657363726944
:10BEB0007074696F6E00617070656E64546F546861
:10BEC000696E6750726F7065727479001A1B1C037B
:10BED000040607090A1718190000000000080808DE
:10BEE00000080A4A4000000A5FEA5FEA0ED92ED332
:10BEF0006E19324489330C924C924D0808000000B0
:10BF000004880808040804848488000A448A4000DD
:10BF1000048EC480000000048800000EC0000000F1
:10BF200000080001224488100C9252524C048C8468
:10BF3000848E1C824C901E1EC244924C06CA525FD4
:10BF4000E21FF01EC13E02448ED12E1FE244881033
:10BF50000ED12ED12E0ED12EC4880008000800006C
:10BF6000048004880244880482000EC00EC00804C5
:10BF70008244880ED126C0040ED135B36C0C925E7B
:10BF8000D2521C925C925C0ED010100E1C92525237
:10BF90005C1ED01C901E1ED01C90100ED013712E53
:10BFA00012525ED2521C8808081C1FE242524C12E8
:10BFB00054981492101010101E113B75B1311139A4
:10BFC00035B3710C9252524C1C925C90100C9252F0
:10BFD0004C861C925C92510ED00C825C1FE48484CF
:10BFE00084125252524C1131312A44113135BB71F5
:10BFF00012524C9252112A4484841EC488101E0E80
:10C00000C808080E10080482410EC242424E048A3B
:10C01000400000000000001F0804800000000ED255
:10C02000524F10101C925C000ED0100E02424ED2E5
:10C030004E0C925C900E06C81C88080ED24EC24C64
:10C0400010101C92520800080808024002424C10CE
:10C05000149814920808080806001B75B131001CDA
:10C06000925252000C92524C001C925C90000ED2E4
:10C070004EC2000ED010100006C8049808080EC862
:10C0800007001252524F0011312A4400113135BBC2
:10C0900000124C8C9200112A4498001EC4881E067F
:10C0A000C48C8486080808080818080C8818000042
:10C0B0000C8360000000000001000000020000008E
:10C0C000030000000400000005000000060000005E
:10C0D0000700000008000000090000000A0000003E
:10C0E0000B0000000C0000000D0000000E0000001E
:10C0F0000F000000100000001200000014000000FB
:10C1000016000000180000001A0000001C000000CB
:10C110001E00000020000000230000002600000098
:10C12000290000002C0000002F0000003200000059
:10C13000360000003A0000003E000000420000000F
:10C14000460000004B0000005000000055000000B9
:10C150005A00000061000000680000006F0000004D
:10C16000760000007D000000840000008B000000CD
:10C170009200000099000000A0000000A70000004D
:10C18000AE000000B5000000BC000000C3000000CD
:10C19000CA000000D1000000D8000000DF0000004D
:10C1A000E6000000ED000000F4000000FB000000CD
:10C1B000FF00000004C20000593200000FC200005E
:10C1C0008137000019C200009134000026C200002F
:10C1D000B13400002DC200000135000036C200005D
:10C1E0005135000042C200002D34000053C200004F
:10C1F0009136000060C200004D3700006469737022
:10C200006C6179006C696768744C6576656C006D6B
:10C2100062446973706C6179006D62446973706C1B
:10C2200061794F6666006D62506C6F74006D625587
:10C230006E706C6F74006D624472617753686170E8
:10C2400065006D625368617065466F724C65747409
:10C250006572006E656F506978656C53656E640039
:10C260006E656F506978656C53657450696E004EE9
:10C270006F7420656E6F75676820726F6F6D2065D3
:10C2800076656E20616674657220636F6D706163A0
:10C2900074696F6E00436F6D7061637465642046EE
:10C2A0006C61736820636F64652073746F72650AD4
:10C2B0002564206279746573207573656420282570
:10C2C00064252529206F6620256400426164207260
:10C2D00065636F726420666F756E64206475726941
:10C2E0006E6720696E697469616C697A6174696FDF
:10C2F0006E0025642025642025642028256420778D
:10C300006F72647329002564207265636F726473B1
:10C310002C20256420776F7264732C206D6178491E
:10C32000442025642C20636F6D70616374696F6EA7
:10C33000206379636C657320256400526573746FA4
:10C34000726564202564207363726970747300538E
:10C3500074617274656400726164696F000000004A
:10C36000EEC3000049410000FBC30000B9430000D8
:10C370000BC400005943000019C4000039450000F7
:10C3800024C400006141000034C40000D541000015
:10C3900048C400007141000057C400001B47000062
:10C3A00063C40000994600006CC400003D460000D4
:10C3B00077C400008545000082C40000C14500002C
:10C3C0008BC40000F545000094C4000085410000C6
:10C3D0006E756D626572006E6F6E65006F74686574
:10C3E00072007061697200737472696E67006469CB
:10C3F0007361626C65526164696F006D657373612E
:10C4000067655265636569766564007061636B6535
:10C410007452656365697665007061636B6574531A
:10C42000656E64007265636569766564496E7465FE
:10C430006765720072656365697665644D657373DF
:10C4400061676554797065007265636569766564D6
:10C45000537472696E670073656E64496E746567C4
:10C4600065720073656E64506169720073656E6415
:10C47000537472696E67007365744368616E6E65AC
:10C480006C0073657447726F757000736574506FDC
:10C49000776572007369676E616C537472656E675D
:10C4A0007468000000000000963007772C610EEEE3
:10C4B000BA51099919C46D078FF46A7035A563E9FB
:10C4C000A395649E3288DB0EA4B8DC791EE9D5E022
:10C4D00088D9D2972B4CB609BD7CB17E072DB8E721
:10C4E000911DBF906410B71DF220B06A4871B9F376
:10C4F000DE41BE847DD4DA1AEBE4DD6D51B5D4F4AF
:10C50000C785D38356986C13C0A86B647AF962FD13
:10C51000ECC9658A4F5C0114D96C0663633D0FFA60
:10C52000F50D088DC8206E3B5E10694CE44160D566
:10C53000727167A2D1E4033C47D4044BFD850DD250
:10C540006BB50AA5FAA8B5356C98B242D6C9BBDB63
:10C5500040F9BCACE36CD832755CDF45CF0DD6DC5E
:10C56000593DD1ABAC30D9263A00DE518051D7C805
:10C570001661D0BFB5F4B42123C4B3569995BACF90
:10C580000FA5BDB89EB802280888055FB2D90CC6B1
:10C5900024E90BB1877C6F2F114C6858AB1D61C12A
:10C5A0003D2D66B69041DC760671DB01BC20D29849
:10C5B0002A10D5EF8985B1711FB5B606A5E4BF9FD6
:10C5C00033D4B8E8A2C9077834F9000F8EA80996C9
:10C5D00018980EE1BB0D6A7F2D3D6D08976C649134
:10C5E000015C63E6F4516B6B62616C1CD83065854D
:10C5F0004E0062F2ED95066C7BA5011BC1F408822A
:10C6000057C40FF5C6D9B06550E9B712EAB8BE8B6A
:10C610007C88B9FCDF1DDD62492DDA15F37CD38CF3
:10C62000654CD4FB5861B24DCE51B53A7400BCA3F1
:10C63000E230BBD441A5DF4AD795D83D6DC4D1A423
:10C64000FBF4D6D36AE96943FCD96E34468867ADFA
:10C65000D0B860DA732D0444E51D03335F4C0AAA99
:10C66000C97C0DDD3C710550AA41022710100BBE9C
:10C6700086200CC925B56857B3856F2009D466B9E3
:10C680009FE461CE0EF9DE5E98C9D9292298D0B018
:10C69000B4A8D7C7173DB359810DB42E3B5CBDB7C5
:10C6A000AD6CBAC02083B8EDB6B3BF9A0CE2B60346
:10C6B0009AD2B1743947D5EAAF77D29D1526DB04FB
:10C6C0008316DC73120B63E3843B64943E6A6D0D46
:10C6D000A85A6A7A0BCF0EE49DFF099327AE000A91
:10C6E000B19E077D44930FF0D2A3088768F2011E24
:10C6F000FEC206695D5762F7CB67658071366C19BB
:10C70000E7066B6E761BD4FEE02BD3895A7ADA10DB
:10C71000CC4ADD676FDFB9F9F9EFBE8E43BEB717BC
:10C72000D58EB060E8A3D6D67E93D1A1C4C2D83846
:10C7300052F2DF4FF167BBD16757BCA6DD06B53FAC
:10C740004B36B248DA2B0DD84C1B0AAFF64A0336EB
:10C75000607A0441C3EF60DF55DF67A8EF8E6E316A
:10C7600079BE69468CB361CB1A8366BCA0D26F25B3
:10C7700036E2685295770CCC03470BBBB916022200
:10C780002F260555BE3BBAC5280BBDB2925AB42B15
:10C79000046AB35CA7FFD7C231CFD0B58B9ED92C2A
:10C7A0001DAEDE5BB0C2649B26F263EC9CA36A758F
:10C7B0000A936D02A906099C3F360EEB8567077246
:10C7C00013570005824ABF95147AB8E2AE2BB17BAD
:10C7D000381BB60C9B8ED2920DBED5E5B7EFDC7C34
:10C7E00021DFDB0BD4D2D38642E2D4F1F8B3DD688B
:10C7F0006E83DA1FCD16BE815B26B9F6E177B06F86
:10C800007747B718E65A0888706A0FFFCA3B066672
:10C810005C0B0111FF9E658F69AE62F8D3FF6B61FF
:10C8200045CF6C1678E20AA0EED20DD75483044EA1
:10C83000C2B30339612667A7F71660D04D4769492F
:10C84000DB776E3E4A6AD1AEDC5AD6D9660BDF4042
:10C85000F03BD83753AEBCA9C59EBBDE7FCFB247F5
:10C86000E9FFB5301CF2BDBD8AC2BACA3093B353DA
:10C87000A6A3B4240536D0BA9306D7CD2957DE54E3
:10C88000BF67D9232E7A66B3B84A61C4021B685DBC
:10C89000942B6F2A37BE0BB4A18E0CC31BDF055A35
:10C8A0008DEF022D416C6C207461736B7320737477
:10C8B0006F70706564007630373100202573202555
:10C8C00073004D656D6F727920636C65617265648C
:10C8D000004E6F2066726565207461736B20656E13
:10C8E000747269657300000030C90000615900006E
:10C8F0003DC90000F955000049C9000097590000E2
:10C900004FC90000A759000055C90000B7590000E1
:10C910005BC900002D56000065C90000C959000020
:10C920006DC900006D57000073656E736F72730000
:10C93000616363656C65726174696F6E0074656DC7
:10C9400070657261747572650074696C74580074F6
:10C95000696C74590074696C745A00746F756368FB
:10C9600052656164006932635265616400693263D3
:10C970005772697465000000ECC90000495A000054
:10C98000FAC900004D5A000003CA0000595A0000BD
:10C990000DCA00005D5A000016CA0000615A00006E
:10C9A0001BCA0000655A000020CA0000695A000036
:10C9B0002CCA00006D5A000033CA0000715A0000F2
:10C9C0003CCA0000755A000041CA0000795A0000B4
:10C9D0004CCA00007D5A000056CA0000515A00009F
:10C9E00060CA0000555A000074667400656E61628A
:10C9F0006C65446973706C6179006765745769642C
:10CA00007468006765744865696768740073657465
:10CA1000506978656C006C696E65007265637400BE
:10CA2000726F756E646564526563740063697263E6
:10CA30006C6500747269616E676C6500746578740A
:10CA400000746674546F756368656400746674542A
:10CA50006F7563685800746674546F756368590025
:10CA6000746674546F75636850726573737572651C
:10CA70000057656C636F6D6520746F204D6963723C
:10CA80006F426C6F636B73210000000000000000B8
:10CA900000000000115B0000CD5A0000F35A0000B6
:10CAA000FD5A0000075B0000F15A0000705F7370D0
:10CAB0006920213D204E554C4C002F686F6D652F2D
:10CAC00062726F6D61676F73612F2E706C61746637
:10CAD0006F726D696F2F7061636B616765732F662D
:10CAE00072616D65776F726B2D61726475696E6FBF
:10CAF0006E6F726469636E7266352F6C6962726103
:10CB0000726965732F5350492F5350492E637070CB
:10CB100000535049436C6173733A3A535049436C24
:10CB2000617373284E52465F5350495F5479706564
:10CB30002A2C2075696E74385F742C2075696E74A8
:10CB4000385F742C2075696E74385F74290000009A
:10CB500003000000020000000100000004000000CB
:10CB600005000000110000000C0000000B00000098
:10CB7000120000000A000000060000001A00000079
:10CB8000140000001700000016000000150000004F
:10CB900010000000FFFFFFFFFFFFFFFF000000008D
:10CBA0001E0000001900000018000000070000002F
:10CBB00008000000090000000D0000000E00000049
:10CBC0000F0000001C0000001B0000001D00000002
:10CBD00013000000000000000000000031610000B0
:10CBE00061680000B1610000C5610000BB61000028
:10CBF0002D61000021610000D16100004D61000045
:10CC00001D61000000000000000000000000304333
:10CC100000000000000030C3737172740000000057
:10CC2000FB21F93FFB2109407CD91240FB2119402F
:10CC30007A6A1F407CD92240BBFD2540FB21294058
:10CC40003A462C407A6A2F405C4731407CD93240CA
:10CC50009C6B3440BBFD3540DB8F3740FB213940B6
:10CC60001BB43A403A463C405AD83D407A6A3F406D
:10CC70004C7E40405C4741406C1042407CD9424071
:10CC80008CA243409C6B4440AC344540BBFD4540C6
:10CC9000CBC64640DB8F4740EB584840FB2149401C
:10CCA00083F9A200444E6E00FC291500D1572700DD
:10CCB000DD34F50062DBC0003C99950041904300F3
:10CCC0006351FE00BBDEAB00B761C5003A6E2400C5
:10CCD000D24D42004906E00009EA2E001C92D10024
:10CCE000EB1DFE0029B11C00E83EA700F5358200CF
:10CCF00044BB2E009CE98400B4267000417E5F0096
:10CD0000D6913900538339009CF439008B5F84003D
:10CD100028F9BD00F81F3B00DEFF97000F980500C3
:10CD2000112FEF000A5A8B006D1F6D00CF7E360069
:10CD300009CB2700464FB7009E663F002DEA5F00F3
:10CD4000BA277500E5EBC7003D7BF100F739070016
:10CD500092528A00FB6BEA001FB15F00085D8D00F4
:10CD6000300356007BFC4600F0AB6B0020BCCF00CC
:10CD700036F49A00E3A91D005E619100081BE600ED
:10CD800085996500A0145F008D40680080D8FF0081
:10CD900027734D0006063100CA561500C9A8730056
:10CDA0007BE260006B8CC00000000040FB21F93F7B
:10CDB000000000002D44743E000000809846F83CBE
:10CDC0000000006051CC783B00000080831BF039EC
:10CDD0000000004020257A38000000802282E336DF
:10CDE000000000001DF36935020000000300000090
:10CDF000040000000600000044850000EE840000EE
:10CE0000EE8400001C860000EA840000EA84000032
:10CE1000128600001C860000EA84000012860000D2
:10CE2000EA8400001C8600002086000020860000A6
:10CE3000208600002886000020900000928E0000CE
:10CE4000D68E00003A8E0000D68E0000C68F0000FD
:10CE5000D68E00003A8E0000928E0000928E000066
:10CE6000C68F00003A8E0000328E0000328E000025
:10CE7000328E0000D48F0000489700004A960000D0
:10CE80004A9600006899000044960000449600000D
:10CE900050990000689900004496000050990000E5
:10CEA00044960000689900005E9900005E990000B9
:10CEB0005E9900006C9900002C2066756E637469A1
:10CEC0006F6E3A2000617373657274696F6E202211
:10CED000257322206661696C65643A2066696C6519
:10CEE00020222573222C206C696E65202564257311
:10CEF00025730A0070000020232D302B2000686C61
:10CF00004C0065666745464700303132333435366C
:10CF100037383941424344454600303132333435A5
:10CF200036373839616263646566000000000000CE
:10CF300000000000000000000000000000000000F1
:10CF400000000000000000000000000000000000E1
:10CF500000000000000000000000000000000000D1
:10CF600000000000000000000000000000000000C1
:10CF700000000000000000000000000000000000B1
:10CF80000000000000000000000000004300504FBF
:10CF9000534958000020202020202020202028282D
:10CFA0002828282020202020202020202020202069
:10CFB00020202020208810101010101010101010A9
:10CFC00010101010100404040404040404040410D9
:10CFD0001010101010104141414141410101010167
:10CFE0000101010101010101010101010101010131
:10CFF000101010101010424242424242020202023D
:10D000000202020202020202020202020202020200
:10D0100010101010200000000000000000000000B0
:10D020000000000000000000000000000000000000
:10D0300000000000000000000000000000000000F0
:10D0400000000000000000000000000000000000E0
:10D0500000000000000000000000000000000000D0
:10D0600000000000000000000000000000000000C0
:10D0700000000000000000000000000000000000B0
:10D0800000000000000000000000000000000000A0
:0CD0900000000000000000000000000094
:08D09C006C30FF7F0100000071
:10D0A400FFFFFFFF40060000010000001800000021
:10D0B40019FCFFFFFFFFFFFFFF000000020000005C
:10D0C40003000000FFFFFFFF00000000010000005C
:10D0D4000000020001000000FFFFFFFF000000004D
:10D0E400020000000000040002000000FFFFFFFF38
:10D0F400000000000300000000000800030000001E
:10D104000A00000008000000010000007000002078
:10D11400000000004CCF00006CCF00002CCF0000BA
:10D1240000000000000000000000000000000000FB
:10D1340000000000000000000000000000000000EB
:10D1440000000000000000000000000000000000DB
:10D1540000000000000000000000000000000000CB
:10D1640000000000000000000000000000000000BB
:10D174004300000000000000000000000000000068
:10D18400000000000000000000000000000000009B
:10D194004300000000000000000000000000000048
:10D1A400000000000000000000000000000000007B
:10D1B4004300000000000000000000000000000028
:10D1C400000000000000000000000000000000005B
:10D1D4004300000000000000000000000000000008
:10D1E400000000000000000000000000000000003B
:10D1F40043000000000000000000000000000000E8
:10D20400000000000000000000000000000000001A
:10D2140043000000000000000000000000000000C7
:10D2240000000000000000000000000000000000FA
:10D2340043000000000000000000000000000000A7
:10D2440000000000000000000000000000000000DA
:10D2540045B800005DB200000000000094CF00005B
:10D2640086BA0000CFBD0000CFBD0000CFBD0000D6
:10D27400CFBD0000CFBD0000CFBD0000CFBD00007A
:10D28400CFBD0000CFBD0000FFFFFFFFFFFFFFFF8A
:10D29400FFFFFFFFFFFF0000010041534349490026
:10D2A400000000000000000000000000000000007A
:10D2B4000000000000000000000041534349490001
:10D2C400000000000000000000000000000000005A
:10D2D400000000000000000000000000E900000061
:10D2E400E55D00003D5F00007D640000C1000000BA
:0400000300005FF1A9
:00000001FF
